
UTS2.elf:     file format elf32-avr

Sections:
Idx Name          Size      VMA       LMA       File off  Algn
  0 .text         00002de4  00000000  00000000  00000094  2**1
                  CONTENTS, ALLOC, LOAD, READONLY, CODE
  1 .data         00000066  00802000  00002de4  00002e78  2**0
                  CONTENTS, ALLOC, LOAD, DATA
  2 .bss          00000296  00802066  00802066  00002ede  2**0
                  ALLOC
  3 .comment      0000005c  00000000  00000000  00002ede  2**0
                  CONTENTS, READONLY
  4 .note.gnu.avr.deviceinfo 00000044  00000000  00000000  00002f3c  2**2
                  CONTENTS, READONLY
  5 .debug_aranges 00000460  00000000  00000000  00002f80  2**3
                  CONTENTS, READONLY, DEBUGGING
  6 .debug_info   000112e6  00000000  00000000  000033e0  2**0
                  CONTENTS, READONLY, DEBUGGING
  7 .debug_abbrev 000056c6  00000000  00000000  000146c6  2**0
                  CONTENTS, READONLY, DEBUGGING
  8 .debug_line   00009334  00000000  00000000  00019d8c  2**0
                  CONTENTS, READONLY, DEBUGGING
  9 .debug_frame  00000fc0  00000000  00000000  000230c0  2**2
                  CONTENTS, READONLY, DEBUGGING
 10 .debug_str    00034712  00000000  00000000  00024080  2**0
                  CONTENTS, READONLY, DEBUGGING
 11 .debug_loc    000073b9  00000000  00000000  00058792  2**0
                  CONTENTS, READONLY, DEBUGGING
 12 .debug_ranges 00000530  00000000  00000000  0005fb50  2**3
                  CONTENTS, READONLY, DEBUGGING
 13 .debug_macro  0000ca44  00000000  00000000  00060080  2**0
                  CONTENTS, READONLY, DEBUGGING

Disassembly of section .text:

00000000 <__vectors>:
       0:	87 c2       	rjmp	.+1294   	; 0x510 <__ctors_end>
       2:	00 00       	nop
       4:	a6 c2       	rjmp	.+1356   	; 0x552 <__bad_interrupt>
       6:	00 00       	nop
       8:	a4 c2       	rjmp	.+1352   	; 0x552 <__bad_interrupt>
       a:	00 00       	nop
       c:	a2 c2       	rjmp	.+1348   	; 0x552 <__bad_interrupt>
       e:	00 00       	nop
      10:	a0 c2       	rjmp	.+1344   	; 0x552 <__bad_interrupt>
      12:	00 00       	nop
      14:	9e c2       	rjmp	.+1340   	; 0x552 <__bad_interrupt>
      16:	00 00       	nop
      18:	9c c2       	rjmp	.+1336   	; 0x552 <__bad_interrupt>
      1a:	00 00       	nop
      1c:	9a c2       	rjmp	.+1332   	; 0x552 <__bad_interrupt>
      1e:	00 00       	nop
      20:	98 c2       	rjmp	.+1328   	; 0x552 <__bad_interrupt>
      22:	00 00       	nop
      24:	96 c2       	rjmp	.+1324   	; 0x552 <__bad_interrupt>
      26:	00 00       	nop
      28:	94 c2       	rjmp	.+1320   	; 0x552 <__bad_interrupt>
      2a:	00 00       	nop
      2c:	92 c2       	rjmp	.+1316   	; 0x552 <__bad_interrupt>
      2e:	00 00       	nop
      30:	90 c2       	rjmp	.+1312   	; 0x552 <__bad_interrupt>
      32:	00 00       	nop
      34:	8e c2       	rjmp	.+1308   	; 0x552 <__bad_interrupt>
      36:	00 00       	nop
      38:	8c c2       	rjmp	.+1304   	; 0x552 <__bad_interrupt>
      3a:	00 00       	nop
      3c:	8a c2       	rjmp	.+1300   	; 0x552 <__bad_interrupt>
      3e:	00 00       	nop
      40:	88 c2       	rjmp	.+1296   	; 0x552 <__bad_interrupt>
      42:	00 00       	nop
      44:	86 c2       	rjmp	.+1292   	; 0x552 <__bad_interrupt>
      46:	00 00       	nop
      48:	84 c2       	rjmp	.+1288   	; 0x552 <__bad_interrupt>
      4a:	00 00       	nop
      4c:	82 c2       	rjmp	.+1284   	; 0x552 <__bad_interrupt>
      4e:	00 00       	nop
      50:	80 c2       	rjmp	.+1280   	; 0x552 <__bad_interrupt>
      52:	00 00       	nop
      54:	7e c2       	rjmp	.+1276   	; 0x552 <__bad_interrupt>
      56:	00 00       	nop
      58:	7c c2       	rjmp	.+1272   	; 0x552 <__bad_interrupt>
      5a:	00 00       	nop
      5c:	7a c2       	rjmp	.+1268   	; 0x552 <__bad_interrupt>
      5e:	00 00       	nop
      60:	78 c2       	rjmp	.+1264   	; 0x552 <__bad_interrupt>
      62:	00 00       	nop
      64:	76 c2       	rjmp	.+1260   	; 0x552 <__bad_interrupt>
      66:	00 00       	nop
      68:	74 c2       	rjmp	.+1256   	; 0x552 <__bad_interrupt>
      6a:	00 00       	nop
      6c:	72 c2       	rjmp	.+1252   	; 0x552 <__bad_interrupt>
      6e:	00 00       	nop
      70:	70 c2       	rjmp	.+1248   	; 0x552 <__bad_interrupt>
      72:	00 00       	nop
      74:	6e c2       	rjmp	.+1244   	; 0x552 <__bad_interrupt>
      76:	00 00       	nop
      78:	6c c2       	rjmp	.+1240   	; 0x552 <__bad_interrupt>
      7a:	00 00       	nop
      7c:	6a c2       	rjmp	.+1236   	; 0x552 <__bad_interrupt>
      7e:	00 00       	nop
      80:	68 c2       	rjmp	.+1232   	; 0x552 <__bad_interrupt>
      82:	00 00       	nop
      84:	66 c2       	rjmp	.+1228   	; 0x552 <__bad_interrupt>
      86:	00 00       	nop
      88:	64 c2       	rjmp	.+1224   	; 0x552 <__bad_interrupt>
      8a:	00 00       	nop
      8c:	62 c2       	rjmp	.+1220   	; 0x552 <__bad_interrupt>
      8e:	00 00       	nop
      90:	60 c2       	rjmp	.+1216   	; 0x552 <__bad_interrupt>
      92:	00 00       	nop
      94:	5e c2       	rjmp	.+1212   	; 0x552 <__bad_interrupt>
      96:	00 00       	nop
      98:	5c c2       	rjmp	.+1208   	; 0x552 <__bad_interrupt>
      9a:	00 00       	nop
      9c:	0c 94 05 0a 	jmp	0x140a	; 0x140a <__vector_39>
      a0:	0c 94 37 0a 	jmp	0x146e	; 0x146e <__vector_40>
      a4:	0c 94 69 0a 	jmp	0x14d2	; 0x14d2 <__vector_41>
      a8:	0c 94 9b 0a 	jmp	0x1536	; 0x1536 <__vector_42>
      ac:	52 c2       	rjmp	.+1188   	; 0x552 <__bad_interrupt>
      ae:	00 00       	nop
      b0:	50 c2       	rjmp	.+1184   	; 0x552 <__bad_interrupt>
      b2:	00 00       	nop
      b4:	4e c2       	rjmp	.+1180   	; 0x552 <__bad_interrupt>
      b6:	00 00       	nop
      b8:	4c c2       	rjmp	.+1176   	; 0x552 <__bad_interrupt>
      ba:	00 00       	nop
      bc:	4a c2       	rjmp	.+1172   	; 0x552 <__bad_interrupt>
      be:	00 00       	nop
      c0:	48 c2       	rjmp	.+1168   	; 0x552 <__bad_interrupt>
      c2:	00 00       	nop
      c4:	46 c2       	rjmp	.+1164   	; 0x552 <__bad_interrupt>
      c6:	00 00       	nop
      c8:	44 c2       	rjmp	.+1160   	; 0x552 <__bad_interrupt>
      ca:	00 00       	nop
      cc:	42 c2       	rjmp	.+1156   	; 0x552 <__bad_interrupt>
      ce:	00 00       	nop
      d0:	40 c2       	rjmp	.+1152   	; 0x552 <__bad_interrupt>
      d2:	00 00       	nop
      d4:	3e c2       	rjmp	.+1148   	; 0x552 <__bad_interrupt>
      d6:	00 00       	nop
      d8:	3c c2       	rjmp	.+1144   	; 0x552 <__bad_interrupt>
      da:	00 00       	nop
      dc:	3a c2       	rjmp	.+1140   	; 0x552 <__bad_interrupt>
      de:	00 00       	nop
      e0:	38 c2       	rjmp	.+1136   	; 0x552 <__bad_interrupt>
      e2:	00 00       	nop
      e4:	36 c2       	rjmp	.+1132   	; 0x552 <__bad_interrupt>
      e6:	00 00       	nop
      e8:	34 c2       	rjmp	.+1128   	; 0x552 <__bad_interrupt>
      ea:	00 00       	nop
      ec:	32 c2       	rjmp	.+1124   	; 0x552 <__bad_interrupt>
      ee:	00 00       	nop
      f0:	30 c2       	rjmp	.+1120   	; 0x552 <__bad_interrupt>
      f2:	00 00       	nop
      f4:	2e c2       	rjmp	.+1116   	; 0x552 <__bad_interrupt>
      f6:	00 00       	nop
      f8:	2c c2       	rjmp	.+1112   	; 0x552 <__bad_interrupt>
      fa:	00 00       	nop
      fc:	2a c2       	rjmp	.+1108   	; 0x552 <__bad_interrupt>
      fe:	00 00       	nop
     100:	28 c2       	rjmp	.+1104   	; 0x552 <__bad_interrupt>
     102:	00 00       	nop
     104:	26 c2       	rjmp	.+1100   	; 0x552 <__bad_interrupt>
     106:	00 00       	nop
     108:	24 c2       	rjmp	.+1096   	; 0x552 <__bad_interrupt>
     10a:	00 00       	nop
     10c:	22 c2       	rjmp	.+1092   	; 0x552 <__bad_interrupt>
     10e:	00 00       	nop
     110:	20 c2       	rjmp	.+1088   	; 0x552 <__bad_interrupt>
     112:	00 00       	nop
     114:	1e c2       	rjmp	.+1084   	; 0x552 <__bad_interrupt>
     116:	00 00       	nop
     118:	1c c2       	rjmp	.+1080   	; 0x552 <__bad_interrupt>
     11a:	00 00       	nop
     11c:	0c 94 3d 09 	jmp	0x127a	; 0x127a <__vector_71>
     120:	0c 94 6f 09 	jmp	0x12de	; 0x12de <__vector_72>
     124:	0c 94 a1 09 	jmp	0x1342	; 0x1342 <__vector_73>
     128:	0c 94 d3 09 	jmp	0x13a6	; 0x13a6 <__vector_74>
     12c:	12 c2       	rjmp	.+1060   	; 0x552 <__bad_interrupt>
     12e:	00 00       	nop
     130:	10 c2       	rjmp	.+1056   	; 0x552 <__bad_interrupt>
     132:	00 00       	nop
     134:	0e c2       	rjmp	.+1052   	; 0x552 <__bad_interrupt>
     136:	00 00       	nop
     138:	0c c2       	rjmp	.+1048   	; 0x552 <__bad_interrupt>
     13a:	00 00       	nop
     13c:	0a c2       	rjmp	.+1044   	; 0x552 <__bad_interrupt>
     13e:	00 00       	nop
     140:	08 c2       	rjmp	.+1040   	; 0x552 <__bad_interrupt>
     142:	00 00       	nop
     144:	06 c2       	rjmp	.+1036   	; 0x552 <__bad_interrupt>
     146:	00 00       	nop
     148:	04 c2       	rjmp	.+1032   	; 0x552 <__bad_interrupt>
     14a:	00 00       	nop
     14c:	02 c2       	rjmp	.+1028   	; 0x552 <__bad_interrupt>
     14e:	00 00       	nop
     150:	00 c2       	rjmp	.+1024   	; 0x552 <__bad_interrupt>
     152:	00 00       	nop
     154:	fe c1       	rjmp	.+1020   	; 0x552 <__bad_interrupt>
     156:	00 00       	nop
     158:	fc c1       	rjmp	.+1016   	; 0x552 <__bad_interrupt>
     15a:	00 00       	nop
     15c:	fa c1       	rjmp	.+1012   	; 0x552 <__bad_interrupt>
     15e:	00 00       	nop
     160:	f8 c1       	rjmp	.+1008   	; 0x552 <__bad_interrupt>
     162:	00 00       	nop
     164:	f6 c1       	rjmp	.+1004   	; 0x552 <__bad_interrupt>
     166:	00 00       	nop
     168:	f4 c1       	rjmp	.+1000   	; 0x552 <__bad_interrupt>
     16a:	00 00       	nop
     16c:	f2 c1       	rjmp	.+996    	; 0x552 <__bad_interrupt>
     16e:	00 00       	nop
     170:	f0 c1       	rjmp	.+992    	; 0x552 <__bad_interrupt>
     172:	00 00       	nop
     174:	ee c1       	rjmp	.+988    	; 0x552 <__bad_interrupt>
     176:	00 00       	nop
     178:	ec c1       	rjmp	.+984    	; 0x552 <__bad_interrupt>
     17a:	00 00       	nop
     17c:	ea c1       	rjmp	.+980    	; 0x552 <__bad_interrupt>
     17e:	00 00       	nop
     180:	e8 c1       	rjmp	.+976    	; 0x552 <__bad_interrupt>
     182:	00 00       	nop
     184:	e6 c1       	rjmp	.+972    	; 0x552 <__bad_interrupt>
     186:	00 00       	nop
     188:	e4 c1       	rjmp	.+968    	; 0x552 <__bad_interrupt>
     18a:	00 00       	nop
     18c:	e2 c1       	rjmp	.+964    	; 0x552 <__bad_interrupt>
     18e:	00 00       	nop
     190:	e0 c1       	rjmp	.+960    	; 0x552 <__bad_interrupt>
     192:	00 00       	nop
     194:	de c1       	rjmp	.+956    	; 0x552 <__bad_interrupt>
     196:	00 00       	nop
     198:	dc c1       	rjmp	.+952    	; 0x552 <__bad_interrupt>
     19a:	00 00       	nop
     19c:	da c1       	rjmp	.+948    	; 0x552 <__bad_interrupt>
     19e:	00 00       	nop
     1a0:	d8 c1       	rjmp	.+944    	; 0x552 <__bad_interrupt>
     1a2:	00 00       	nop
     1a4:	d6 c1       	rjmp	.+940    	; 0x552 <__bad_interrupt>
     1a6:	00 00       	nop
     1a8:	d4 c1       	rjmp	.+936    	; 0x552 <__bad_interrupt>
     1aa:	00 00       	nop
     1ac:	d2 c1       	rjmp	.+932    	; 0x552 <__bad_interrupt>
     1ae:	00 00       	nop
     1b0:	d0 c1       	rjmp	.+928    	; 0x552 <__bad_interrupt>
     1b2:	00 00       	nop
     1b4:	ce c1       	rjmp	.+924    	; 0x552 <__bad_interrupt>
     1b6:	00 00       	nop
     1b8:	cc c1       	rjmp	.+920    	; 0x552 <__bad_interrupt>
     1ba:	00 00       	nop
     1bc:	ca c1       	rjmp	.+916    	; 0x552 <__bad_interrupt>
     1be:	00 00       	nop
     1c0:	c8 c1       	rjmp	.+912    	; 0x552 <__bad_interrupt>
     1c2:	00 00       	nop
     1c4:	c6 c1       	rjmp	.+908    	; 0x552 <__bad_interrupt>
     1c6:	00 00       	nop
     1c8:	c4 c1       	rjmp	.+904    	; 0x552 <__bad_interrupt>
     1ca:	00 00       	nop
     1cc:	c2 c1       	rjmp	.+900    	; 0x552 <__bad_interrupt>
     1ce:	00 00       	nop
     1d0:	c0 c1       	rjmp	.+896    	; 0x552 <__bad_interrupt>
     1d2:	00 00       	nop
     1d4:	be c1       	rjmp	.+892    	; 0x552 <__bad_interrupt>
     1d6:	00 00       	nop
     1d8:	bc c1       	rjmp	.+888    	; 0x552 <__bad_interrupt>
     1da:	00 00       	nop
     1dc:	ba c1       	rjmp	.+884    	; 0x552 <__bad_interrupt>
     1de:	00 00       	nop
     1e0:	b8 c1       	rjmp	.+880    	; 0x552 <__bad_interrupt>
     1e2:	00 00       	nop
     1e4:	b6 c1       	rjmp	.+876    	; 0x552 <__bad_interrupt>
     1e6:	00 00       	nop
     1e8:	b4 c1       	rjmp	.+872    	; 0x552 <__bad_interrupt>
     1ea:	00 00       	nop
     1ec:	b2 c1       	rjmp	.+868    	; 0x552 <__bad_interrupt>
     1ee:	00 00       	nop
     1f0:	b0 c1       	rjmp	.+864    	; 0x552 <__bad_interrupt>
     1f2:	00 00       	nop
     1f4:	ae c1       	rjmp	.+860    	; 0x552 <__bad_interrupt>
     1f6:	00 00       	nop
     1f8:	ac c1       	rjmp	.+856    	; 0x552 <__bad_interrupt>
     1fa:	00 00       	nop
     1fc:	08 00       	.word	0x0008	; ????
     1fe:	00 00       	nop
     200:	be 92       	st	-X, r11
     202:	24 49       	sbci	r18, 0x94	; 148
     204:	12 3e       	cpi	r17, 0xE2	; 226
     206:	ab aa       	std	Y+51, r10	; 0x33
     208:	aa 2a       	or	r10, r26
     20a:	be cd       	rjmp	.-1156   	; 0xfffffd88 <__eeprom_end+0xff7efd88>
     20c:	cc cc       	rjmp	.-1640   	; 0xfffffba6 <__eeprom_end+0xff7efba6>
     20e:	4c 3e       	cpi	r20, 0xEC	; 236
     210:	00 00       	nop
     212:	00 80       	ld	r0, Z
     214:	be ab       	std	Y+54, r27	; 0x36
     216:	aa aa       	std	Y+50, r10	; 0x32
     218:	aa 3e       	cpi	r26, 0xEA	; 234
     21a:	00 00       	nop
     21c:	00 00       	nop
     21e:	bf 00       	.word	0x00bf	; ????
     220:	00 00       	nop
     222:	80 3f       	cpi	r24, 0xF0	; 240
     224:	00 00       	nop
     226:	00 00       	nop
     228:	00 08       	sbc	r0, r0
     22a:	41 78       	andi	r20, 0x81	; 129
     22c:	d3 bb       	out	0x13, r29	; 19
     22e:	43 87       	std	Z+11, r20	; 0x0b
     230:	d1 13       	cpse	r29, r17
     232:	3d 19       	sub	r19, r13
     234:	0e 3c       	cpi	r16, 0xCE	; 206
     236:	c3 bd       	out	0x23, r28	; 35
     238:	42 82       	std	Z+2, r4	; 0x02
     23a:	ad 2b       	or	r26, r29
     23c:	3e 68       	ori	r19, 0x8E	; 142
     23e:	ec 82       	std	Y+4, r14	; 0x04
     240:	76 be       	out	0x36, r7	; 54
     242:	d9 8f       	std	Y+25, r29	; 0x19
     244:	e1 a9       	ldd	r30, Z+49	; 0x31
     246:	3e 4c       	sbci	r19, 0xCE	; 206
     248:	80 ef       	ldi	r24, 0xF0	; 240
     24a:	ff be       	out	0x3f, r15	; 63
     24c:	01 c4       	rjmp	.+2050   	; 0xa50 <st7565r_init+0x2ec>
     24e:	ff 7f       	andi	r31, 0xFF	; 255
     250:	3f 00       	.word	0x003f	; ????
     252:	00 00       	nop
     254:	00 00       	nop
     256:	07 63       	ori	r16, 0x37	; 55
     258:	42 36       	cpi	r20, 0x62	; 98
     25a:	b7 9b       	sbis	0x16, 7	; 22
     25c:	d8 a7       	std	Y+40, r29	; 0x28
     25e:	1a 39       	cpi	r17, 0x9A	; 154
     260:	68 56       	subi	r22, 0x68	; 104
     262:	18 ae       	std	Y+56, r1	; 0x38
     264:	ba ab       	std	Y+50, r27	; 0x32
     266:	55 8c       	ldd	r5, Z+29	; 0x1d
     268:	1d 3c       	cpi	r17, 0xCD	; 205
     26a:	b7 cc       	rjmp	.-1682   	; 0xfffffbda <__eeprom_end+0xff7efbda>
     26c:	57 63       	ori	r21, 0x37	; 55
     26e:	bd 6d       	ori	r27, 0xDD	; 221
     270:	ed fd       	.word	0xfded	; ????
     272:	75 3e       	cpi	r23, 0xE5	; 229
     274:	f6 17       	cp	r31, r22
     276:	72 31       	cpi	r23, 0x12	; 18
     278:	bf 00       	.word	0x00bf	; ????
     27a:	00 00       	nop
     27c:	80 3f       	cpi	r24, 0xF0	; 240

0000027e <__trampolines_end>:
     27e:	00 00       	nop
     280:	00 00       	nop
     282:	00 00       	nop
     284:	00 20       	and	r0, r0
     286:	20 20       	and	r2, r0
     288:	20 20       	and	r2, r0
     28a:	00 20       	and	r0, r0
     28c:	50 50       	subi	r21, 0x00	; 0
     28e:	50 00       	.word	0x0050	; ????
     290:	00 00       	nop
     292:	00 50       	subi	r16, 0x00	; 0
     294:	50 f8       	bld	r5, 0
     296:	50 f8       	bld	r5, 0
     298:	50 50       	subi	r21, 0x00	; 0
     29a:	20 78       	andi	r18, 0x80	; 128
     29c:	a0 70       	andi	r26, 0x00	; 0
     29e:	28 f0       	brcs	.+10     	; 0x2aa <__trampolines_end+0x2c>
     2a0:	20 c0       	rjmp	.+64     	; 0x2e2 <__trampolines_end+0x64>
     2a2:	c8 10       	cpse	r12, r8
     2a4:	20 40       	sbci	r18, 0x00	; 0
     2a6:	98 18       	sub	r9, r8
     2a8:	60 90 a0 40 	lds	r6, 0x40A0	; 0x8040a0 <__bss_end+0x1da4>
     2ac:	a8 90       	.word	0x90a8	; ????
     2ae:	68 60       	ori	r22, 0x08	; 8
     2b0:	20 40       	sbci	r18, 0x00	; 0
     2b2:	00 00       	nop
     2b4:	00 00       	nop
     2b6:	10 20       	and	r1, r0
     2b8:	40 40       	sbci	r20, 0x00	; 0
     2ba:	40 20       	and	r4, r0
     2bc:	10 40       	sbci	r17, 0x00	; 0
     2be:	20 10       	cpse	r2, r0
     2c0:	10 10       	cpse	r1, r0
     2c2:	20 40       	sbci	r18, 0x00	; 0
     2c4:	00 50       	subi	r16, 0x00	; 0
     2c6:	20 f8       	bld	r2, 0
     2c8:	20 50       	subi	r18, 0x00	; 0
     2ca:	00 00       	nop
     2cc:	20 20       	and	r2, r0
     2ce:	f8 20       	and	r15, r8
     2d0:	20 00       	.word	0x0020	; ????
     2d2:	00 00       	nop
     2d4:	00 00       	nop
     2d6:	60 20       	and	r6, r0
     2d8:	40 00       	.word	0x0040	; ????
     2da:	00 00       	nop
     2dc:	f8 00       	.word	0x00f8	; ????
     2de:	00 00       	nop
     2e0:	00 00       	nop
     2e2:	00 00       	nop
     2e4:	00 60       	ori	r16, 0x00	; 0
     2e6:	60 00       	.word	0x0060	; ????
     2e8:	08 10       	cpse	r0, r8
     2ea:	20 40       	sbci	r18, 0x00	; 0
     2ec:	80 00       	.word	0x0080	; ????
     2ee:	70 88       	ldd	r7, Z+16	; 0x10
     2f0:	98 a8       	ldd	r9, Y+48	; 0x30
     2f2:	c8 88       	ldd	r12, Y+16	; 0x10
     2f4:	70 20       	and	r7, r0
     2f6:	60 20       	and	r6, r0
     2f8:	20 20       	and	r2, r0
     2fa:	20 70       	andi	r18, 0x00	; 0
     2fc:	70 88       	ldd	r7, Z+16	; 0x10
     2fe:	08 10       	cpse	r0, r8
     300:	20 40       	sbci	r18, 0x00	; 0
     302:	f8 f8       	.word	0xf8f8	; ????
     304:	10 20       	and	r1, r0
     306:	10 08       	sbc	r1, r0
     308:	88 70       	andi	r24, 0x08	; 8
     30a:	10 30       	cpi	r17, 0x00	; 0
     30c:	50 90 f8 10 	lds	r5, 0x10F8	; 0x8010f8 <__TEXT_REGION_LENGTH__+0x7bf0f8>
     310:	10 f8       	bld	r1, 0
     312:	80 f0       	brcs	.+32     	; 0x334 <__trampolines_end+0xb6>
     314:	08 08       	sbc	r0, r8
     316:	88 70       	andi	r24, 0x08	; 8
     318:	30 40       	sbci	r19, 0x00	; 0
     31a:	80 f0       	brcs	.+32     	; 0x33c <__trampolines_end+0xbe>
     31c:	88 88       	ldd	r8, Y+16	; 0x10
     31e:	70 f8       	bld	r7, 0
     320:	08 10       	cpse	r0, r8
     322:	20 40       	sbci	r18, 0x00	; 0
     324:	40 40       	sbci	r20, 0x00	; 0
     326:	70 88       	ldd	r7, Z+16	; 0x10
     328:	88 70       	andi	r24, 0x08	; 8
     32a:	88 88       	ldd	r8, Y+16	; 0x10
     32c:	70 70       	andi	r23, 0x00	; 0
     32e:	88 88       	ldd	r8, Y+16	; 0x10
     330:	78 08       	sbc	r7, r8
     332:	10 60       	ori	r17, 0x00	; 0
     334:	00 60       	ori	r16, 0x00	; 0
     336:	60 00       	.word	0x0060	; ????
     338:	60 60       	ori	r22, 0x00	; 0
     33a:	00 00       	nop
     33c:	60 60       	ori	r22, 0x00	; 0
     33e:	00 60       	ori	r16, 0x00	; 0
     340:	20 40       	sbci	r18, 0x00	; 0
     342:	08 10       	cpse	r0, r8
     344:	20 40       	sbci	r18, 0x00	; 0
     346:	20 10       	cpse	r2, r0
     348:	08 00       	.word	0x0008	; ????
     34a:	00 f8       	bld	r0, 0
     34c:	00 f8       	bld	r0, 0
     34e:	00 00       	nop
     350:	80 40       	sbci	r24, 0x00	; 0
     352:	20 10       	cpse	r2, r0
     354:	20 40       	sbci	r18, 0x00	; 0
     356:	80 70       	andi	r24, 0x00	; 0
     358:	88 08       	sbc	r8, r8
     35a:	10 20       	and	r1, r0
     35c:	00 20       	and	r0, r0
     35e:	70 88       	ldd	r7, Z+16	; 0x10
     360:	08 68       	ori	r16, 0x88	; 136
     362:	a8 a8       	ldd	r10, Y+48	; 0x30
     364:	70 70       	andi	r23, 0x00	; 0
     366:	88 88       	ldd	r8, Y+16	; 0x10
     368:	88 f8       	.word	0xf888	; ????
     36a:	88 88       	ldd	r8, Y+16	; 0x10
     36c:	f0 88       	ldd	r15, Z+16	; 0x10
     36e:	88 f0       	brcs	.+34     	; 0x392 <__trampolines_end+0x114>
     370:	88 88       	ldd	r8, Y+16	; 0x10
     372:	f0 70       	andi	r31, 0x00	; 0
     374:	88 80       	ld	r8, Y
     376:	80 80       	ld	r8, Z
     378:	88 70       	andi	r24, 0x08	; 8
     37a:	e0 90 88 88 	lds	r14, 0x8888	; 0x808888 <__bss_end+0x658c>
     37e:	88 90       	.word	0x9088	; ????
     380:	e0 f8       	bld	r14, 0
     382:	80 80       	ld	r8, Z
     384:	f0 80       	ld	r15, Z
     386:	80 f8       	bld	r8, 0
     388:	f8 80       	ld	r15, Y
     38a:	80 e0       	ldi	r24, 0x00	; 0
     38c:	80 80       	ld	r8, Z
     38e:	80 70       	andi	r24, 0x00	; 0
     390:	88 80       	ld	r8, Y
     392:	80 98       	cbi	0x10, 0	; 16
     394:	88 70       	andi	r24, 0x08	; 8
     396:	88 88       	ldd	r8, Y+16	; 0x10
     398:	88 f8       	.word	0xf888	; ????
     39a:	88 88       	ldd	r8, Y+16	; 0x10
     39c:	88 70       	andi	r24, 0x08	; 8
     39e:	20 20       	and	r2, r0
     3a0:	20 20       	and	r2, r0
     3a2:	20 70       	andi	r18, 0x00	; 0
     3a4:	38 10       	cpse	r3, r8
     3a6:	10 10       	cpse	r1, r0
     3a8:	10 90 60 88 	lds	r1, 0x8860	; 0x808860 <__bss_end+0x6564>
     3ac:	90 a0       	ldd	r9, Z+32	; 0x20
     3ae:	c0 a0       	ldd	r12, Z+32	; 0x20
     3b0:	90 88       	ldd	r9, Z+16	; 0x10
     3b2:	80 80       	ld	r8, Z
     3b4:	80 80       	ld	r8, Z
     3b6:	80 80       	ld	r8, Z
     3b8:	f8 88       	ldd	r15, Y+16	; 0x10
     3ba:	d8 a8       	ldd	r13, Y+48	; 0x30
     3bc:	88 88       	ldd	r8, Y+16	; 0x10
     3be:	88 88       	ldd	r8, Y+16	; 0x10
     3c0:	88 88       	ldd	r8, Y+16	; 0x10
     3c2:	c8 a8       	ldd	r12, Y+48	; 0x30
     3c4:	98 88       	ldd	r9, Y+16	; 0x10
     3c6:	88 70       	andi	r24, 0x08	; 8
     3c8:	88 88       	ldd	r8, Y+16	; 0x10
     3ca:	88 88       	ldd	r8, Y+16	; 0x10
     3cc:	88 70       	andi	r24, 0x08	; 8
     3ce:	f0 88       	ldd	r15, Z+16	; 0x10
     3d0:	88 f0       	brcs	.+34     	; 0x3f4 <__trampolines_end+0x176>
     3d2:	80 80       	ld	r8, Z
     3d4:	80 70       	andi	r24, 0x00	; 0
     3d6:	88 88       	ldd	r8, Y+16	; 0x10
     3d8:	88 a8       	ldd	r8, Y+48	; 0x30
     3da:	90 68       	ori	r25, 0x80	; 128
     3dc:	f0 88       	ldd	r15, Z+16	; 0x10
     3de:	88 f0       	brcs	.+34     	; 0x402 <__LOCK_REGION_LENGTH__+0x2>
     3e0:	a0 90 88 78 	lds	r10, 0x7888	; 0x807888 <__bss_end+0x558c>
     3e4:	80 80       	ld	r8, Z
     3e6:	70 08       	sbc	r7, r0
     3e8:	08 f0       	brcs	.+2      	; 0x3ec <__trampolines_end+0x16e>
     3ea:	f8 20       	and	r15, r8
     3ec:	20 20       	and	r2, r0
     3ee:	20 20       	and	r2, r0
     3f0:	20 88       	ldd	r2, Z+16	; 0x10
     3f2:	88 88       	ldd	r8, Y+16	; 0x10
     3f4:	88 88       	ldd	r8, Y+16	; 0x10
     3f6:	88 70       	andi	r24, 0x08	; 8
     3f8:	88 88       	ldd	r8, Y+16	; 0x10
     3fa:	88 88       	ldd	r8, Y+16	; 0x10
     3fc:	88 50       	subi	r24, 0x08	; 8
     3fe:	20 88       	ldd	r2, Z+16	; 0x10
     400:	88 88       	ldd	r8, Y+16	; 0x10
     402:	a8 a8       	ldd	r10, Y+48	; 0x30
     404:	d8 88       	ldd	r13, Y+16	; 0x10
     406:	88 88       	ldd	r8, Y+16	; 0x10
     408:	50 20       	and	r5, r0
     40a:	50 88       	ldd	r5, Z+16	; 0x10
     40c:	88 88       	ldd	r8, Y+16	; 0x10
     40e:	88 50       	subi	r24, 0x08	; 8
     410:	20 20       	and	r2, r0
     412:	20 20       	and	r2, r0
     414:	f8 08       	sbc	r15, r8
     416:	10 20       	and	r1, r0
     418:	40 80       	ld	r4, Z
     41a:	f8 38       	cpi	r31, 0x88	; 136
     41c:	20 20       	and	r2, r0
     41e:	20 20       	and	r2, r0
     420:	20 38       	cpi	r18, 0x80	; 128
     422:	00 80       	ld	r0, Z
     424:	40 20       	and	r4, r0
     426:	10 08       	sbc	r1, r0
     428:	00 e0       	ldi	r16, 0x00	; 0
     42a:	20 20       	and	r2, r0
     42c:	20 20       	and	r2, r0
     42e:	20 e0       	ldi	r18, 0x00	; 0
     430:	20 50       	subi	r18, 0x00	; 0
     432:	88 00       	.word	0x0088	; ????
	...
     43c:	00 f8       	bld	r0, 0
     43e:	40 20       	and	r4, r0
     440:	10 00       	.word	0x0010	; ????
     442:	00 00       	nop
     444:	00 00       	nop
     446:	00 70       	andi	r16, 0x00	; 0
     448:	08 78       	andi	r16, 0x88	; 136
     44a:	88 78       	andi	r24, 0x88	; 136
     44c:	80 80       	ld	r8, Z
     44e:	b0 c8       	rjmp	.-3744   	; 0xfffff5b0 <__eeprom_end+0xff7ef5b0>
     450:	88 88       	ldd	r8, Y+16	; 0x10
     452:	f0 00       	.word	0x00f0	; ????
     454:	00 70       	andi	r16, 0x00	; 0
     456:	80 80       	ld	r8, Z
     458:	88 70       	andi	r24, 0x08	; 8
     45a:	08 08       	sbc	r0, r8
     45c:	68 98       	cbi	0x0d, 0	; 13
     45e:	88 88       	ldd	r8, Y+16	; 0x10
     460:	78 00       	.word	0x0078	; ????
     462:	00 70       	andi	r16, 0x00	; 0
     464:	88 f8       	.word	0xf888	; ????
     466:	80 70       	andi	r24, 0x00	; 0
     468:	30 48       	sbci	r19, 0x80	; 128
     46a:	40 e0       	ldi	r20, 0x00	; 0
     46c:	40 40       	sbci	r20, 0x00	; 0
     46e:	40 00       	.word	0x0040	; ????
     470:	00 78       	andi	r16, 0x80	; 128
     472:	88 78       	andi	r24, 0x88	; 136
     474:	08 30       	cpi	r16, 0x08	; 8
     476:	80 80       	ld	r8, Z
     478:	b0 c8       	rjmp	.-3744   	; 0xfffff5da <__eeprom_end+0xff7ef5da>
     47a:	88 88       	ldd	r8, Y+16	; 0x10
     47c:	88 20       	and	r8, r8
     47e:	00 60       	ori	r16, 0x00	; 0
     480:	20 20       	and	r2, r0
     482:	20 70       	andi	r18, 0x00	; 0
     484:	10 00       	.word	0x0010	; ????
     486:	30 10       	cpse	r3, r0
     488:	10 90 60 40 	lds	r1, 0x4060	; 0x804060 <__bss_end+0x1d64>
     48c:	40 48       	sbci	r20, 0x80	; 128
     48e:	50 60       	ori	r21, 0x00	; 0
     490:	50 48       	sbci	r21, 0x80	; 128
     492:	60 20       	and	r6, r0
     494:	20 20       	and	r2, r0
     496:	20 20       	and	r2, r0
     498:	70 00       	.word	0x0070	; ????
     49a:	00 d0       	rcall	.+0      	; 0x49c <__LOCK_REGION_LENGTH__+0x9c>
     49c:	a8 a8       	ldd	r10, Y+48	; 0x30
     49e:	88 88       	ldd	r8, Y+16	; 0x10
     4a0:	00 00       	nop
     4a2:	b0 c8       	rjmp	.-3744   	; 0xfffff604 <__eeprom_end+0xff7ef604>
     4a4:	88 88       	ldd	r8, Y+16	; 0x10
     4a6:	88 00       	.word	0x0088	; ????
     4a8:	00 70       	andi	r16, 0x00	; 0
     4aa:	88 88       	ldd	r8, Y+16	; 0x10
     4ac:	88 70       	andi	r24, 0x08	; 8
     4ae:	00 00       	nop
     4b0:	f0 88       	ldd	r15, Z+16	; 0x10
     4b2:	f0 80       	ld	r15, Z
     4b4:	80 00       	.word	0x0080	; ????
     4b6:	00 68       	ori	r16, 0x80	; 128
     4b8:	98 78       	andi	r25, 0x88	; 136
     4ba:	08 08       	sbc	r0, r8
     4bc:	00 00       	nop
     4be:	b0 c8       	rjmp	.-3744   	; 0xfffff620 <__eeprom_end+0xff7ef620>
     4c0:	80 80       	ld	r8, Z
     4c2:	80 00       	.word	0x0080	; ????
     4c4:	00 70       	andi	r16, 0x00	; 0
     4c6:	80 70       	andi	r24, 0x00	; 0
     4c8:	08 f0       	brcs	.+2      	; 0x4cc <__LOCK_REGION_LENGTH__+0xcc>
     4ca:	40 40       	sbci	r20, 0x00	; 0
     4cc:	e0 40       	sbci	r30, 0x00	; 0
     4ce:	40 48       	sbci	r20, 0x80	; 128
     4d0:	30 00       	.word	0x0030	; ????
     4d2:	00 88       	ldd	r0, Z+16	; 0x10
     4d4:	88 88       	ldd	r8, Y+16	; 0x10
     4d6:	98 68       	ori	r25, 0x88	; 136
     4d8:	00 00       	nop
     4da:	88 88       	ldd	r8, Y+16	; 0x10
     4dc:	88 50       	subi	r24, 0x08	; 8
     4de:	20 00       	.word	0x0020	; ????
     4e0:	00 88       	ldd	r0, Z+16	; 0x10
     4e2:	88 a8       	ldd	r8, Y+48	; 0x30
     4e4:	a8 50       	subi	r26, 0x08	; 8
     4e6:	00 00       	nop
     4e8:	88 50       	subi	r24, 0x08	; 8
     4ea:	20 50       	subi	r18, 0x00	; 0
     4ec:	88 00       	.word	0x0088	; ????
     4ee:	00 88       	ldd	r0, Z+16	; 0x10
     4f0:	88 78       	andi	r24, 0x88	; 136
     4f2:	08 70       	andi	r16, 0x08	; 8
     4f4:	00 00       	nop
     4f6:	f8 10       	cpse	r15, r8
     4f8:	20 40       	sbci	r18, 0x00	; 0
     4fa:	f8 10       	cpse	r15, r8
     4fc:	20 20       	and	r2, r0
     4fe:	40 20       	and	r4, r0
     500:	20 10       	cpse	r2, r0
     502:	20 20       	and	r2, r0
     504:	20 20       	and	r2, r0
     506:	20 20       	and	r2, r0
     508:	20 40       	sbci	r18, 0x00	; 0
     50a:	20 20       	and	r2, r0
     50c:	10 20       	and	r1, r0
     50e:	20 40       	sbci	r18, 0x00	; 0

00000510 <__ctors_end>:
     510:	11 24       	eor	r1, r1
     512:	1f be       	out	0x3f, r1	; 63
     514:	cf ef       	ldi	r28, 0xFF	; 255
     516:	cd bf       	out	0x3d, r28	; 61
     518:	df e5       	ldi	r29, 0x5F	; 95
     51a:	de bf       	out	0x3e, r29	; 62
     51c:	00 e0       	ldi	r16, 0x00	; 0
     51e:	0c bf       	out	0x3c, r16	; 60

00000520 <__do_copy_data>:
     520:	10 e2       	ldi	r17, 0x20	; 32
     522:	a0 e0       	ldi	r26, 0x00	; 0
     524:	b0 e2       	ldi	r27, 0x20	; 32
     526:	e4 ee       	ldi	r30, 0xE4	; 228
     528:	fd e2       	ldi	r31, 0x2D	; 45
     52a:	00 e0       	ldi	r16, 0x00	; 0
     52c:	0b bf       	out	0x3b, r16	; 59
     52e:	02 c0       	rjmp	.+4      	; 0x534 <__do_copy_data+0x14>
     530:	07 90       	elpm	r0, Z+
     532:	0d 92       	st	X+, r0
     534:	a6 36       	cpi	r26, 0x66	; 102
     536:	b1 07       	cpc	r27, r17
     538:	d9 f7       	brne	.-10     	; 0x530 <__do_copy_data+0x10>

0000053a <__do_clear_bss>:
     53a:	22 e2       	ldi	r18, 0x22	; 34
     53c:	a6 e6       	ldi	r26, 0x66	; 102
     53e:	b0 e2       	ldi	r27, 0x20	; 32
     540:	01 c0       	rjmp	.+2      	; 0x544 <.do_clear_bss_start>

00000542 <.do_clear_bss_loop>:
     542:	1d 92       	st	X+, r1

00000544 <.do_clear_bss_start>:
     544:	ac 3f       	cpi	r26, 0xFC	; 252
     546:	b2 07       	cpc	r27, r18
     548:	e1 f7       	brne	.-8      	; 0x542 <.do_clear_bss_loop>
     54a:	0e 94 af 0f 	call	0x1f5e	; 0x1f5e <main>
     54e:	0c 94 f0 16 	jmp	0x2de0	; 0x2de0 <_exit>

00000552 <__bad_interrupt>:
     552:	56 cd       	rjmp	.-1364   	; 0x0 <__vectors>

00000554 <adc_handler>:
 * \retval the raw ADC value from the current ntc_sensor_sample
 */
int16_t ntc_get_raw_value(void)
{
	return ntc_sensor_sample;
}
     554:	cf 93       	push	r28
     556:	df 93       	push	r29
     558:	1f 92       	push	r1
     55a:	1f 92       	push	r1
     55c:	cd b7       	in	r28, 0x3d	; 61
     55e:	de b7       	in	r29, 0x3e	; 62
     560:	61 30       	cpi	r22, 0x01	; 1
     562:	69 f5       	brne	.+90     	; 0x5be <adc_handler+0x6a>
     564:	80 91 67 20 	lds	r24, 0x2067	; 0x802067 <light_sensor_samples.4860>
     568:	8f 5f       	subi	r24, 0xFF	; 255
     56a:	80 93 67 20 	sts	0x2067, r24	; 0x802067 <light_sensor_samples.4860>
     56e:	81 30       	cpi	r24, 0x01	; 1
     570:	39 f4       	brne	.+14     	; 0x580 <adc_handler+0x2c>
     572:	40 93 68 20 	sts	0x2068, r20	; 0x802068 <light_sensor_sample>
     576:	50 93 69 20 	sts	0x2069, r21	; 0x802069 <light_sensor_sample+0x1>
     57a:	10 92 6c 20 	sts	0x206C, r1	; 0x80206c <light_sensor_data_ready>
     57e:	14 c0       	rjmp	.+40     	; 0x5a8 <adc_handler+0x54>
     580:	20 91 68 20 	lds	r18, 0x2068	; 0x802068 <light_sensor_sample>
     584:	30 91 69 20 	lds	r19, 0x2069	; 0x802069 <light_sensor_sample+0x1>
     588:	42 0f       	add	r20, r18
     58a:	53 1f       	adc	r21, r19
     58c:	56 95       	lsr	r21
     58e:	47 95       	ror	r20
     590:	40 93 68 20 	sts	0x2068, r20	; 0x802068 <light_sensor_sample>
     594:	50 93 69 20 	sts	0x2069, r21	; 0x802069 <light_sensor_sample+0x1>
     598:	84 30       	cpi	r24, 0x04	; 4
     59a:	31 f4       	brne	.+12     	; 0x5a8 <adc_handler+0x54>
     59c:	10 92 67 20 	sts	0x2067, r1	; 0x802067 <light_sensor_samples.4860>
     5a0:	81 e0       	ldi	r24, 0x01	; 1
     5a2:	80 93 6c 20 	sts	0x206C, r24	; 0x80206c <light_sensor_data_ready>
     5a6:	39 c0       	rjmp	.+114    	; 0x61a <adc_handler+0xc6>
     5a8:	8f b7       	in	r24, 0x3f	; 63
     5aa:	8a 83       	std	Y+2, r24	; 0x02
     5ac:	f8 94       	cli
     5ae:	9a 81       	ldd	r25, Y+2	; 0x02
     5b0:	e0 e0       	ldi	r30, 0x00	; 0
     5b2:	f2 e0       	ldi	r31, 0x02	; 2
     5b4:	80 81       	ld	r24, Z
     5b6:	84 60       	ori	r24, 0x04	; 4
     5b8:	80 83       	st	Z, r24
     5ba:	9f bf       	out	0x3f, r25	; 63
     5bc:	2e c0       	rjmp	.+92     	; 0x61a <adc_handler+0xc6>
     5be:	62 30       	cpi	r22, 0x02	; 2
     5c0:	61 f5       	brne	.+88     	; 0x61a <adc_handler+0xc6>
     5c2:	80 91 66 20 	lds	r24, 0x2066	; 0x802066 <__data_end>
     5c6:	8f 5f       	subi	r24, 0xFF	; 255
     5c8:	80 93 66 20 	sts	0x2066, r24	; 0x802066 <__data_end>
     5cc:	81 30       	cpi	r24, 0x01	; 1
     5ce:	39 f4       	brne	.+14     	; 0x5de <adc_handler+0x8a>
     5d0:	40 93 6a 20 	sts	0x206A, r20	; 0x80206a <ntc_sensor_sample>
     5d4:	50 93 6b 20 	sts	0x206B, r21	; 0x80206b <ntc_sensor_sample+0x1>
     5d8:	10 92 6d 20 	sts	0x206D, r1	; 0x80206d <ntc_sensor_data_ready>
     5dc:	14 c0       	rjmp	.+40     	; 0x606 <adc_handler+0xb2>
     5de:	20 91 6a 20 	lds	r18, 0x206A	; 0x80206a <ntc_sensor_sample>
     5e2:	30 91 6b 20 	lds	r19, 0x206B	; 0x80206b <ntc_sensor_sample+0x1>
     5e6:	42 0f       	add	r20, r18
     5e8:	53 1f       	adc	r21, r19
     5ea:	56 95       	lsr	r21
     5ec:	47 95       	ror	r20
     5ee:	40 93 6a 20 	sts	0x206A, r20	; 0x80206a <ntc_sensor_sample>
     5f2:	50 93 6b 20 	sts	0x206B, r21	; 0x80206b <ntc_sensor_sample+0x1>
     5f6:	84 30       	cpi	r24, 0x04	; 4
     5f8:	31 f4       	brne	.+12     	; 0x606 <adc_handler+0xb2>
     5fa:	10 92 66 20 	sts	0x2066, r1	; 0x802066 <__data_end>
     5fe:	81 e0       	ldi	r24, 0x01	; 1
     600:	80 93 6d 20 	sts	0x206D, r24	; 0x80206d <ntc_sensor_data_ready>
     604:	0a c0       	rjmp	.+20     	; 0x61a <adc_handler+0xc6>
     606:	8f b7       	in	r24, 0x3f	; 63
     608:	89 83       	std	Y+1, r24	; 0x01
     60a:	f8 94       	cli
     60c:	99 81       	ldd	r25, Y+1	; 0x01
     60e:	e0 e0       	ldi	r30, 0x00	; 0
     610:	f2 e0       	ldi	r31, 0x02	; 2
     612:	80 81       	ld	r24, Z
     614:	88 60       	ori	r24, 0x08	; 8
     616:	80 83       	st	Z, r24
     618:	9f bf       	out	0x3f, r25	; 63
     61a:	0f 90       	pop	r0
     61c:	0f 90       	pop	r0
     61e:	df 91       	pop	r29
     620:	cf 91       	pop	r28
     622:	08 95       	ret

00000624 <ntc_data_is_ready>:
     624:	cf 93       	push	r28
     626:	df 93       	push	r29
     628:	1f 92       	push	r1
     62a:	cd b7       	in	r28, 0x3d	; 61
     62c:	de b7       	in	r29, 0x3e	; 62
     62e:	8f b7       	in	r24, 0x3f	; 63
     630:	89 83       	std	Y+1, r24	; 0x01
     632:	f8 94       	cli
     634:	99 81       	ldd	r25, Y+1	; 0x01
     636:	80 91 6d 20 	lds	r24, 0x206D	; 0x80206d <ntc_sensor_data_ready>
     63a:	88 23       	and	r24, r24
     63c:	21 f0       	breq	.+8      	; 0x646 <ntc_data_is_ready+0x22>
     63e:	10 92 6d 20 	sts	0x206D, r1	; 0x80206d <ntc_sensor_data_ready>
     642:	9f bf       	out	0x3f, r25	; 63
     644:	01 c0       	rjmp	.+2      	; 0x648 <ntc_data_is_ready+0x24>
     646:	9f bf       	out	0x3f, r25	; 63
     648:	0f 90       	pop	r0
     64a:	df 91       	pop	r29
     64c:	cf 91       	pop	r28
     64e:	08 95       	ret

00000650 <adc_sensors_init>:
     650:	1f 93       	push	r17
     652:	cf 93       	push	r28
     654:	df 93       	push	r29
     656:	cd b7       	in	r28, 0x3d	; 61
     658:	de b7       	in	r29, 0x3e	; 62
     65a:	2b 97       	sbiw	r28, 0x0b	; 11
     65c:	cd bf       	out	0x3d, r28	; 61
     65e:	de bf       	out	0x3e, r29	; 62
     660:	be 01       	movw	r22, r28
     662:	6f 5f       	subi	r22, 0xFF	; 255
     664:	7f 4f       	sbci	r23, 0xFF	; 255
     666:	80 e0       	ldi	r24, 0x00	; 0
     668:	92 e0       	ldi	r25, 0x02	; 2
     66a:	fd d7       	rcall	.+4090   	; 0x1666 <adc_read_configuration>
     66c:	ae 01       	movw	r20, r28
     66e:	48 5f       	subi	r20, 0xF8	; 248
     670:	5f 4f       	sbci	r21, 0xFF	; 255
     672:	61 e0       	ldi	r22, 0x01	; 1
     674:	80 e0       	ldi	r24, 0x00	; 0
     676:	92 e0       	ldi	r25, 0x02	; 2
     678:	0e 94 b7 0b 	call	0x176e	; 0x176e <adcch_read_configuration>
     67c:	8a 81       	ldd	r24, Y+2	; 0x02
     67e:	9b 81       	ldd	r25, Y+3	; 0x03
     680:	9f 78       	andi	r25, 0x8F	; 143
     682:	90 61       	ori	r25, 0x10	; 16
     684:	9b 83       	std	Y+3, r25	; 0x03
     686:	92 e0       	ldi	r25, 0x02	; 2
     688:	9d 83       	std	Y+5, r25	; 0x05
     68a:	81 7e       	andi	r24, 0xE1	; 225
     68c:	80 61       	ori	r24, 0x10	; 16
     68e:	8a 83       	std	Y+2, r24	; 0x02
     690:	1c 82       	std	Y+4, r1	; 0x04
     692:	be 01       	movw	r22, r28
     694:	6f 5f       	subi	r22, 0xFF	; 255
     696:	7f 4f       	sbci	r23, 0xFF	; 255
     698:	80 e0       	ldi	r24, 0x00	; 0
     69a:	92 e0       	ldi	r25, 0x02	; 2
     69c:	7e d7       	rcall	.+3836   	; 0x159a <adc_write_configuration>
     69e:	6a ea       	ldi	r22, 0xAA	; 170
     6a0:	72 e0       	ldi	r23, 0x02	; 2
     6a2:	80 e0       	ldi	r24, 0x00	; 0
     6a4:	92 e0       	ldi	r25, 0x02	; 2
     6a6:	4b d3       	rcall	.+1686   	; 0xd3e <adc_set_callback>
     6a8:	11 e0       	ldi	r17, 0x01	; 1
     6aa:	18 87       	std	Y+8, r17	; 0x08
     6ac:	19 86       	std	Y+9, r1	; 0x09
     6ae:	8a 85       	ldd	r24, Y+10	; 0x0a
     6b0:	80 7f       	andi	r24, 0xF0	; 240
     6b2:	81 60       	ori	r24, 0x01	; 1
     6b4:	8a 87       	std	Y+10, r24	; 0x0a
     6b6:	ae 01       	movw	r20, r28
     6b8:	48 5f       	subi	r20, 0xF8	; 248
     6ba:	5f 4f       	sbci	r21, 0xFF	; 255
     6bc:	61 e0       	ldi	r22, 0x01	; 1
     6be:	80 e0       	ldi	r24, 0x00	; 0
     6c0:	92 e0       	ldi	r25, 0x02	; 2
     6c2:	0e 94 6c 0b 	call	0x16d8	; 0x16d8 <adcch_write_configuration>
     6c6:	18 87       	std	Y+8, r17	; 0x08
     6c8:	88 e0       	ldi	r24, 0x08	; 8
     6ca:	89 87       	std	Y+9, r24	; 0x09
     6cc:	ae 01       	movw	r20, r28
     6ce:	48 5f       	subi	r20, 0xF8	; 248
     6d0:	5f 4f       	sbci	r21, 0xFF	; 255
     6d2:	62 e0       	ldi	r22, 0x02	; 2
     6d4:	80 e0       	ldi	r24, 0x00	; 0
     6d6:	92 e0       	ldi	r25, 0x02	; 2
     6d8:	ff d7       	rcall	.+4094   	; 0x16d8 <adcch_write_configuration>
     6da:	80 e0       	ldi	r24, 0x00	; 0
     6dc:	92 e0       	ldi	r25, 0x02	; 2
     6de:	8b d3       	rcall	.+1814   	; 0xdf6 <adc_enable>
     6e0:	2b 96       	adiw	r28, 0x0b	; 11
     6e2:	cd bf       	out	0x3d, r28	; 61
     6e4:	de bf       	out	0x3e, r29	; 62
     6e6:	df 91       	pop	r29
     6e8:	cf 91       	pop	r28
     6ea:	1f 91       	pop	r17
     6ec:	08 95       	ret

000006ee <ntc_get_temperature>:
 * \note The result is inaccurate for temperatures outside 5-45 degrees.
 *
 * \retval the temperature in Celsius
 */
int8_t ntc_get_temperature(void)
{
     6ee:	cf 93       	push	r28
     6f0:	df 93       	push	r29
	int8_t retval = 0;
	float ntc_sample = ntc_sensor_sample;
     6f2:	c0 91 6a 20 	lds	r28, 0x206A	; 0x80206a <ntc_sensor_sample>
     6f6:	d0 91 6b 20 	lds	r29, 0x206B	; 0x80206b <ntc_sensor_sample+0x1>
     6fa:	be 01       	movw	r22, r28
     6fc:	80 e0       	ldi	r24, 0x00	; 0
     6fe:	90 e0       	ldi	r25, 0x00	; 0
     700:	0e 94 9b 11 	call	0x2336	; 0x2336 <__floatunsisf>
	if (ntc_sensor_sample > 697) {
		retval = (int8_t)((-0.0295 * ntc_sample) + 40.5);
	} if (ntc_sensor_sample > 420) {
     704:	c5 3a       	cpi	r28, 0xA5	; 165
     706:	d1 40       	sbci	r29, 0x01	; 1
     708:	80 f0       	brcs	.+32     	; 0x72a <ntc_get_temperature+0x3c>
		retval = (int8_t)((-0.0474 * ntc_sample) + 53.3);
     70a:	21 e8       	ldi	r18, 0x81	; 129
     70c:	36 e2       	ldi	r19, 0x26	; 38
     70e:	42 e4       	ldi	r20, 0x42	; 66
     710:	5d eb       	ldi	r21, 0xBD	; 189
     712:	0e 94 6e 12 	call	0x24dc	; 0x24dc <__mulsf3>
     716:	23 e3       	ldi	r18, 0x33	; 51
     718:	33 e3       	ldi	r19, 0x33	; 51
     71a:	45 e5       	ldi	r20, 0x55	; 85
     71c:	52 e4       	ldi	r21, 0x42	; 66
     71e:	0e 94 9e 10 	call	0x213c	; 0x213c <__addsf3>
     722:	0e 94 6a 11 	call	0x22d4	; 0x22d4 <__fixsfsi>
     726:	86 2f       	mov	r24, r22
     728:	0f c0       	rjmp	.+30     	; 0x748 <ntc_get_temperature+0x5a>
	} else {
		retval = (int8_t)((-0.0777 * ntc_sample) + 65.1);
     72a:	2d e2       	ldi	r18, 0x2D	; 45
     72c:	31 e2       	ldi	r19, 0x21	; 33
     72e:	4f e9       	ldi	r20, 0x9F	; 159
     730:	5d eb       	ldi	r21, 0xBD	; 189
     732:	0e 94 6e 12 	call	0x24dc	; 0x24dc <__mulsf3>
     736:	23 e3       	ldi	r18, 0x33	; 51
     738:	33 e3       	ldi	r19, 0x33	; 51
     73a:	42 e8       	ldi	r20, 0x82	; 130
     73c:	52 e4       	ldi	r21, 0x42	; 66
     73e:	0e 94 9e 10 	call	0x213c	; 0x213c <__addsf3>
     742:	0e 94 6a 11 	call	0x22d4	; 0x22d4 <__fixsfsi>
     746:	86 2f       	mov	r24, r22
	}
	return retval;
}
     748:	df 91       	pop	r29
     74a:	cf 91       	pop	r28
     74c:	08 95       	ret

0000074e <__portable_avr_delay_cycles>:
 *
 * @{
 */
__always_optimize
static inline void __portable_avr_delay_cycles(unsigned long n)
{
     74e:	04 c0       	rjmp	.+8      	; 0x758 <__portable_avr_delay_cycles+0xa>
	while (n) {
		barrier();
		n--;
     750:	61 50       	subi	r22, 0x01	; 1
     752:	71 09       	sbc	r23, r1
     754:	81 09       	sbc	r24, r1
     756:	91 09       	sbc	r25, r1
 * @{
 */
__always_optimize
static inline void __portable_avr_delay_cycles(unsigned long n)
{
	while (n) {
     758:	61 15       	cp	r22, r1
     75a:	71 05       	cpc	r23, r1
     75c:	81 05       	cpc	r24, r1
     75e:	91 05       	cpc	r25, r1
     760:	b9 f7       	brne	.-18     	; 0x750 <__portable_avr_delay_cycles+0x2>
     762:	08 95       	ret

00000764 <st7565r_init>:
 * Call this function to initialize the hardware interface and the LCD
 * controller. When initialization is done the display is turned on and ready
 * to receive data.
 */
void st7565r_init(void)
{
     764:	bf 92       	push	r11
     766:	cf 92       	push	r12
     768:	df 92       	push	r13
     76a:	ef 92       	push	r14
     76c:	ff 92       	push	r15
     76e:	0f 93       	push	r16
     770:	1f 93       	push	r17
     772:	cf 93       	push	r28
     774:	df 93       	push	r29
     776:	1f 92       	push	r1
     778:	cd b7       	in	r28, 0x3d	; 61
     77a:	de b7       	in	r29, 0x3e	; 62
	PORT_t *base = arch_ioport_pin_to_base(pin);

	if (level) {
		base->OUTSET = arch_ioport_pin_to_mask(pin);
	} else {
		base->OUTCLR = arch_ioport_pin_to_mask(pin);
     77c:	00 e0       	ldi	r16, 0x00	; 0
     77e:	16 e0       	ldi	r17, 0x06	; 6
     780:	68 94       	set
     782:	ff 24       	eor	r15, r15
     784:	f3 f8       	bld	r15, 3
     786:	f8 01       	movw	r30, r16
     788:	f6 82       	std	Z+6, r15	; 0x06
 * function, this command will control the RST pin.
 */
static inline void st7565r_hard_reset(void)
{
	ioport_set_pin_low(ST7565R_RESET_PIN);
	delay_us(10);
     78a:	64 e0       	ldi	r22, 0x04	; 4
     78c:	70 e0       	ldi	r23, 0x00	; 0
     78e:	80 e0       	ldi	r24, 0x00	; 0
     790:	90 e0       	ldi	r25, 0x00	; 0
     792:	dd df       	rcall	.-70     	; 0x74e <__portable_avr_delay_cycles>
		bool level)
{
	PORT_t *base = arch_ioport_pin_to_base(pin);

	if (level) {
		base->OUTSET = arch_ioport_pin_to_mask(pin);
     794:	f8 01       	movw	r30, r16
     796:	f5 82       	std	Z+5, r15	; 0x05
	ioport_set_pin_high(ST7565R_RESET_PIN);
	delay_us(10);
     798:	64 e0       	ldi	r22, 0x04	; 4
     79a:	70 e0       	ldi	r23, 0x00	; 0
     79c:	80 e0       	ldi	r24, 0x00	; 0
     79e:	90 e0       	ldi	r25, 0x00	; 0
     7a0:	d6 df       	rcall	.-84     	; 0x74e <__portable_avr_delay_cycles>
	spi_flags_t spi_flags = SPI_MODE_3;
	board_spi_select_id_t spi_select_id = 0;
#endif

#if defined(ST7565R_USART_SPI_INTERFACE)
	struct usart_spi_device device = {
     7a2:	0f 2e       	mov	r0, r31
     7a4:	fb e2       	ldi	r31, 0x2B	; 43
     7a6:	bf 2e       	mov	r11, r31
     7a8:	f0 2d       	mov	r31, r0
     7aa:	b9 82       	std	Y+1, r11	; 0x01
		.id = ST7565R_CS_PIN,
	};
	usart_spi_init(ST7565R_USART_SPI);
     7ac:	80 ea       	ldi	r24, 0xA0	; 160
     7ae:	99 e0       	ldi	r25, 0x09	; 9
     7b0:	0e 94 02 0c 	call	0x1804	; 0x1804 <usart_spi_init>
	usart_spi_setup_device(ST7565R_USART_SPI, &device, spi_flags,
     7b4:	c1 2c       	mov	r12, r1
     7b6:	d1 2c       	mov	r13, r1
     7b8:	76 01       	movw	r14, r12
     7ba:	00 e4       	ldi	r16, 0x40	; 64
     7bc:	12 e4       	ldi	r17, 0x42	; 66
     7be:	2f e0       	ldi	r18, 0x0F	; 15
     7c0:	30 e0       	ldi	r19, 0x00	; 0
     7c2:	43 e0       	ldi	r20, 0x03	; 3
     7c4:	be 01       	movw	r22, r28
     7c6:	6f 5f       	subi	r22, 0xFF	; 255
     7c8:	7f 4f       	sbci	r23, 0xFF	; 255
     7ca:	80 ea       	ldi	r24, 0xA0	; 160
     7cc:	99 e0       	ldi	r25, 0x09	; 9
     7ce:	0e 94 31 0c 	call	0x1862	; 0x1862 <usart_spi_setup_device>
	} else {
		base->OUTCLR = arch_ioport_pin_to_mask(pin);
     7d2:	00 e6       	ldi	r16, 0x60	; 96
     7d4:	16 e0       	ldi	r17, 0x06	; 6
     7d6:	ff 24       	eor	r15, r15
     7d8:	f3 94       	inc	r15
     7da:	f8 01       	movw	r30, r16
     7dc:	f6 82       	std	Z+6, r15	; 0x06
 * \param command the command to write
 */
static inline void st7565r_write_command(uint8_t command)
{
#if defined(ST7565R_USART_SPI_INTERFACE)
	struct usart_spi_device device = {.id = ST7565R_CS_PIN};
     7de:	b9 82       	std	Y+1, r11	; 0x01
	usart_spi_select_device(ST7565R_USART_SPI, &device);
     7e0:	be 01       	movw	r22, r28
     7e2:	6f 5f       	subi	r22, 0xFF	; 255
     7e4:	7f 4f       	sbci	r23, 0xFF	; 255
     7e6:	80 ea       	ldi	r24, 0xA0	; 160
     7e8:	99 e0       	ldi	r25, 0x09	; 9
     7ea:	0e 94 4b 0c 	call	0x1896	; 0x1896 <usart_spi_select_device>
     7ee:	f8 01       	movw	r30, r16
     7f0:	f6 82       	std	Z+6, r15	; 0x06
 *
 * \param usart The USART module.
 */
static inline bool usart_data_register_is_empty(USART_t * usart)
{
	return (usart)->STATUS & USART_DREIF_bm;
     7f2:	e0 ea       	ldi	r30, 0xA0	; 160
     7f4:	f9 e0       	ldi	r31, 0x09	; 9
     7f6:	81 81       	ldd	r24, Z+1	; 0x01
 * \return The received data
 */
static inline uint8_t usart_spi_transmit(USART_t * usart,
		uint8_t txdata)
{
	while (usart_data_register_is_empty(usart) == false);
     7f8:	85 ff       	sbrs	r24, 5
     7fa:	fd cf       	rjmp	.-6      	; 0x7f6 <st7565r_init+0x92>
 * \param usart The USART module.
 * \param txdata The data to be transmitted.
 */
static inline void usart_put(USART_t * usart, uint8_t txdata)
{
	(usart)->DATA = txdata;
     7fc:	80 ea       	ldi	r24, 0xA0	; 160
     7fe:	80 93 a0 09 	sts	0x09A0, r24	; 0x8009a0 <__TEXT_REGION_LENGTH__+0x7be9a0>
 *
 * \param usart The USART module.
 */
static inline bool usart_tx_is_complete(USART_t * usart)
{
	return (usart)->STATUS & USART_TXCIF_bm;
     802:	e0 ea       	ldi	r30, 0xA0	; 160
     804:	f9 e0       	ldi	r31, 0x09	; 9
     806:	81 81       	ldd	r24, Z+1	; 0x01
static inline uint8_t usart_spi_transmit(USART_t * usart,
		uint8_t txdata)
{
	while (usart_data_register_is_empty(usart) == false);
	usart_put(usart, txdata);
	while (!usart_tx_is_complete(usart));
     808:	86 ff       	sbrs	r24, 6
     80a:	fd cf       	rjmp	.-6      	; 0x806 <st7565r_init+0xa2>
 *
 * \param usart The USART module.
 */
static inline void usart_clear_tx_complete(USART_t * usart)
{
	(usart)->STATUS = USART_TXCIF_bm;
     80c:	e0 ea       	ldi	r30, 0xA0	; 160
     80e:	f9 e0       	ldi	r31, 0x09	; 9
     810:	80 e4       	ldi	r24, 0x40	; 64
     812:	81 83       	std	Z+1, r24	; 0x01
 *
 * \return The received data
 */
static inline uint8_t usart_get(USART_t * usart)
{
	return (usart)->DATA;
     814:	80 81       	ld	r24, Z
	ioport_set_pin_low(ST7565R_A0_PIN);
	usart_spi_transmit(ST7565R_USART_SPI, command);
	usart_spi_deselect_device(ST7565R_USART_SPI, &device);
     816:	be 01       	movw	r22, r28
     818:	6f 5f       	subi	r22, 0xFF	; 255
     81a:	7f 4f       	sbci	r23, 0xFF	; 255
     81c:	80 ea       	ldi	r24, 0xA0	; 160
     81e:	99 e0       	ldi	r25, 0x09	; 9
     820:	0e 94 61 0c 	call	0x18c2	; 0x18c2 <usart_spi_deselect_device>
 * \param command the command to write
 */
static inline void st7565r_write_command(uint8_t command)
{
#if defined(ST7565R_USART_SPI_INTERFACE)
	struct usart_spi_device device = {.id = ST7565R_CS_PIN};
     824:	8b e2       	ldi	r24, 0x2B	; 43
     826:	89 83       	std	Y+1, r24	; 0x01
	usart_spi_select_device(ST7565R_USART_SPI, &device);
     828:	be 01       	movw	r22, r28
     82a:	6f 5f       	subi	r22, 0xFF	; 255
     82c:	7f 4f       	sbci	r23, 0xFF	; 255
     82e:	80 ea       	ldi	r24, 0xA0	; 160
     830:	99 e0       	ldi	r25, 0x09	; 9
     832:	0e 94 4b 0c 	call	0x1896	; 0x1896 <usart_spi_select_device>
     836:	81 e0       	ldi	r24, 0x01	; 1
     838:	80 93 66 06 	sts	0x0666, r24	; 0x800666 <__TEXT_REGION_LENGTH__+0x7be666>
 *
 * \param usart The USART module.
 */
static inline bool usart_data_register_is_empty(USART_t * usart)
{
	return (usart)->STATUS & USART_DREIF_bm;
     83c:	e0 ea       	ldi	r30, 0xA0	; 160
     83e:	f9 e0       	ldi	r31, 0x09	; 9
     840:	81 81       	ldd	r24, Z+1	; 0x01
 * \return The received data
 */
static inline uint8_t usart_spi_transmit(USART_t * usart,
		uint8_t txdata)
{
	while (usart_data_register_is_empty(usart) == false);
     842:	85 ff       	sbrs	r24, 5
     844:	fd cf       	rjmp	.-6      	; 0x840 <st7565r_init+0xdc>
 * \param usart The USART module.
 * \param txdata The data to be transmitted.
 */
static inline void usart_put(USART_t * usart, uint8_t txdata)
{
	(usart)->DATA = txdata;
     846:	86 ea       	ldi	r24, 0xA6	; 166
     848:	80 93 a0 09 	sts	0x09A0, r24	; 0x8009a0 <__TEXT_REGION_LENGTH__+0x7be9a0>
 *
 * \param usart The USART module.
 */
static inline bool usart_tx_is_complete(USART_t * usart)
{
	return (usart)->STATUS & USART_TXCIF_bm;
     84c:	e0 ea       	ldi	r30, 0xA0	; 160
     84e:	f9 e0       	ldi	r31, 0x09	; 9
     850:	81 81       	ldd	r24, Z+1	; 0x01
static inline uint8_t usart_spi_transmit(USART_t * usart,
		uint8_t txdata)
{
	while (usart_data_register_is_empty(usart) == false);
	usart_put(usart, txdata);
	while (!usart_tx_is_complete(usart));
     852:	86 ff       	sbrs	r24, 6
     854:	fd cf       	rjmp	.-6      	; 0x850 <st7565r_init+0xec>
 *
 * \param usart The USART module.
 */
static inline void usart_clear_tx_complete(USART_t * usart)
{
	(usart)->STATUS = USART_TXCIF_bm;
     856:	e0 ea       	ldi	r30, 0xA0	; 160
     858:	f9 e0       	ldi	r31, 0x09	; 9
     85a:	80 e4       	ldi	r24, 0x40	; 64
     85c:	81 83       	std	Z+1, r24	; 0x01
 *
 * \return The received data
 */
static inline uint8_t usart_get(USART_t * usart)
{
	return (usart)->DATA;
     85e:	80 81       	ld	r24, Z
	ioport_set_pin_low(ST7565R_A0_PIN);
	usart_spi_transmit(ST7565R_USART_SPI, command);
	usart_spi_deselect_device(ST7565R_USART_SPI, &device);
     860:	be 01       	movw	r22, r28
     862:	6f 5f       	subi	r22, 0xFF	; 255
     864:	7f 4f       	sbci	r23, 0xFF	; 255
     866:	80 ea       	ldi	r24, 0xA0	; 160
     868:	99 e0       	ldi	r25, 0x09	; 9
     86a:	0e 94 61 0c 	call	0x18c2	; 0x18c2 <usart_spi_deselect_device>
 * \param command the command to write
 */
static inline void st7565r_write_command(uint8_t command)
{
#if defined(ST7565R_USART_SPI_INTERFACE)
	struct usart_spi_device device = {.id = ST7565R_CS_PIN};
     86e:	8b e2       	ldi	r24, 0x2B	; 43
     870:	89 83       	std	Y+1, r24	; 0x01
	usart_spi_select_device(ST7565R_USART_SPI, &device);
     872:	be 01       	movw	r22, r28
     874:	6f 5f       	subi	r22, 0xFF	; 255
     876:	7f 4f       	sbci	r23, 0xFF	; 255
     878:	80 ea       	ldi	r24, 0xA0	; 160
     87a:	99 e0       	ldi	r25, 0x09	; 9
     87c:	0e 94 4b 0c 	call	0x1896	; 0x1896 <usart_spi_select_device>
     880:	81 e0       	ldi	r24, 0x01	; 1
     882:	80 93 66 06 	sts	0x0666, r24	; 0x800666 <__TEXT_REGION_LENGTH__+0x7be666>
 *
 * \param usart The USART module.
 */
static inline bool usart_data_register_is_empty(USART_t * usart)
{
	return (usart)->STATUS & USART_DREIF_bm;
     886:	e0 ea       	ldi	r30, 0xA0	; 160
     888:	f9 e0       	ldi	r31, 0x09	; 9
     88a:	81 81       	ldd	r24, Z+1	; 0x01
 * \return The received data
 */
static inline uint8_t usart_spi_transmit(USART_t * usart,
		uint8_t txdata)
{
	while (usart_data_register_is_empty(usart) == false);
     88c:	85 ff       	sbrs	r24, 5
     88e:	fd cf       	rjmp	.-6      	; 0x88a <st7565r_init+0x126>
 * \param usart The USART module.
 * \param txdata The data to be transmitted.
 */
static inline void usart_put(USART_t * usart, uint8_t txdata)
{
	(usart)->DATA = txdata;
     890:	88 ec       	ldi	r24, 0xC8	; 200
     892:	80 93 a0 09 	sts	0x09A0, r24	; 0x8009a0 <__TEXT_REGION_LENGTH__+0x7be9a0>
 *
 * \param usart The USART module.
 */
static inline bool usart_tx_is_complete(USART_t * usart)
{
	return (usart)->STATUS & USART_TXCIF_bm;
     896:	e0 ea       	ldi	r30, 0xA0	; 160
     898:	f9 e0       	ldi	r31, 0x09	; 9
     89a:	81 81       	ldd	r24, Z+1	; 0x01
static inline uint8_t usart_spi_transmit(USART_t * usart,
		uint8_t txdata)
{
	while (usart_data_register_is_empty(usart) == false);
	usart_put(usart, txdata);
	while (!usart_tx_is_complete(usart));
     89c:	86 ff       	sbrs	r24, 6
     89e:	fd cf       	rjmp	.-6      	; 0x89a <st7565r_init+0x136>
 *
 * \param usart The USART module.
 */
static inline void usart_clear_tx_complete(USART_t * usart)
{
	(usart)->STATUS = USART_TXCIF_bm;
     8a0:	e0 ea       	ldi	r30, 0xA0	; 160
     8a2:	f9 e0       	ldi	r31, 0x09	; 9
     8a4:	80 e4       	ldi	r24, 0x40	; 64
     8a6:	81 83       	std	Z+1, r24	; 0x01
 *
 * \return The received data
 */
static inline uint8_t usart_get(USART_t * usart)
{
	return (usart)->DATA;
     8a8:	80 81       	ld	r24, Z
	ioport_set_pin_low(ST7565R_A0_PIN);
	usart_spi_transmit(ST7565R_USART_SPI, command);
	usart_spi_deselect_device(ST7565R_USART_SPI, &device);
     8aa:	be 01       	movw	r22, r28
     8ac:	6f 5f       	subi	r22, 0xFF	; 255
     8ae:	7f 4f       	sbci	r23, 0xFF	; 255
     8b0:	80 ea       	ldi	r24, 0xA0	; 160
     8b2:	99 e0       	ldi	r25, 0x09	; 9
     8b4:	0e 94 61 0c 	call	0x18c2	; 0x18c2 <usart_spi_deselect_device>
 * \param command the command to write
 */
static inline void st7565r_write_command(uint8_t command)
{
#if defined(ST7565R_USART_SPI_INTERFACE)
	struct usart_spi_device device = {.id = ST7565R_CS_PIN};
     8b8:	8b e2       	ldi	r24, 0x2B	; 43
     8ba:	89 83       	std	Y+1, r24	; 0x01
	usart_spi_select_device(ST7565R_USART_SPI, &device);
     8bc:	be 01       	movw	r22, r28
     8be:	6f 5f       	subi	r22, 0xFF	; 255
     8c0:	7f 4f       	sbci	r23, 0xFF	; 255
     8c2:	80 ea       	ldi	r24, 0xA0	; 160
     8c4:	99 e0       	ldi	r25, 0x09	; 9
     8c6:	e7 d7       	rcall	.+4046   	; 0x1896 <usart_spi_select_device>
     8c8:	81 e0       	ldi	r24, 0x01	; 1
     8ca:	80 93 66 06 	sts	0x0666, r24	; 0x800666 <__TEXT_REGION_LENGTH__+0x7be666>
 *
 * \param usart The USART module.
 */
static inline bool usart_data_register_is_empty(USART_t * usart)
{
	return (usart)->STATUS & USART_DREIF_bm;
     8ce:	e0 ea       	ldi	r30, 0xA0	; 160
     8d0:	f9 e0       	ldi	r31, 0x09	; 9
     8d2:	81 81       	ldd	r24, Z+1	; 0x01
 * \return The received data
 */
static inline uint8_t usart_spi_transmit(USART_t * usart,
		uint8_t txdata)
{
	while (usart_data_register_is_empty(usart) == false);
     8d4:	85 ff       	sbrs	r24, 5
     8d6:	fd cf       	rjmp	.-6      	; 0x8d2 <st7565r_init+0x16e>
 * \param usart The USART module.
 * \param txdata The data to be transmitted.
 */
static inline void usart_put(USART_t * usart, uint8_t txdata)
{
	(usart)->DATA = txdata;
     8d8:	82 ea       	ldi	r24, 0xA2	; 162
     8da:	80 93 a0 09 	sts	0x09A0, r24	; 0x8009a0 <__TEXT_REGION_LENGTH__+0x7be9a0>
 *
 * \param usart The USART module.
 */
static inline bool usart_tx_is_complete(USART_t * usart)
{
	return (usart)->STATUS & USART_TXCIF_bm;
     8de:	e0 ea       	ldi	r30, 0xA0	; 160
     8e0:	f9 e0       	ldi	r31, 0x09	; 9
     8e2:	81 81       	ldd	r24, Z+1	; 0x01
static inline uint8_t usart_spi_transmit(USART_t * usart,
		uint8_t txdata)
{
	while (usart_data_register_is_empty(usart) == false);
	usart_put(usart, txdata);
	while (!usart_tx_is_complete(usart));
     8e4:	86 ff       	sbrs	r24, 6
     8e6:	fd cf       	rjmp	.-6      	; 0x8e2 <st7565r_init+0x17e>
 *
 * \param usart The USART module.
 */
static inline void usart_clear_tx_complete(USART_t * usart)
{
	(usart)->STATUS = USART_TXCIF_bm;
     8e8:	e0 ea       	ldi	r30, 0xA0	; 160
     8ea:	f9 e0       	ldi	r31, 0x09	; 9
     8ec:	80 e4       	ldi	r24, 0x40	; 64
     8ee:	81 83       	std	Z+1, r24	; 0x01
 *
 * \return The received data
 */
static inline uint8_t usart_get(USART_t * usart)
{
	return (usart)->DATA;
     8f0:	80 81       	ld	r24, Z
	ioport_set_pin_low(ST7565R_A0_PIN);
	usart_spi_transmit(ST7565R_USART_SPI, command);
	usart_spi_deselect_device(ST7565R_USART_SPI, &device);
     8f2:	be 01       	movw	r22, r28
     8f4:	6f 5f       	subi	r22, 0xFF	; 255
     8f6:	7f 4f       	sbci	r23, 0xFF	; 255
     8f8:	80 ea       	ldi	r24, 0xA0	; 160
     8fa:	99 e0       	ldi	r25, 0x09	; 9
     8fc:	e2 d7       	rcall	.+4036   	; 0x18c2 <usart_spi_deselect_device>
 * \param command the command to write
 */
static inline void st7565r_write_command(uint8_t command)
{
#if defined(ST7565R_USART_SPI_INTERFACE)
	struct usart_spi_device device = {.id = ST7565R_CS_PIN};
     8fe:	8b e2       	ldi	r24, 0x2B	; 43
     900:	89 83       	std	Y+1, r24	; 0x01
	usart_spi_select_device(ST7565R_USART_SPI, &device);
     902:	be 01       	movw	r22, r28
     904:	6f 5f       	subi	r22, 0xFF	; 255
     906:	7f 4f       	sbci	r23, 0xFF	; 255
     908:	80 ea       	ldi	r24, 0xA0	; 160
     90a:	99 e0       	ldi	r25, 0x09	; 9
     90c:	c4 d7       	rcall	.+3976   	; 0x1896 <usart_spi_select_device>
     90e:	81 e0       	ldi	r24, 0x01	; 1
     910:	80 93 66 06 	sts	0x0666, r24	; 0x800666 <__TEXT_REGION_LENGTH__+0x7be666>
 *
 * \param usart The USART module.
 */
static inline bool usart_data_register_is_empty(USART_t * usart)
{
	return (usart)->STATUS & USART_DREIF_bm;
     914:	e0 ea       	ldi	r30, 0xA0	; 160
     916:	f9 e0       	ldi	r31, 0x09	; 9
     918:	81 81       	ldd	r24, Z+1	; 0x01
 * \return The received data
 */
static inline uint8_t usart_spi_transmit(USART_t * usart,
		uint8_t txdata)
{
	while (usart_data_register_is_empty(usart) == false);
     91a:	85 ff       	sbrs	r24, 5
     91c:	fd cf       	rjmp	.-6      	; 0x918 <st7565r_init+0x1b4>
 * \param usart The USART module.
 * \param txdata The data to be transmitted.
 */
static inline void usart_put(USART_t * usart, uint8_t txdata)
{
	(usart)->DATA = txdata;
     91e:	8f e2       	ldi	r24, 0x2F	; 47
     920:	80 93 a0 09 	sts	0x09A0, r24	; 0x8009a0 <__TEXT_REGION_LENGTH__+0x7be9a0>
 *
 * \param usart The USART module.
 */
static inline bool usart_tx_is_complete(USART_t * usart)
{
	return (usart)->STATUS & USART_TXCIF_bm;
     924:	e0 ea       	ldi	r30, 0xA0	; 160
     926:	f9 e0       	ldi	r31, 0x09	; 9
     928:	81 81       	ldd	r24, Z+1	; 0x01
static inline uint8_t usart_spi_transmit(USART_t * usart,
		uint8_t txdata)
{
	while (usart_data_register_is_empty(usart) == false);
	usart_put(usart, txdata);
	while (!usart_tx_is_complete(usart));
     92a:	86 ff       	sbrs	r24, 6
     92c:	fd cf       	rjmp	.-6      	; 0x928 <st7565r_init+0x1c4>
 *
 * \param usart The USART module.
 */
static inline void usart_clear_tx_complete(USART_t * usart)
{
	(usart)->STATUS = USART_TXCIF_bm;
     92e:	e0 ea       	ldi	r30, 0xA0	; 160
     930:	f9 e0       	ldi	r31, 0x09	; 9
     932:	80 e4       	ldi	r24, 0x40	; 64
     934:	81 83       	std	Z+1, r24	; 0x01
 *
 * \return The received data
 */
static inline uint8_t usart_get(USART_t * usart)
{
	return (usart)->DATA;
     936:	80 81       	ld	r24, Z
	ioport_set_pin_low(ST7565R_A0_PIN);
	usart_spi_transmit(ST7565R_USART_SPI, command);
	usart_spi_deselect_device(ST7565R_USART_SPI, &device);
     938:	be 01       	movw	r22, r28
     93a:	6f 5f       	subi	r22, 0xFF	; 255
     93c:	7f 4f       	sbci	r23, 0xFF	; 255
     93e:	80 ea       	ldi	r24, 0xA0	; 160
     940:	99 e0       	ldi	r25, 0x09	; 9
     942:	bf d7       	rcall	.+3966   	; 0x18c2 <usart_spi_deselect_device>
 * \param command the command to write
 */
static inline void st7565r_write_command(uint8_t command)
{
#if defined(ST7565R_USART_SPI_INTERFACE)
	struct usart_spi_device device = {.id = ST7565R_CS_PIN};
     944:	8b e2       	ldi	r24, 0x2B	; 43
     946:	89 83       	std	Y+1, r24	; 0x01
	usart_spi_select_device(ST7565R_USART_SPI, &device);
     948:	be 01       	movw	r22, r28
     94a:	6f 5f       	subi	r22, 0xFF	; 255
     94c:	7f 4f       	sbci	r23, 0xFF	; 255
     94e:	80 ea       	ldi	r24, 0xA0	; 160
     950:	99 e0       	ldi	r25, 0x09	; 9
     952:	a1 d7       	rcall	.+3906   	; 0x1896 <usart_spi_select_device>
     954:	81 e0       	ldi	r24, 0x01	; 1
     956:	80 93 66 06 	sts	0x0666, r24	; 0x800666 <__TEXT_REGION_LENGTH__+0x7be666>
 *
 * \param usart The USART module.
 */
static inline bool usart_data_register_is_empty(USART_t * usart)
{
	return (usart)->STATUS & USART_DREIF_bm;
     95a:	e0 ea       	ldi	r30, 0xA0	; 160
     95c:	f9 e0       	ldi	r31, 0x09	; 9
     95e:	81 81       	ldd	r24, Z+1	; 0x01
 * \return The received data
 */
static inline uint8_t usart_spi_transmit(USART_t * usart,
		uint8_t txdata)
{
	while (usart_data_register_is_empty(usart) == false);
     960:	85 ff       	sbrs	r24, 5
     962:	fd cf       	rjmp	.-6      	; 0x95e <st7565r_init+0x1fa>
 * \param usart The USART module.
 * \param txdata The data to be transmitted.
 */
static inline void usart_put(USART_t * usart, uint8_t txdata)
{
	(usart)->DATA = txdata;
     964:	88 ef       	ldi	r24, 0xF8	; 248
     966:	80 93 a0 09 	sts	0x09A0, r24	; 0x8009a0 <__TEXT_REGION_LENGTH__+0x7be9a0>
 *
 * \param usart The USART module.
 */
static inline bool usart_tx_is_complete(USART_t * usart)
{
	return (usart)->STATUS & USART_TXCIF_bm;
     96a:	e0 ea       	ldi	r30, 0xA0	; 160
     96c:	f9 e0       	ldi	r31, 0x09	; 9
     96e:	81 81       	ldd	r24, Z+1	; 0x01
static inline uint8_t usart_spi_transmit(USART_t * usart,
		uint8_t txdata)
{
	while (usart_data_register_is_empty(usart) == false);
	usart_put(usart, txdata);
	while (!usart_tx_is_complete(usart));
     970:	86 ff       	sbrs	r24, 6
     972:	fd cf       	rjmp	.-6      	; 0x96e <st7565r_init+0x20a>
 *
 * \param usart The USART module.
 */
static inline void usart_clear_tx_complete(USART_t * usart)
{
	(usart)->STATUS = USART_TXCIF_bm;
     974:	e0 ea       	ldi	r30, 0xA0	; 160
     976:	f9 e0       	ldi	r31, 0x09	; 9
     978:	80 e4       	ldi	r24, 0x40	; 64
     97a:	81 83       	std	Z+1, r24	; 0x01
 *
 * \return The received data
 */
static inline uint8_t usart_get(USART_t * usart)
{
	return (usart)->DATA;
     97c:	80 81       	ld	r24, Z
	ioport_set_pin_low(ST7565R_A0_PIN);
	usart_spi_transmit(ST7565R_USART_SPI, command);
	usart_spi_deselect_device(ST7565R_USART_SPI, &device);
     97e:	be 01       	movw	r22, r28
     980:	6f 5f       	subi	r22, 0xFF	; 255
     982:	7f 4f       	sbci	r23, 0xFF	; 255
     984:	80 ea       	ldi	r24, 0xA0	; 160
     986:	99 e0       	ldi	r25, 0x09	; 9
     988:	9c d7       	rcall	.+3896   	; 0x18c2 <usart_spi_deselect_device>
 * \param command the command to write
 */
static inline void st7565r_write_command(uint8_t command)
{
#if defined(ST7565R_USART_SPI_INTERFACE)
	struct usart_spi_device device = {.id = ST7565R_CS_PIN};
     98a:	8b e2       	ldi	r24, 0x2B	; 43
     98c:	89 83       	std	Y+1, r24	; 0x01
	usart_spi_select_device(ST7565R_USART_SPI, &device);
     98e:	be 01       	movw	r22, r28
     990:	6f 5f       	subi	r22, 0xFF	; 255
     992:	7f 4f       	sbci	r23, 0xFF	; 255
     994:	80 ea       	ldi	r24, 0xA0	; 160
     996:	99 e0       	ldi	r25, 0x09	; 9
     998:	7e d7       	rcall	.+3836   	; 0x1896 <usart_spi_select_device>
     99a:	81 e0       	ldi	r24, 0x01	; 1
     99c:	80 93 66 06 	sts	0x0666, r24	; 0x800666 <__TEXT_REGION_LENGTH__+0x7be666>
 *
 * \param usart The USART module.
 */
static inline bool usart_data_register_is_empty(USART_t * usart)
{
	return (usart)->STATUS & USART_DREIF_bm;
     9a0:	e0 ea       	ldi	r30, 0xA0	; 160
     9a2:	f9 e0       	ldi	r31, 0x09	; 9
     9a4:	81 81       	ldd	r24, Z+1	; 0x01
 * \return The received data
 */
static inline uint8_t usart_spi_transmit(USART_t * usart,
		uint8_t txdata)
{
	while (usart_data_register_is_empty(usart) == false);
     9a6:	85 ff       	sbrs	r24, 5
     9a8:	fd cf       	rjmp	.-6      	; 0x9a4 <st7565r_init+0x240>
 * \param usart The USART module.
 * \param txdata The data to be transmitted.
 */
static inline void usart_put(USART_t * usart, uint8_t txdata)
{
	(usart)->DATA = txdata;
     9aa:	10 92 a0 09 	sts	0x09A0, r1	; 0x8009a0 <__TEXT_REGION_LENGTH__+0x7be9a0>
 *
 * \param usart The USART module.
 */
static inline bool usart_tx_is_complete(USART_t * usart)
{
	return (usart)->STATUS & USART_TXCIF_bm;
     9ae:	e0 ea       	ldi	r30, 0xA0	; 160
     9b0:	f9 e0       	ldi	r31, 0x09	; 9
     9b2:	81 81       	ldd	r24, Z+1	; 0x01
static inline uint8_t usart_spi_transmit(USART_t * usart,
		uint8_t txdata)
{
	while (usart_data_register_is_empty(usart) == false);
	usart_put(usart, txdata);
	while (!usart_tx_is_complete(usart));
     9b4:	86 ff       	sbrs	r24, 6
     9b6:	fd cf       	rjmp	.-6      	; 0x9b2 <st7565r_init+0x24e>
 *
 * \param usart The USART module.
 */
static inline void usart_clear_tx_complete(USART_t * usart)
{
	(usart)->STATUS = USART_TXCIF_bm;
     9b8:	e0 ea       	ldi	r30, 0xA0	; 160
     9ba:	f9 e0       	ldi	r31, 0x09	; 9
     9bc:	80 e4       	ldi	r24, 0x40	; 64
     9be:	81 83       	std	Z+1, r24	; 0x01
 *
 * \return The received data
 */
static inline uint8_t usart_get(USART_t * usart)
{
	return (usart)->DATA;
     9c0:	80 81       	ld	r24, Z
	ioport_set_pin_low(ST7565R_A0_PIN);
	usart_spi_transmit(ST7565R_USART_SPI, command);
	usart_spi_deselect_device(ST7565R_USART_SPI, &device);
     9c2:	be 01       	movw	r22, r28
     9c4:	6f 5f       	subi	r22, 0xFF	; 255
     9c6:	7f 4f       	sbci	r23, 0xFF	; 255
     9c8:	80 ea       	ldi	r24, 0xA0	; 160
     9ca:	99 e0       	ldi	r25, 0x09	; 9
     9cc:	7a d7       	rcall	.+3828   	; 0x18c2 <usart_spi_deselect_device>
 * \param command the command to write
 */
static inline void st7565r_write_command(uint8_t command)
{
#if defined(ST7565R_USART_SPI_INTERFACE)
	struct usart_spi_device device = {.id = ST7565R_CS_PIN};
     9ce:	8b e2       	ldi	r24, 0x2B	; 43
	usart_spi_select_device(ST7565R_USART_SPI, &device);
     9d0:	89 83       	std	Y+1, r24	; 0x01
     9d2:	be 01       	movw	r22, r28
     9d4:	6f 5f       	subi	r22, 0xFF	; 255
     9d6:	7f 4f       	sbci	r23, 0xFF	; 255
     9d8:	80 ea       	ldi	r24, 0xA0	; 160
     9da:	99 e0       	ldi	r25, 0x09	; 9
     9dc:	5c d7       	rcall	.+3768   	; 0x1896 <usart_spi_select_device>
     9de:	81 e0       	ldi	r24, 0x01	; 1
     9e0:	80 93 66 06 	sts	0x0666, r24	; 0x800666 <__TEXT_REGION_LENGTH__+0x7be666>
 *
 * \param usart The USART module.
 */
static inline bool usart_data_register_is_empty(USART_t * usart)
{
	return (usart)->STATUS & USART_DREIF_bm;
     9e4:	e0 ea       	ldi	r30, 0xA0	; 160
     9e6:	f9 e0       	ldi	r31, 0x09	; 9
     9e8:	81 81       	ldd	r24, Z+1	; 0x01
 * \return The received data
 */
static inline uint8_t usart_spi_transmit(USART_t * usart,
		uint8_t txdata)
{
	while (usart_data_register_is_empty(usart) == false);
     9ea:	85 ff       	sbrs	r24, 5
     9ec:	fd cf       	rjmp	.-6      	; 0x9e8 <st7565r_init+0x284>
 * \param usart The USART module.
 * \param txdata The data to be transmitted.
 */
static inline void usart_put(USART_t * usart, uint8_t txdata)
{
	(usart)->DATA = txdata;
     9ee:	81 e2       	ldi	r24, 0x21	; 33
     9f0:	80 93 a0 09 	sts	0x09A0, r24	; 0x8009a0 <__TEXT_REGION_LENGTH__+0x7be9a0>
 *
 * \param usart The USART module.
 */
static inline bool usart_tx_is_complete(USART_t * usart)
{
	return (usart)->STATUS & USART_TXCIF_bm;
     9f4:	e0 ea       	ldi	r30, 0xA0	; 160
     9f6:	f9 e0       	ldi	r31, 0x09	; 9
     9f8:	81 81       	ldd	r24, Z+1	; 0x01
static inline uint8_t usart_spi_transmit(USART_t * usart,
		uint8_t txdata)
{
	while (usart_data_register_is_empty(usart) == false);
	usart_put(usart, txdata);
	while (!usart_tx_is_complete(usart));
     9fa:	86 ff       	sbrs	r24, 6
     9fc:	fd cf       	rjmp	.-6      	; 0x9f8 <st7565r_init+0x294>
 *
 * \param usart The USART module.
 */
static inline void usart_clear_tx_complete(USART_t * usart)
{
	(usart)->STATUS = USART_TXCIF_bm;
     9fe:	e0 ea       	ldi	r30, 0xA0	; 160
     a00:	f9 e0       	ldi	r31, 0x09	; 9
     a02:	80 e4       	ldi	r24, 0x40	; 64
 *
 * \return The received data
 */
static inline uint8_t usart_get(USART_t * usart)
{
	return (usart)->DATA;
     a04:	81 83       	std	Z+1, r24	; 0x01
	ioport_set_pin_low(ST7565R_A0_PIN);
	usart_spi_transmit(ST7565R_USART_SPI, command);
	usart_spi_deselect_device(ST7565R_USART_SPI, &device);
     a06:	80 81       	ld	r24, Z
     a08:	be 01       	movw	r22, r28
     a0a:	6f 5f       	subi	r22, 0xFF	; 255
     a0c:	7f 4f       	sbci	r23, 0xFF	; 255
     a0e:	80 ea       	ldi	r24, 0xA0	; 160
     a10:	99 e0       	ldi	r25, 0x09	; 9
 * \param command the command to write
 */
static inline void st7565r_write_command(uint8_t command)
{
#if defined(ST7565R_USART_SPI_INTERFACE)
	struct usart_spi_device device = {.id = ST7565R_CS_PIN};
     a12:	57 d7       	rcall	.+3758   	; 0x18c2 <usart_spi_deselect_device>
     a14:	8b e2       	ldi	r24, 0x2B	; 43
	usart_spi_select_device(ST7565R_USART_SPI, &device);
     a16:	89 83       	std	Y+1, r24	; 0x01
     a18:	be 01       	movw	r22, r28
     a1a:	6f 5f       	subi	r22, 0xFF	; 255
     a1c:	7f 4f       	sbci	r23, 0xFF	; 255
     a1e:	80 ea       	ldi	r24, 0xA0	; 160
     a20:	99 e0       	ldi	r25, 0x09	; 9
     a22:	39 d7       	rcall	.+3698   	; 0x1896 <usart_spi_select_device>
     a24:	81 e0       	ldi	r24, 0x01	; 1
     a26:	80 93 66 06 	sts	0x0666, r24	; 0x800666 <__TEXT_REGION_LENGTH__+0x7be666>
 *
 * \param usart The USART module.
 */
static inline bool usart_data_register_is_empty(USART_t * usart)
{
	return (usart)->STATUS & USART_DREIF_bm;
     a2a:	e0 ea       	ldi	r30, 0xA0	; 160
     a2c:	f9 e0       	ldi	r31, 0x09	; 9
     a2e:	81 81       	ldd	r24, Z+1	; 0x01
 * \return The received data
 */
static inline uint8_t usart_spi_transmit(USART_t * usart,
		uint8_t txdata)
{
	while (usart_data_register_is_empty(usart) == false);
     a30:	85 ff       	sbrs	r24, 5
     a32:	fd cf       	rjmp	.-6      	; 0xa2e <st7565r_init+0x2ca>
 * \param usart The USART module.
 * \param txdata The data to be transmitted.
 */
static inline void usart_put(USART_t * usart, uint8_t txdata)
{
	(usart)->DATA = txdata;
     a34:	81 e8       	ldi	r24, 0x81	; 129
     a36:	80 93 a0 09 	sts	0x09A0, r24	; 0x8009a0 <__TEXT_REGION_LENGTH__+0x7be9a0>
 *
 * \param usart The USART module.
 */
static inline bool usart_tx_is_complete(USART_t * usart)
{
	return (usart)->STATUS & USART_TXCIF_bm;
     a3a:	e0 ea       	ldi	r30, 0xA0	; 160
     a3c:	f9 e0       	ldi	r31, 0x09	; 9
     a3e:	81 81       	ldd	r24, Z+1	; 0x01
static inline uint8_t usart_spi_transmit(USART_t * usart,
		uint8_t txdata)
{
	while (usart_data_register_is_empty(usart) == false);
	usart_put(usart, txdata);
	while (!usart_tx_is_complete(usart));
     a40:	86 ff       	sbrs	r24, 6
     a42:	fd cf       	rjmp	.-6      	; 0xa3e <st7565r_init+0x2da>
 *
 * \param usart The USART module.
 */
static inline void usart_clear_tx_complete(USART_t * usart)
{
	(usart)->STATUS = USART_TXCIF_bm;
     a44:	e0 ea       	ldi	r30, 0xA0	; 160
     a46:	f9 e0       	ldi	r31, 0x09	; 9
     a48:	80 e4       	ldi	r24, 0x40	; 64
 *
 * \return The received data
 */
static inline uint8_t usart_get(USART_t * usart)
{
	return (usart)->DATA;
     a4a:	81 83       	std	Z+1, r24	; 0x01
	ioport_set_pin_low(ST7565R_A0_PIN);
	usart_spi_transmit(ST7565R_USART_SPI, command);
	usart_spi_deselect_device(ST7565R_USART_SPI, &device);
     a4c:	80 81       	ld	r24, Z
     a4e:	be 01       	movw	r22, r28
     a50:	6f 5f       	subi	r22, 0xFF	; 255
     a52:	7f 4f       	sbci	r23, 0xFF	; 255
     a54:	80 ea       	ldi	r24, 0xA0	; 160
     a56:	99 e0       	ldi	r25, 0x09	; 9
 * \param command the command to write
 */
static inline void st7565r_write_command(uint8_t command)
{
#if defined(ST7565R_USART_SPI_INTERFACE)
	struct usart_spi_device device = {.id = ST7565R_CS_PIN};
     a58:	34 d7       	rcall	.+3688   	; 0x18c2 <usart_spi_deselect_device>
     a5a:	8b e2       	ldi	r24, 0x2B	; 43
	usart_spi_select_device(ST7565R_USART_SPI, &device);
     a5c:	89 83       	std	Y+1, r24	; 0x01
     a5e:	be 01       	movw	r22, r28
     a60:	6f 5f       	subi	r22, 0xFF	; 255
     a62:	7f 4f       	sbci	r23, 0xFF	; 255
     a64:	80 ea       	ldi	r24, 0xA0	; 160
     a66:	99 e0       	ldi	r25, 0x09	; 9
     a68:	16 d7       	rcall	.+3628   	; 0x1896 <usart_spi_select_device>
     a6a:	81 e0       	ldi	r24, 0x01	; 1
     a6c:	80 93 66 06 	sts	0x0666, r24	; 0x800666 <__TEXT_REGION_LENGTH__+0x7be666>
 *
 * \param usart The USART module.
 */
static inline bool usart_data_register_is_empty(USART_t * usart)
{
	return (usart)->STATUS & USART_DREIF_bm;
     a70:	e0 ea       	ldi	r30, 0xA0	; 160
     a72:	f9 e0       	ldi	r31, 0x09	; 9
     a74:	81 81       	ldd	r24, Z+1	; 0x01
 * \return The received data
 */
static inline uint8_t usart_spi_transmit(USART_t * usart,
		uint8_t txdata)
{
	while (usart_data_register_is_empty(usart) == false);
     a76:	85 ff       	sbrs	r24, 5
     a78:	fd cf       	rjmp	.-6      	; 0xa74 <st7565r_init+0x310>
 * \param usart The USART module.
 * \param txdata The data to be transmitted.
 */
static inline void usart_put(USART_t * usart, uint8_t txdata)
{
	(usart)->DATA = txdata;
     a7a:	81 e2       	ldi	r24, 0x21	; 33
     a7c:	80 93 a0 09 	sts	0x09A0, r24	; 0x8009a0 <__TEXT_REGION_LENGTH__+0x7be9a0>
 *
 * \param usart The USART module.
 */
static inline bool usart_tx_is_complete(USART_t * usart)
{
	return (usart)->STATUS & USART_TXCIF_bm;
     a80:	e0 ea       	ldi	r30, 0xA0	; 160
     a82:	f9 e0       	ldi	r31, 0x09	; 9
     a84:	81 81       	ldd	r24, Z+1	; 0x01
static inline uint8_t usart_spi_transmit(USART_t * usart,
		uint8_t txdata)
{
	while (usart_data_register_is_empty(usart) == false);
	usart_put(usart, txdata);
	while (!usart_tx_is_complete(usart));
     a86:	86 ff       	sbrs	r24, 6
 *
 * \param usart The USART module.
 */
static inline void usart_clear_tx_complete(USART_t * usart)
{
	(usart)->STATUS = USART_TXCIF_bm;
     a88:	fd cf       	rjmp	.-6      	; 0xa84 <st7565r_init+0x320>
     a8a:	e0 ea       	ldi	r30, 0xA0	; 160
     a8c:	f9 e0       	ldi	r31, 0x09	; 9
     a8e:	80 e4       	ldi	r24, 0x40	; 64
 *
 * \return The received data
 */
static inline uint8_t usart_get(USART_t * usart)
{
	return (usart)->DATA;
     a90:	81 83       	std	Z+1, r24	; 0x01
	ioport_set_pin_low(ST7565R_A0_PIN);
	usart_spi_transmit(ST7565R_USART_SPI, command);
	usart_spi_deselect_device(ST7565R_USART_SPI, &device);
     a92:	80 81       	ld	r24, Z
     a94:	be 01       	movw	r22, r28
     a96:	6f 5f       	subi	r22, 0xFF	; 255
     a98:	7f 4f       	sbci	r23, 0xFF	; 255
     a9a:	80 ea       	ldi	r24, 0xA0	; 160
     a9c:	99 e0       	ldi	r25, 0x09	; 9
 * \param command the command to write
 */
static inline void st7565r_write_command(uint8_t command)
{
#if defined(ST7565R_USART_SPI_INTERFACE)
	struct usart_spi_device device = {.id = ST7565R_CS_PIN};
     a9e:	11 d7       	rcall	.+3618   	; 0x18c2 <usart_spi_deselect_device>
     aa0:	8b e2       	ldi	r24, 0x2B	; 43
	usart_spi_select_device(ST7565R_USART_SPI, &device);
     aa2:	89 83       	std	Y+1, r24	; 0x01
     aa4:	be 01       	movw	r22, r28
     aa6:	6f 5f       	subi	r22, 0xFF	; 255
     aa8:	7f 4f       	sbci	r23, 0xFF	; 255
     aaa:	80 ea       	ldi	r24, 0xA0	; 160
     aac:	99 e0       	ldi	r25, 0x09	; 9
     aae:	f3 d6       	rcall	.+3558   	; 0x1896 <usart_spi_select_device>
     ab0:	81 e0       	ldi	r24, 0x01	; 1
     ab2:	80 93 66 06 	sts	0x0666, r24	; 0x800666 <__TEXT_REGION_LENGTH__+0x7be666>
 *
 * \param usart The USART module.
 */
static inline bool usart_data_register_is_empty(USART_t * usart)
{
	return (usart)->STATUS & USART_DREIF_bm;
     ab6:	e0 ea       	ldi	r30, 0xA0	; 160
     ab8:	f9 e0       	ldi	r31, 0x09	; 9
     aba:	81 81       	ldd	r24, Z+1	; 0x01
 * \return The received data
 */
static inline uint8_t usart_spi_transmit(USART_t * usart,
		uint8_t txdata)
{
	while (usart_data_register_is_empty(usart) == false);
     abc:	85 ff       	sbrs	r24, 5
     abe:	fd cf       	rjmp	.-6      	; 0xaba <st7565r_init+0x356>
 * \param usart The USART module.
 * \param txdata The data to be transmitted.
 */
static inline void usart_put(USART_t * usart, uint8_t txdata)
{
	(usart)->DATA = txdata;
     ac0:	8f ea       	ldi	r24, 0xAF	; 175
     ac2:	80 93 a0 09 	sts	0x09A0, r24	; 0x8009a0 <__TEXT_REGION_LENGTH__+0x7be9a0>
 *
 * \param usart The USART module.
 */
static inline bool usart_tx_is_complete(USART_t * usart)
{
	return (usart)->STATUS & USART_TXCIF_bm;
     ac6:	e0 ea       	ldi	r30, 0xA0	; 160
     ac8:	f9 e0       	ldi	r31, 0x09	; 9
static inline uint8_t usart_spi_transmit(USART_t * usart,
		uint8_t txdata)
{
	while (usart_data_register_is_empty(usart) == false);
	usart_put(usart, txdata);
	while (!usart_tx_is_complete(usart));
     aca:	81 81       	ldd	r24, Z+1	; 0x01
     acc:	86 ff       	sbrs	r24, 6
 *
 * \param usart The USART module.
 */
static inline void usart_clear_tx_complete(USART_t * usart)
{
	(usart)->STATUS = USART_TXCIF_bm;
     ace:	fd cf       	rjmp	.-6      	; 0xaca <st7565r_init+0x366>
     ad0:	e0 ea       	ldi	r30, 0xA0	; 160
     ad2:	f9 e0       	ldi	r31, 0x09	; 9
     ad4:	80 e4       	ldi	r24, 0x40	; 64
 *
 * \return The received data
 */
static inline uint8_t usart_get(USART_t * usart)
{
	return (usart)->DATA;
     ad6:	81 83       	std	Z+1, r24	; 0x01
	ioport_set_pin_low(ST7565R_A0_PIN);
	usart_spi_transmit(ST7565R_USART_SPI, command);
	usart_spi_deselect_device(ST7565R_USART_SPI, &device);
     ad8:	80 81       	ld	r24, Z
     ada:	be 01       	movw	r22, r28
     adc:	6f 5f       	subi	r22, 0xFF	; 255
     ade:	7f 4f       	sbci	r23, 0xFF	; 255
     ae0:	80 ea       	ldi	r24, 0xA0	; 160
     ae2:	99 e0       	ldi	r25, 0x09	; 9
     ae4:	ee d6       	rcall	.+3548   	; 0x18c2 <usart_spi_deselect_device>
	is set to the defined min*/
	st7565r_set_contrast(ST7565R_DISPLAY_CONTRAST_MIN);

	// Turn on the display
	st7565r_display_on();
}
     ae6:	0f 90       	pop	r0
     ae8:	df 91       	pop	r29
     aea:	cf 91       	pop	r28
     aec:	1f 91       	pop	r17
     aee:	0f 91       	pop	r16
     af0:	ff 90       	pop	r15
     af2:	ef 90       	pop	r14
     af4:	df 90       	pop	r13
     af6:	cf 90       	pop	r12
     af8:	bf 90       	pop	r11
     afa:	08 95       	ret

00000afc <gfx_mono_st7565r_put_byte>:
	gfx_mono_st7565r_put_byte(0, 0, 0xFF);
\endcode
 */
void gfx_mono_st7565r_put_byte(gfx_coord_t page, gfx_coord_t column,
		uint8_t data)
{
     afc:	ff 92       	push	r15
     afe:	0f 93       	push	r16
     b00:	1f 93       	push	r17
     b02:	cf 93       	push	r28
     b04:	df 93       	push	r29
     b06:	1f 92       	push	r1
     b08:	cd b7       	in	r28, 0x3d	; 61
     b0a:	de b7       	in	r29, 0x3e	; 62
     b0c:	08 2f       	mov	r16, r24
     b0e:	f6 2e       	mov	r15, r22
     b10:	14 2f       	mov	r17, r20
#ifdef CONFIG_ST7565R_FRAMEBUFFER
	gfx_mono_framebuffer_put_byte(page, column, data);
     b12:	f2 d6       	rcall	.+3556   	; 0x18f8 <gfx_mono_framebuffer_put_byte>
 */
static inline void st7565r_set_page_address(uint8_t address)
{
	// Make sure that the address is 4 bits (only 8 pages)
	address &= 0x0F;
	st7565r_write_command(ST7565R_CMD_PAGE_ADDRESS_SET(address));
     b14:	0f 70       	andi	r16, 0x0F	; 15
     b16:	00 6b       	ori	r16, 0xB0	; 176
 * \param command the command to write
 */
static inline void st7565r_write_command(uint8_t command)
{
#if defined(ST7565R_USART_SPI_INTERFACE)
	struct usart_spi_device device = {.id = ST7565R_CS_PIN};
     b18:	8b e2       	ldi	r24, 0x2B	; 43
     b1a:	89 83       	std	Y+1, r24	; 0x01
	usart_spi_select_device(ST7565R_USART_SPI, &device);
     b1c:	be 01       	movw	r22, r28
     b1e:	6f 5f       	subi	r22, 0xFF	; 255
     b20:	7f 4f       	sbci	r23, 0xFF	; 255
     b22:	80 ea       	ldi	r24, 0xA0	; 160
     b24:	99 e0       	ldi	r25, 0x09	; 9
     b26:	b7 d6       	rcall	.+3438   	; 0x1896 <usart_spi_select_device>
     b28:	81 e0       	ldi	r24, 0x01	; 1
     b2a:	80 93 66 06 	sts	0x0666, r24	; 0x800666 <__TEXT_REGION_LENGTH__+0x7be666>
 *
 * \param usart The USART module.
 */
static inline bool usart_data_register_is_empty(USART_t * usart)
{
	return (usart)->STATUS & USART_DREIF_bm;
     b2e:	e0 ea       	ldi	r30, 0xA0	; 160
     b30:	f9 e0       	ldi	r31, 0x09	; 9
     b32:	91 81       	ldd	r25, Z+1	; 0x01
 * \return The received data
 */
static inline uint8_t usart_spi_transmit(USART_t * usart,
		uint8_t txdata)
{
	while (usart_data_register_is_empty(usart) == false);
     b34:	95 ff       	sbrs	r25, 5
     b36:	fd cf       	rjmp	.-6      	; 0xb32 <gfx_mono_st7565r_put_byte+0x36>
 * \param usart The USART module.
 * \param txdata The data to be transmitted.
 */
static inline void usart_put(USART_t * usart, uint8_t txdata)
{
	(usart)->DATA = txdata;
     b38:	00 93 a0 09 	sts	0x09A0, r16	; 0x8009a0 <__TEXT_REGION_LENGTH__+0x7be9a0>
 *
 * \param usart The USART module.
 */
static inline bool usart_tx_is_complete(USART_t * usart)
{
	return (usart)->STATUS & USART_TXCIF_bm;
     b3c:	e0 ea       	ldi	r30, 0xA0	; 160
     b3e:	f9 e0       	ldi	r31, 0x09	; 9
     b40:	81 81       	ldd	r24, Z+1	; 0x01
static inline uint8_t usart_spi_transmit(USART_t * usart,
		uint8_t txdata)
{
	while (usart_data_register_is_empty(usart) == false);
	usart_put(usart, txdata);
	while (!usart_tx_is_complete(usart));
     b42:	86 ff       	sbrs	r24, 6
     b44:	fd cf       	rjmp	.-6      	; 0xb40 <gfx_mono_st7565r_put_byte+0x44>
 *
 * \param usart The USART module.
 */
static inline void usart_clear_tx_complete(USART_t * usart)
{
	(usart)->STATUS = USART_TXCIF_bm;
     b46:	e0 ea       	ldi	r30, 0xA0	; 160
     b48:	f9 e0       	ldi	r31, 0x09	; 9
     b4a:	80 e4       	ldi	r24, 0x40	; 64
     b4c:	81 83       	std	Z+1, r24	; 0x01
 *
 * \return The received data
 */
static inline uint8_t usart_get(USART_t * usart)
{
	return (usart)->DATA;
     b4e:	80 81       	ld	r24, Z
	ioport_set_pin_low(ST7565R_A0_PIN);
	usart_spi_transmit(ST7565R_USART_SPI, command);
	usart_spi_deselect_device(ST7565R_USART_SPI, &device);
     b50:	be 01       	movw	r22, r28
     b52:	6f 5f       	subi	r22, 0xFF	; 255
     b54:	7f 4f       	sbci	r23, 0xFF	; 255
     b56:	80 ea       	ldi	r24, 0xA0	; 160
     b58:	99 e0       	ldi	r25, 0x09	; 9
     b5a:	b3 d6       	rcall	.+3430   	; 0x18c2 <usart_spi_deselect_device>
 */
static inline void st7565r_set_column_address(uint8_t address)
{
	// Make sure the address is 7 bits
	address &= 0x7F;
	st7565r_write_command(ST7565R_CMD_COLUMN_ADDRESS_SET_MSB(address >> 4));
     b5c:	0f 2d       	mov	r16, r15
     b5e:	0f 77       	andi	r16, 0x7F	; 127
     b60:	02 95       	swap	r16
     b62:	0f 70       	andi	r16, 0x0F	; 15
     b64:	00 61       	ori	r16, 0x10	; 16
 * \param command the command to write
 */
static inline void st7565r_write_command(uint8_t command)
{
#if defined(ST7565R_USART_SPI_INTERFACE)
	struct usart_spi_device device = {.id = ST7565R_CS_PIN};
     b66:	8b e2       	ldi	r24, 0x2B	; 43
     b68:	89 83       	std	Y+1, r24	; 0x01
	usart_spi_select_device(ST7565R_USART_SPI, &device);
     b6a:	be 01       	movw	r22, r28
     b6c:	6f 5f       	subi	r22, 0xFF	; 255
     b6e:	7f 4f       	sbci	r23, 0xFF	; 255
     b70:	80 ea       	ldi	r24, 0xA0	; 160
     b72:	99 e0       	ldi	r25, 0x09	; 9
     b74:	90 d6       	rcall	.+3360   	; 0x1896 <usart_spi_select_device>
     b76:	81 e0       	ldi	r24, 0x01	; 1
     b78:	80 93 66 06 	sts	0x0666, r24	; 0x800666 <__TEXT_REGION_LENGTH__+0x7be666>
 *
 * \param usart The USART module.
 */
static inline bool usart_data_register_is_empty(USART_t * usart)
{
	return (usart)->STATUS & USART_DREIF_bm;
     b7c:	e0 ea       	ldi	r30, 0xA0	; 160
     b7e:	f9 e0       	ldi	r31, 0x09	; 9
     b80:	81 81       	ldd	r24, Z+1	; 0x01
 * \return The received data
 */
static inline uint8_t usart_spi_transmit(USART_t * usart,
		uint8_t txdata)
{
	while (usart_data_register_is_empty(usart) == false);
     b82:	85 ff       	sbrs	r24, 5
     b84:	fd cf       	rjmp	.-6      	; 0xb80 <gfx_mono_st7565r_put_byte+0x84>
 * \param usart The USART module.
 * \param txdata The data to be transmitted.
 */
static inline void usart_put(USART_t * usart, uint8_t txdata)
{
	(usart)->DATA = txdata;
     b86:	00 93 a0 09 	sts	0x09A0, r16	; 0x8009a0 <__TEXT_REGION_LENGTH__+0x7be9a0>
 *
 * \param usart The USART module.
 */
static inline bool usart_tx_is_complete(USART_t * usart)
{
	return (usart)->STATUS & USART_TXCIF_bm;
     b8a:	e0 ea       	ldi	r30, 0xA0	; 160
     b8c:	f9 e0       	ldi	r31, 0x09	; 9
     b8e:	81 81       	ldd	r24, Z+1	; 0x01
static inline uint8_t usart_spi_transmit(USART_t * usart,
		uint8_t txdata)
{
	while (usart_data_register_is_empty(usart) == false);
	usart_put(usart, txdata);
	while (!usart_tx_is_complete(usart));
     b90:	86 ff       	sbrs	r24, 6
     b92:	fd cf       	rjmp	.-6      	; 0xb8e <gfx_mono_st7565r_put_byte+0x92>
 *
 * \param usart The USART module.
 */
static inline void usart_clear_tx_complete(USART_t * usart)
{
	(usart)->STATUS = USART_TXCIF_bm;
     b94:	e0 ea       	ldi	r30, 0xA0	; 160
     b96:	f9 e0       	ldi	r31, 0x09	; 9
     b98:	80 e4       	ldi	r24, 0x40	; 64
     b9a:	81 83       	std	Z+1, r24	; 0x01
 *
 * \return The received data
 */
static inline uint8_t usart_get(USART_t * usart)
{
	return (usart)->DATA;
     b9c:	80 81       	ld	r24, Z
	ioport_set_pin_low(ST7565R_A0_PIN);
	usart_spi_transmit(ST7565R_USART_SPI, command);
	usart_spi_deselect_device(ST7565R_USART_SPI, &device);
     b9e:	be 01       	movw	r22, r28
     ba0:	6f 5f       	subi	r22, 0xFF	; 255
     ba2:	7f 4f       	sbci	r23, 0xFF	; 255
     ba4:	80 ea       	ldi	r24, 0xA0	; 160
     ba6:	99 e0       	ldi	r25, 0x09	; 9
     ba8:	8c d6       	rcall	.+3352   	; 0x18c2 <usart_spi_deselect_device>
static inline void st7565r_set_column_address(uint8_t address)
{
	// Make sure the address is 7 bits
	address &= 0x7F;
	st7565r_write_command(ST7565R_CMD_COLUMN_ADDRESS_SET_MSB(address >> 4));
	st7565r_write_command(ST7565R_CMD_COLUMN_ADDRESS_SET_LSB(address & 0x0F));
     baa:	0f 2d       	mov	r16, r15
     bac:	0f 70       	andi	r16, 0x0F	; 15
 * \param command the command to write
 */
static inline void st7565r_write_command(uint8_t command)
{
#if defined(ST7565R_USART_SPI_INTERFACE)
	struct usart_spi_device device = {.id = ST7565R_CS_PIN};
     bae:	8b e2       	ldi	r24, 0x2B	; 43
     bb0:	89 83       	std	Y+1, r24	; 0x01
	usart_spi_select_device(ST7565R_USART_SPI, &device);
     bb2:	be 01       	movw	r22, r28
     bb4:	6f 5f       	subi	r22, 0xFF	; 255
     bb6:	7f 4f       	sbci	r23, 0xFF	; 255
     bb8:	80 ea       	ldi	r24, 0xA0	; 160
     bba:	99 e0       	ldi	r25, 0x09	; 9
     bbc:	6c d6       	rcall	.+3288   	; 0x1896 <usart_spi_select_device>
     bbe:	81 e0       	ldi	r24, 0x01	; 1
     bc0:	80 93 66 06 	sts	0x0666, r24	; 0x800666 <__TEXT_REGION_LENGTH__+0x7be666>
 *
 * \param usart The USART module.
 */
static inline bool usart_data_register_is_empty(USART_t * usart)
{
	return (usart)->STATUS & USART_DREIF_bm;
     bc4:	e0 ea       	ldi	r30, 0xA0	; 160
     bc6:	f9 e0       	ldi	r31, 0x09	; 9
     bc8:	81 81       	ldd	r24, Z+1	; 0x01
 * \return The received data
 */
static inline uint8_t usart_spi_transmit(USART_t * usart,
		uint8_t txdata)
{
	while (usart_data_register_is_empty(usart) == false);
     bca:	85 ff       	sbrs	r24, 5
     bcc:	fd cf       	rjmp	.-6      	; 0xbc8 <gfx_mono_st7565r_put_byte+0xcc>
 * \param usart The USART module.
 * \param txdata The data to be transmitted.
 */
static inline void usart_put(USART_t * usart, uint8_t txdata)
{
	(usart)->DATA = txdata;
     bce:	00 93 a0 09 	sts	0x09A0, r16	; 0x8009a0 <__TEXT_REGION_LENGTH__+0x7be9a0>
 *
 * \param usart The USART module.
 */
static inline bool usart_tx_is_complete(USART_t * usart)
{
	return (usart)->STATUS & USART_TXCIF_bm;
     bd2:	e0 ea       	ldi	r30, 0xA0	; 160
     bd4:	f9 e0       	ldi	r31, 0x09	; 9
     bd6:	81 81       	ldd	r24, Z+1	; 0x01
static inline uint8_t usart_spi_transmit(USART_t * usart,
		uint8_t txdata)
{
	while (usart_data_register_is_empty(usart) == false);
	usart_put(usart, txdata);
	while (!usart_tx_is_complete(usart));
     bd8:	86 ff       	sbrs	r24, 6
     bda:	fd cf       	rjmp	.-6      	; 0xbd6 <gfx_mono_st7565r_put_byte+0xda>
 *
 * \param usart The USART module.
 */
static inline void usart_clear_tx_complete(USART_t * usart)
{
	(usart)->STATUS = USART_TXCIF_bm;
     bdc:	e0 ea       	ldi	r30, 0xA0	; 160
     bde:	f9 e0       	ldi	r31, 0x09	; 9
     be0:	80 e4       	ldi	r24, 0x40	; 64
     be2:	81 83       	std	Z+1, r24	; 0x01
	ioport_set_pin_low(ST7565R_A0_PIN);
	usart_spi_transmit(ST7565R_USART_SPI, command);
	usart_spi_deselect_device(ST7565R_USART_SPI, &device);
     be4:	80 81       	ld	r24, Z
     be6:	be 01       	movw	r22, r28
     be8:	6f 5f       	subi	r22, 0xFF	; 255
     bea:	7f 4f       	sbci	r23, 0xFF	; 255
     bec:	80 ea       	ldi	r24, 0xA0	; 160
     bee:	99 e0       	ldi	r25, 0x09	; 9
     bf0:	68 d6       	rcall	.+3280   	; 0x18c2 <usart_spi_deselect_device>
 * \param data the data to write
 */
static inline void st7565r_write_data(uint8_t data)
{
#if defined(ST7565R_USART_SPI_INTERFACE)
	struct usart_spi_device device = {.id = ST7565R_CS_PIN};
     bf2:	8b e2       	ldi	r24, 0x2B	; 43
	usart_spi_select_device(ST7565R_USART_SPI, &device);
     bf4:	89 83       	std	Y+1, r24	; 0x01
     bf6:	be 01       	movw	r22, r28
     bf8:	6f 5f       	subi	r22, 0xFF	; 255
     bfa:	7f 4f       	sbci	r23, 0xFF	; 255
     bfc:	80 ea       	ldi	r24, 0xA0	; 160
     bfe:	99 e0       	ldi	r25, 0x09	; 9
     c00:	4a d6       	rcall	.+3220   	; 0x1896 <usart_spi_select_device>
		bool level)
{
	PORT_t *base = arch_ioport_pin_to_base(pin);

	if (level) {
		base->OUTSET = arch_ioport_pin_to_mask(pin);
     c02:	81 e0       	ldi	r24, 0x01	; 1
     c04:	80 93 65 06 	sts	0x0665, r24	; 0x800665 <__TEXT_REGION_LENGTH__+0x7be665>
 *
 * \param usart The USART module.
 */
static inline bool usart_data_register_is_empty(USART_t * usart)
{
	return (usart)->STATUS & USART_DREIF_bm;
     c08:	e0 ea       	ldi	r30, 0xA0	; 160
     c0a:	f9 e0       	ldi	r31, 0x09	; 9
     c0c:	81 81       	ldd	r24, Z+1	; 0x01
 * \return The received data
 */
static inline uint8_t usart_spi_transmit(USART_t * usart,
		uint8_t txdata)
{
	while (usart_data_register_is_empty(usart) == false);
     c0e:	85 ff       	sbrs	r24, 5
     c10:	fd cf       	rjmp	.-6      	; 0xc0c <gfx_mono_st7565r_put_byte+0x110>
 * \param usart The USART module.
 * \param txdata The data to be transmitted.
 */
static inline void usart_put(USART_t * usart, uint8_t txdata)
{
	(usart)->DATA = txdata;
     c12:	10 93 a0 09 	sts	0x09A0, r17	; 0x8009a0 <__TEXT_REGION_LENGTH__+0x7be9a0>
 *
 * \param usart The USART module.
 */
static inline bool usart_tx_is_complete(USART_t * usart)
{
	return (usart)->STATUS & USART_TXCIF_bm;
     c16:	e0 ea       	ldi	r30, 0xA0	; 160
     c18:	f9 e0       	ldi	r31, 0x09	; 9
     c1a:	81 81       	ldd	r24, Z+1	; 0x01
static inline uint8_t usart_spi_transmit(USART_t * usart,
		uint8_t txdata)
{
	while (usart_data_register_is_empty(usart) == false);
	usart_put(usart, txdata);
	while (!usart_tx_is_complete(usart));
     c1c:	86 ff       	sbrs	r24, 6
     c1e:	fd cf       	rjmp	.-6      	; 0xc1a <gfx_mono_st7565r_put_byte+0x11e>
 *
 * \param usart The USART module.
 */
static inline void usart_clear_tx_complete(USART_t * usart)
{
	(usart)->STATUS = USART_TXCIF_bm;
     c20:	e0 ea       	ldi	r30, 0xA0	; 160
     c22:	f9 e0       	ldi	r31, 0x09	; 9
     c24:	80 e4       	ldi	r24, 0x40	; 64
     c26:	81 83       	std	Z+1, r24	; 0x01
 *
 * \return The received data
 */
static inline uint8_t usart_get(USART_t * usart)
{
	return (usart)->DATA;
     c28:	80 81       	ld	r24, Z
	} else {
		base->OUTCLR = arch_ioport_pin_to_mask(pin);
     c2a:	81 e0       	ldi	r24, 0x01	; 1
     c2c:	80 93 66 06 	sts	0x0666, r24	; 0x800666 <__TEXT_REGION_LENGTH__+0x7be666>
	ioport_set_pin_high(ST7565R_A0_PIN);
	usart_spi_transmit(ST7565R_USART_SPI, data);
	ioport_set_pin_low(ST7565R_A0_PIN);
	usart_spi_deselect_device(ST7565R_USART_SPI, &device);
     c30:	be 01       	movw	r22, r28
     c32:	6f 5f       	subi	r22, 0xFF	; 255
     c34:	7f 4f       	sbci	r23, 0xFF	; 255
     c36:	80 ea       	ldi	r24, 0xA0	; 160
     c38:	99 e0       	ldi	r25, 0x09	; 9
     c3a:	43 d6       	rcall	.+3206   	; 0x18c2 <usart_spi_deselect_device>

	st7565r_set_page_address(page);
	st7565r_set_column_address(column);

	st7565r_write_data(data);
}
     c3c:	0f 90       	pop	r0
     c3e:	df 91       	pop	r29
     c40:	cf 91       	pop	r28
     c42:	1f 91       	pop	r17
     c44:	0f 91       	pop	r16
     c46:	ff 90       	pop	r15
     c48:	08 95       	ret

00000c4a <gfx_mono_st7565r_init>:
 * It will also write the graphic controller RAM to all zeroes.
 *
 * \note This function will clear the contents of the display.
 */
void gfx_mono_st7565r_init(void)
{
     c4a:	0f 93       	push	r16
     c4c:	1f 93       	push	r17
     c4e:	cf 93       	push	r28
     c50:	df 93       	push	r29
     c52:	1f 92       	push	r1
     c54:	cd b7       	in	r28, 0x3d	; 61
     c56:	de b7       	in	r29, 0x3e	; 62
	uint8_t page;
	uint8_t column;

#ifdef CONFIG_ST7565R_FRAMEBUFFER
	gfx_mono_set_framebuffer(framebuffer);
     c58:	8e e6       	ldi	r24, 0x6E	; 110
     c5a:	90 e2       	ldi	r25, 0x20	; 32
     c5c:	48 d6       	rcall	.+3216   	; 0x18ee <gfx_mono_set_framebuffer>
#endif

	/* Initialize the low-level display controller. */
	st7565r_init();
     c5e:	82 dd       	rcall	.-1276   	; 0x764 <st7565r_init>
     c60:	8b e2       	ldi	r24, 0x2B	; 43
 * \param command the command to write
 */
static inline void st7565r_write_command(uint8_t command)
{
#if defined(ST7565R_USART_SPI_INTERFACE)
	struct usart_spi_device device = {.id = ST7565R_CS_PIN};
     c62:	89 83       	std	Y+1, r24	; 0x01
     c64:	be 01       	movw	r22, r28
	usart_spi_select_device(ST7565R_USART_SPI, &device);
     c66:	6f 5f       	subi	r22, 0xFF	; 255
     c68:	7f 4f       	sbci	r23, 0xFF	; 255
     c6a:	80 ea       	ldi	r24, 0xA0	; 160
     c6c:	99 e0       	ldi	r25, 0x09	; 9
     c6e:	13 d6       	rcall	.+3110   	; 0x1896 <usart_spi_select_device>
     c70:	81 e0       	ldi	r24, 0x01	; 1
     c72:	80 93 66 06 	sts	0x0666, r24	; 0x800666 <__TEXT_REGION_LENGTH__+0x7be666>
     c76:	e0 ea       	ldi	r30, 0xA0	; 160
 *
 * \param usart The USART module.
 */
static inline bool usart_data_register_is_empty(USART_t * usart)
{
	return (usart)->STATUS & USART_DREIF_bm;
     c78:	f9 e0       	ldi	r31, 0x09	; 9
     c7a:	81 81       	ldd	r24, Z+1	; 0x01
     c7c:	85 ff       	sbrs	r24, 5
 * \return The received data
 */
static inline uint8_t usart_spi_transmit(USART_t * usart,
		uint8_t txdata)
{
	while (usart_data_register_is_empty(usart) == false);
     c7e:	fd cf       	rjmp	.-6      	; 0xc7a <gfx_mono_st7565r_init+0x30>
     c80:	80 e4       	ldi	r24, 0x40	; 64
 * \param usart The USART module.
 * \param txdata The data to be transmitted.
 */
static inline void usart_put(USART_t * usart, uint8_t txdata)
{
	(usart)->DATA = txdata;
     c82:	80 93 a0 09 	sts	0x09A0, r24	; 0x8009a0 <__TEXT_REGION_LENGTH__+0x7be9a0>
     c86:	e0 ea       	ldi	r30, 0xA0	; 160
 *
 * \param usart The USART module.
 */
static inline bool usart_tx_is_complete(USART_t * usart)
{
	return (usart)->STATUS & USART_TXCIF_bm;
     c88:	f9 e0       	ldi	r31, 0x09	; 9
     c8a:	81 81       	ldd	r24, Z+1	; 0x01
     c8c:	86 ff       	sbrs	r24, 6
static inline uint8_t usart_spi_transmit(USART_t * usart,
		uint8_t txdata)
{
	while (usart_data_register_is_empty(usart) == false);
	usart_put(usart, txdata);
	while (!usart_tx_is_complete(usart));
     c8e:	fd cf       	rjmp	.-6      	; 0xc8a <gfx_mono_st7565r_init+0x40>
     c90:	e0 ea       	ldi	r30, 0xA0	; 160
 *
 * \param usart The USART module.
 */
static inline void usart_clear_tx_complete(USART_t * usart)
{
	(usart)->STATUS = USART_TXCIF_bm;
     c92:	f9 e0       	ldi	r31, 0x09	; 9
     c94:	80 e4       	ldi	r24, 0x40	; 64
     c96:	81 83       	std	Z+1, r24	; 0x01
     c98:	80 81       	ld	r24, Z
 *
 * \return The received data
 */
static inline uint8_t usart_get(USART_t * usart)
{
	return (usart)->DATA;
     c9a:	be 01       	movw	r22, r28
	ioport_set_pin_low(ST7565R_A0_PIN);
	usart_spi_transmit(ST7565R_USART_SPI, command);
	usart_spi_deselect_device(ST7565R_USART_SPI, &device);
     c9c:	6f 5f       	subi	r22, 0xFF	; 255
     c9e:	7f 4f       	sbci	r23, 0xFF	; 255
     ca0:	80 ea       	ldi	r24, 0xA0	; 160
     ca2:	99 e0       	ldi	r25, 0x09	; 9
     ca4:	0e d6       	rcall	.+3100   	; 0x18c2 <usart_spi_deselect_device>
     ca6:	00 e0       	ldi	r16, 0x00	; 0

	/* Clear the contents of the display.
	 * If using a framebuffer (SPI interface) it will both clear the
	 * controller memory and the framebuffer.
	 */
	for (page = 0; page < GFX_MONO_LCD_PAGES; page++) {
     ca8:	0a c0       	rjmp	.+20     	; 0xcbe <gfx_mono_st7565r_init+0x74>
		for (column = 0; column < GFX_MONO_LCD_WIDTH; column++) {
			gfx_mono_put_byte(page, column, 0x00);
     caa:	40 e0       	ldi	r20, 0x00	; 0
     cac:	61 2f       	mov	r22, r17
     cae:	80 2f       	mov	r24, r16
     cb0:	25 df       	rcall	.-438    	; 0xafc <gfx_mono_st7565r_put_byte>
     cb2:	1f 5f       	subi	r17, 0xFF	; 255
	/* Clear the contents of the display.
	 * If using a framebuffer (SPI interface) it will both clear the
	 * controller memory and the framebuffer.
	 */
	for (page = 0; page < GFX_MONO_LCD_PAGES; page++) {
		for (column = 0; column < GFX_MONO_LCD_WIDTH; column++) {
     cb4:	10 38       	cpi	r17, 0x80	; 128
     cb6:	c9 f7       	brne	.-14     	; 0xcaa <gfx_mono_st7565r_init+0x60>
     cb8:	0f 5f       	subi	r16, 0xFF	; 255

	/* Clear the contents of the display.
	 * If using a framebuffer (SPI interface) it will both clear the
	 * controller memory and the framebuffer.
	 */
	for (page = 0; page < GFX_MONO_LCD_PAGES; page++) {
     cba:	04 30       	cpi	r16, 0x04	; 4
     cbc:	11 f0       	breq	.+4      	; 0xcc2 <gfx_mono_st7565r_init+0x78>
     cbe:	10 e0       	ldi	r17, 0x00	; 0
 * It will also write the graphic controller RAM to all zeroes.
 *
 * \note This function will clear the contents of the display.
 */
void gfx_mono_st7565r_init(void)
{
     cc0:	f4 cf       	rjmp	.-24     	; 0xcaa <gfx_mono_st7565r_init+0x60>
     cc2:	0f 90       	pop	r0
	for (page = 0; page < GFX_MONO_LCD_PAGES; page++) {
		for (column = 0; column < GFX_MONO_LCD_WIDTH; column++) {
			gfx_mono_put_byte(page, column, 0x00);
		}
	}
}
     cc4:	df 91       	pop	r29
     cc6:	cf 91       	pop	r28
     cc8:	1f 91       	pop	r17
     cca:	0f 91       	pop	r16
     ccc:	08 95       	ret

00000cce <gfx_mono_st7565r_draw_pixel>:
     cce:	ff 92       	push	r15
	gfx_mono_st7565r_draw_pixel(10, 10, GFX_PIXEL_XOR);
\endcode
 */
void gfx_mono_st7565r_draw_pixel(gfx_coord_t x, gfx_coord_t y,
		gfx_coord_t color)
{
     cd0:	0f 93       	push	r16
     cd2:	1f 93       	push	r17
     cd4:	cf 93       	push	r28
     cd6:	df 93       	push	r29
	uint8_t page;
	uint8_t pixel_mask;
	uint8_t pixel_value;

	/* Discard pixels drawn outside the screen */
	if ((x > GFX_MONO_LCD_WIDTH - 1) || (y > GFX_MONO_LCD_HEIGHT - 1)) {
     cd8:	88 23       	and	r24, r24
     cda:	4c f1       	brlt	.+82     	; 0xd2e <gfx_mono_st7565r_draw_pixel+0x60>
     cdc:	60 32       	cpi	r22, 0x20	; 32
     cde:	38 f5       	brcc	.+78     	; 0xd2e <gfx_mono_st7565r_draw_pixel+0x60>
     ce0:	d4 2f       	mov	r29, r20
     ce2:	c8 2f       	mov	r28, r24
		return;
	}

	page = y / GFX_MONO_LCD_PIXELS_PER_BYTE;
     ce4:	f6 2e       	mov	r15, r22
     ce6:	f6 94       	lsr	r15
     ce8:	f6 94       	lsr	r15
     cea:	f6 94       	lsr	r15
	pixel_mask = (1 << (y - (page * 8)));
     cec:	70 e0       	ldi	r23, 0x00	; 0
     cee:	88 e0       	ldi	r24, 0x08	; 8
     cf0:	f8 9e       	mul	r15, r24
     cf2:	60 19       	sub	r22, r0
     cf4:	71 09       	sbc	r23, r1
     cf6:	11 24       	eor	r1, r1
     cf8:	81 e0       	ldi	r24, 0x01	; 1
     cfa:	90 e0       	ldi	r25, 0x00	; 0
     cfc:	8c 01       	movw	r16, r24
     cfe:	02 c0       	rjmp	.+4      	; 0xd04 <gfx_mono_st7565r_draw_pixel+0x36>
     d00:	00 0f       	add	r16, r16
     d02:	11 1f       	adc	r17, r17
     d04:	6a 95       	dec	r22
     d06:	e2 f7       	brpl	.-8      	; 0xd00 <gfx_mono_st7565r_draw_pixel+0x32>
\endcode
 */
uint8_t gfx_mono_st7565r_get_byte(gfx_coord_t page, gfx_coord_t column)
{
#ifdef CONFIG_ST7565R_FRAMEBUFFER
	return gfx_mono_framebuffer_get_byte(page, column);
     d08:	6c 2f       	mov	r22, r28
     d0a:	8f 2d       	mov	r24, r15
     d0c:	03 d6       	rcall	.+3078   	; 0x1914 <gfx_mono_framebuffer_get_byte>
	 * requested action on this pixel before writing the page back to the
	 * display.
	 */
	pixel_value = gfx_mono_get_byte(page, x);

	switch (color) {
     d0e:	d1 30       	cpi	r29, 0x01	; 1
     d10:	21 f0       	breq	.+8      	; 0xd1a <gfx_mono_st7565r_draw_pixel+0x4c>
     d12:	28 f0       	brcs	.+10     	; 0xd1e <gfx_mono_st7565r_draw_pixel+0x50>
     d14:	d2 30       	cpi	r29, 0x02	; 2
     d16:	31 f0       	breq	.+12     	; 0xd24 <gfx_mono_st7565r_draw_pixel+0x56>
     d18:	06 c0       	rjmp	.+12     	; 0xd26 <gfx_mono_st7565r_draw_pixel+0x58>
	case GFX_PIXEL_SET:
		pixel_value |= pixel_mask;
     d1a:	80 2b       	or	r24, r16
		break;
     d1c:	04 c0       	rjmp	.+8      	; 0xd26 <gfx_mono_st7565r_draw_pixel+0x58>

	case GFX_PIXEL_CLR:
		pixel_value &= ~pixel_mask;
     d1e:	00 95       	com	r16
     d20:	80 23       	and	r24, r16
		break;
     d22:	01 c0       	rjmp	.+2      	; 0xd26 <gfx_mono_st7565r_draw_pixel+0x58>

	case GFX_PIXEL_XOR:
		pixel_value ^= pixel_mask;
     d24:	80 27       	eor	r24, r16

	default:
		break;
	}

	gfx_mono_put_byte(page, x, pixel_value);
     d26:	48 2f       	mov	r20, r24
     d28:	6c 2f       	mov	r22, r28
     d2a:	8f 2d       	mov	r24, r15
     d2c:	e7 de       	rcall	.-562    	; 0xafc <gfx_mono_st7565r_put_byte>
}
     d2e:	df 91       	pop	r29
     d30:	cf 91       	pop	r28
     d32:	1f 91       	pop	r17
     d34:	0f 91       	pop	r16
     d36:	ff 90       	pop	r15
     d38:	08 95       	ret

00000d3a <gfx_mono_st7565r_get_byte>:
\endcode
 */
uint8_t gfx_mono_st7565r_get_byte(gfx_coord_t page, gfx_coord_t column)
{
#ifdef CONFIG_ST7565R_FRAMEBUFFER
	return gfx_mono_framebuffer_get_byte(page, column);
     d3a:	ec c5       	rjmp	.+3032   	; 0x1914 <gfx_mono_framebuffer_get_byte>
	st7565r_set_column_address(column);

	return st7565r_read_data();

#endif
}
     d3c:	08 95       	ret

00000d3e <adc_set_callback>:
 *
 * \param adc Pointer to ADC module.
 * \param callback Pointer to the callback function to set.
 */
void adc_set_callback(ADC_t *adc, adc_callback_t callback)
{
     d3e:	cf 93       	push	r28
     d40:	df 93       	push	r29
     d42:	1f 92       	push	r1
     d44:	cd b7       	in	r28, 0x3d	; 61
     d46:	de b7       	in	r29, 0x3e	; 62

typedef uint8_t irqflags_t;

static inline irqflags_t cpu_irq_save(void)
{
	volatile irqflags_t flags = SREG;
     d48:	2f b7       	in	r18, 0x3f	; 63
     d4a:	29 83       	std	Y+1, r18	; 0x01
	cpu_irq_disable();
     d4c:	f8 94       	cli
	return flags;
     d4e:	49 81       	ldd	r20, Y+1	; 0x01
	Assert(callback);

	flags = cpu_irq_save();

#ifdef ADCA
	if ((uintptr_t)adc == (uintptr_t)&ADCA) {
     d50:	28 2f       	mov	r18, r24
     d52:	39 2f       	mov	r19, r25
     d54:	21 15       	cp	r18, r1
     d56:	82 e0       	ldi	r24, 0x02	; 2
     d58:	38 07       	cpc	r19, r24
     d5a:	29 f4       	brne	.+10     	; 0xd66 <adc_set_callback+0x28>
		adca_callback = callback;
     d5c:	60 93 f4 22 	sts	0x22F4, r22	; 0x8022f4 <adca_callback>
     d60:	70 93 f5 22 	sts	0x22F5, r23	; 0x8022f5 <adca_callback+0x1>
     d64:	07 c0       	rjmp	.+14     	; 0xd74 <adc_set_callback+0x36>
	} else
#endif

#ifdef ADCB
	if ((uintptr_t)adc == (uintptr_t)&ADCB) {
     d66:	20 34       	cpi	r18, 0x40	; 64
     d68:	32 40       	sbci	r19, 0x02	; 2
     d6a:	21 f4       	brne	.+8      	; 0xd74 <adc_set_callback+0x36>
		adcb_callback = callback;
     d6c:	60 93 f2 22 	sts	0x22F2, r22	; 0x8022f2 <adcb_callback>
     d70:	70 93 f3 22 	sts	0x22F3, r23	; 0x8022f3 <adcb_callback+0x1>
}

static inline void cpu_irq_restore(irqflags_t flags)
{
	barrier();
	SREG = flags;
     d74:	4f bf       	out	0x3f, r20	; 63
	{
		Assert(0);
	}

	cpu_irq_restore(flags);
}
     d76:	0f 90       	pop	r0
     d78:	df 91       	pop	r29
     d7a:	cf 91       	pop	r28
     d7c:	08 95       	ret

00000d7e <adc_enable_clock>:
void adc_enable_clock(ADC_t *adc);

void adc_enable_clock(ADC_t *adc)
{
#ifdef ADCA
	if ((uintptr_t)adc == (uintptr_t)(&ADCA)) {
     d7e:	81 15       	cp	r24, r1
     d80:	22 e0       	ldi	r18, 0x02	; 2
     d82:	92 07       	cpc	r25, r18
     d84:	61 f4       	brne	.+24     	; 0xd9e <adc_enable_clock+0x20>
		Assert(adca_enable_count < 0xff);
		if (!adca_enable_count++) {
     d86:	80 91 6f 22 	lds	r24, 0x226F	; 0x80226f <adca_enable_count>
     d8a:	91 e0       	ldi	r25, 0x01	; 1
     d8c:	98 0f       	add	r25, r24
     d8e:	90 93 6f 22 	sts	0x226F, r25	; 0x80226f <adca_enable_count>
     d92:	81 11       	cpse	r24, r1
     d94:	12 c0       	rjmp	.+36     	; 0xdba <adc_enable_clock+0x3c>
			sysclk_enable_module(SYSCLK_PORT_A, SYSCLK_ADC);
     d96:	62 e0       	ldi	r22, 0x02	; 2
     d98:	81 e0       	ldi	r24, 0x01	; 1
     d9a:	46 c6       	rjmp	.+3212   	; 0x1a28 <sysclk_enable_module>
     d9c:	08 95       	ret
		}
	} else
#endif

#ifdef ADCB
	if ((uintptr_t)adc == (uintptr_t)(&ADCB)) {
     d9e:	80 34       	cpi	r24, 0x40	; 64
     da0:	92 40       	sbci	r25, 0x02	; 2
     da2:	59 f4       	brne	.+22     	; 0xdba <adc_enable_clock+0x3c>
		Assert(adcb_enable_count < 0xff);
		if (!adcb_enable_count++) {
     da4:	80 91 6e 22 	lds	r24, 0x226E	; 0x80226e <adcb_enable_count>
     da8:	91 e0       	ldi	r25, 0x01	; 1
     daa:	98 0f       	add	r25, r24
     dac:	90 93 6e 22 	sts	0x226E, r25	; 0x80226e <adcb_enable_count>
     db0:	81 11       	cpse	r24, r1
     db2:	03 c0       	rjmp	.+6      	; 0xdba <adc_enable_clock+0x3c>
			sysclk_enable_module(SYSCLK_PORT_B, SYSCLK_ADC);
     db4:	62 e0       	ldi	r22, 0x02	; 2
     db6:	82 e0       	ldi	r24, 0x02	; 2
     db8:	37 c6       	rjmp	.+3182   	; 0x1a28 <sysclk_enable_module>
     dba:	08 95       	ret

00000dbc <adc_disable_clock>:
void adc_disable_clock(ADC_t *adc);

void adc_disable_clock(ADC_t *adc)
{
#ifdef ADCA
	if ((uintptr_t)adc == (uintptr_t)(&ADCA)) {
     dbc:	81 15       	cp	r24, r1
     dbe:	22 e0       	ldi	r18, 0x02	; 2
     dc0:	92 07       	cpc	r25, r18
     dc2:	59 f4       	brne	.+22     	; 0xdda <adc_disable_clock+0x1e>
		Assert(adca_enable_count);
		if (!--adca_enable_count) {
     dc4:	80 91 6f 22 	lds	r24, 0x226F	; 0x80226f <adca_enable_count>
     dc8:	81 50       	subi	r24, 0x01	; 1
     dca:	80 93 6f 22 	sts	0x226F, r24	; 0x80226f <adca_enable_count>
     dce:	81 11       	cpse	r24, r1
     dd0:	11 c0       	rjmp	.+34     	; 0xdf4 <adc_disable_clock+0x38>
			sysclk_disable_module(SYSCLK_PORT_A, SYSCLK_ADC);
     dd2:	62 e0       	ldi	r22, 0x02	; 2
     dd4:	81 e0       	ldi	r24, 0x01	; 1
     dd6:	3e c6       	rjmp	.+3196   	; 0x1a54 <sysclk_disable_module>
     dd8:	08 95       	ret
		}
	} else
#endif

#ifdef ADCB
	if ((uintptr_t)adc == (uintptr_t)(&ADCB)) {
     dda:	80 34       	cpi	r24, 0x40	; 64
     ddc:	92 40       	sbci	r25, 0x02	; 2
     dde:	51 f4       	brne	.+20     	; 0xdf4 <adc_disable_clock+0x38>
		Assert(adcb_enable_count);
		if (!--adcb_enable_count) {
     de0:	80 91 6e 22 	lds	r24, 0x226E	; 0x80226e <adcb_enable_count>
     de4:	81 50       	subi	r24, 0x01	; 1
     de6:	80 93 6e 22 	sts	0x226E, r24	; 0x80226e <adcb_enable_count>
     dea:	81 11       	cpse	r24, r1
     dec:	03 c0       	rjmp	.+6      	; 0xdf4 <adc_disable_clock+0x38>
			sysclk_disable_module(SYSCLK_PORT_B, SYSCLK_ADC);
     dee:	62 e0       	ldi	r22, 0x02	; 2
     df0:	82 e0       	ldi	r24, 0x02	; 2
     df2:	30 c6       	rjmp	.+3168   	; 0x1a54 <sysclk_disable_module>
     df4:	08 95       	ret

00000df6 <adc_enable>:
 * a conversion. For most XMEGA devices the start-up time is specified
 * to be a maximum of 24 ADC clock cycles. Please verify the start-up time for
 * the device in use.
 */
void adc_enable(ADC_t *adc)
{
     df6:	ef 92       	push	r14
     df8:	ff 92       	push	r15
     dfa:	1f 93       	push	r17
     dfc:	cf 93       	push	r28
     dfe:	df 93       	push	r29
     e00:	1f 92       	push	r1
     e02:	1f 92       	push	r1
     e04:	cd b7       	in	r28, 0x3d	; 61
     e06:	de b7       	in	r29, 0x3e	; 62
     e08:	7c 01       	movw	r14, r24

typedef uint8_t irqflags_t;

static inline irqflags_t cpu_irq_save(void)
{
	volatile irqflags_t flags = SREG;
     e0a:	8f b7       	in	r24, 0x3f	; 63
     e0c:	89 83       	std	Y+1, r24	; 0x01
	cpu_irq_disable();
     e0e:	f8 94       	cli
	return flags;
     e10:	19 81       	ldd	r17, Y+1	; 0x01
	irqflags_t flags = cpu_irq_save();
	adc_enable_clock(adc);
     e12:	c7 01       	movw	r24, r14
     e14:	b4 df       	rcall	.-152    	; 0xd7e <adc_enable_clock>
	adc->CTRLA |= ADC_ENABLE_bm;
     e16:	f7 01       	movw	r30, r14
     e18:	80 81       	ld	r24, Z
     e1a:	81 60       	ori	r24, 0x01	; 1
     e1c:	80 83       	st	Z, r24
}

static inline void cpu_irq_restore(irqflags_t flags)
{
	barrier();
	SREG = flags;
     e1e:	1f bf       	out	0x3f, r17	; 63
static inline void sleepmgr_lock_mode(enum sleepmgr_mode mode)
{
#ifdef CONFIG_SLEEPMGR_ENABLE
	irqflags_t flags;

	if(sleepmgr_locks[mode] >= 0xff) {
     e20:	80 91 f7 22 	lds	r24, 0x22F7	; 0x8022f7 <sleepmgr_locks+0x1>
     e24:	8f 3f       	cpi	r24, 0xFF	; 255
     e26:	09 f4       	brne	.+2      	; 0xe2a <adc_enable+0x34>
     e28:	ff cf       	rjmp	.-2      	; 0xe28 <adc_enable+0x32>

typedef uint8_t irqflags_t;

static inline irqflags_t cpu_irq_save(void)
{
	volatile irqflags_t flags = SREG;
     e2a:	8f b7       	in	r24, 0x3f	; 63
     e2c:	8a 83       	std	Y+2, r24	; 0x02
	cpu_irq_disable();
     e2e:	f8 94       	cli
	return flags;
     e30:	9a 81       	ldd	r25, Y+2	; 0x02
	}

	// Enter a critical section
	flags = cpu_irq_save();

	++sleepmgr_locks[mode];
     e32:	e6 ef       	ldi	r30, 0xF6	; 246
     e34:	f2 e2       	ldi	r31, 0x22	; 34
     e36:	81 81       	ldd	r24, Z+1	; 0x01
     e38:	8f 5f       	subi	r24, 0xFF	; 255
     e3a:	81 83       	std	Z+1, r24	; 0x01
}

static inline void cpu_irq_restore(irqflags_t flags)
{
	barrier();
	SREG = flags;
     e3c:	9f bf       	out	0x3f, r25	; 63
	cpu_irq_restore(flags);

	sleepmgr_lock_mode(SLEEPMGR_IDLE);
}
     e3e:	0f 90       	pop	r0
     e40:	0f 90       	pop	r0
     e42:	df 91       	pop	r29
     e44:	cf 91       	pop	r28
     e46:	1f 91       	pop	r17
     e48:	ff 90       	pop	r15
     e4a:	ef 90       	pop	r14
     e4c:	08 95       	ret

00000e4e <usart_spi_set_baudrate>:
 * \param usart The USART(SPI) module.
 * \param baud The baudrate.
 * \param cpu_hz The CPU frequency.
 */
void usart_spi_set_baudrate(USART_t *usart, uint32_t baud, uint32_t cpu_hz)
{
     e4e:	cf 92       	push	r12
     e50:	df 92       	push	r13
     e52:	ef 92       	push	r14
     e54:	ff 92       	push	r15
     e56:	0f 93       	push	r16
     e58:	1f 93       	push	r17
     e5a:	cf 93       	push	r28
     e5c:	df 93       	push	r29
     e5e:	ec 01       	movw	r28, r24
	uint16_t bsel_value;

	/* Check if baudrate is less than the maximim limit specified in
	 * datasheet */
	if (baud < (cpu_hz / 2)) {
     e60:	d9 01       	movw	r26, r18
     e62:	c8 01       	movw	r24, r16
     e64:	b6 95       	lsr	r27
     e66:	a7 95       	ror	r26
     e68:	97 95       	ror	r25
     e6a:	87 95       	ror	r24
     e6c:	48 17       	cp	r20, r24
     e6e:	59 07       	cpc	r21, r25
     e70:	6a 07       	cpc	r22, r26
     e72:	7b 07       	cpc	r23, r27
     e74:	78 f4       	brcc	.+30     	; 0xe94 <usart_spi_set_baudrate+0x46>
		bsel_value = (cpu_hz / (baud * 2)) - 1;
     e76:	6a 01       	movw	r12, r20
     e78:	7b 01       	movw	r14, r22
     e7a:	cc 0c       	add	r12, r12
     e7c:	dd 1c       	adc	r13, r13
     e7e:	ee 1c       	adc	r14, r14
     e80:	ff 1c       	adc	r15, r15
     e82:	c9 01       	movw	r24, r18
     e84:	b8 01       	movw	r22, r16
     e86:	a7 01       	movw	r20, r14
     e88:	96 01       	movw	r18, r12
     e8a:	0e 94 f1 13 	call	0x27e2	; 0x27e2 <__udivmodsi4>
     e8e:	21 50       	subi	r18, 0x01	; 1
     e90:	31 09       	sbc	r19, r1
     e92:	02 c0       	rjmp	.+4      	; 0xe98 <usart_spi_set_baudrate+0x4a>
	} else {
		/* If baudrate is not within the specfication in datasheet,
		 * assign maximum baudrate possible for the current CPU frequency */
		bsel_value = 0;
     e94:	20 e0       	ldi	r18, 0x00	; 0
     e96:	30 e0       	ldi	r19, 0x00	; 0
	}

	(usart)->BAUDCTRLB = (uint8_t)((~USART_BSCALE_gm) & (bsel_value >> 8));
     e98:	83 2f       	mov	r24, r19
     e9a:	8f 70       	andi	r24, 0x0F	; 15
     e9c:	8f 83       	std	Y+7, r24	; 0x07
	(usart)->BAUDCTRLA = (uint8_t)(bsel_value);
     e9e:	2e 83       	std	Y+6, r18	; 0x06
}
     ea0:	df 91       	pop	r29
     ea2:	cf 91       	pop	r28
     ea4:	1f 91       	pop	r17
     ea6:	0f 91       	pop	r16
     ea8:	ff 90       	pop	r15
     eaa:	ef 90       	pop	r14
     eac:	df 90       	pop	r13
     eae:	cf 90       	pop	r12
     eb0:	08 95       	ret

00000eb2 <usart_init_spi>:
 *
 * \param usart The USART module.
 * \param opt The RS232 configuration option.
 */
void usart_init_spi(USART_t *usart, const usart_spi_options_t *opt)
{
     eb2:	df 92       	push	r13
     eb4:	ef 92       	push	r14
     eb6:	ff 92       	push	r15
     eb8:	0f 93       	push	r16
     eba:	1f 93       	push	r17
     ebc:	cf 93       	push	r28
     ebe:	df 93       	push	r29
     ec0:	1f 92       	push	r1
     ec2:	cd b7       	in	r28, 0x3d	; 61
     ec4:	de b7       	in	r29, 0x3e	; 62
     ec6:	7c 01       	movw	r14, r24
     ec8:	8b 01       	movw	r16, r22
 *
 * \param module Pointer to the module's base address.
 */
static inline void sysclk_enable_peripheral_clock(const volatile void *module)
{
	if (module == NULL) {
     eca:	00 97       	sbiw	r24, 0x00	; 0
     ecc:	09 f4       	brne	.+2      	; 0xed0 <usart_init_spi+0x1e>
     ece:	b2 c1       	rjmp	.+868    	; 0x1234 <__EEPROM_REGION_LENGTH__+0x234>
		Assert(false);
	}
#ifdef AES
	else if (module == &AES) {
     ed0:	80 3c       	cpi	r24, 0xC0	; 192
     ed2:	91 05       	cpc	r25, r1
     ed4:	21 f4       	brne	.+8      	; 0xede <usart_init_spi+0x2c>
		sysclk_enable_module(SYSCLK_PORT_GEN, SYSCLK_AES);
     ed6:	60 e1       	ldi	r22, 0x10	; 16
     ed8:	80 e0       	ldi	r24, 0x00	; 0
     eda:	a6 d5       	rcall	.+2892   	; 0x1a28 <sysclk_enable_module>
     edc:	ab c1       	rjmp	.+854    	; 0x1234 <__EEPROM_REGION_LENGTH__+0x234>
	else if (module == &RTC) {
		sysclk_enable_module(SYSCLK_PORT_GEN, SYSCLK_RTC);
	}
#endif
#ifdef EVSYS
	else if (module == &EVSYS) {
     ede:	80 e8       	ldi	r24, 0x80	; 128
     ee0:	e8 16       	cp	r14, r24
     ee2:	81 e0       	ldi	r24, 0x01	; 1
     ee4:	f8 06       	cpc	r15, r24
     ee6:	21 f4       	brne	.+8      	; 0xef0 <usart_init_spi+0x3e>
		sysclk_enable_module(SYSCLK_PORT_GEN, SYSCLK_EVSYS);
     ee8:	62 e0       	ldi	r22, 0x02	; 2
     eea:	80 e0       	ldi	r24, 0x00	; 0
     eec:	9d d5       	rcall	.+2874   	; 0x1a28 <sysclk_enable_module>
     eee:	a2 c1       	rjmp	.+836    	; 0x1234 <__EEPROM_REGION_LENGTH__+0x234>
	}
#endif
#ifdef DMA
	else if (module == &DMA) {
     ef0:	e1 14       	cp	r14, r1
     ef2:	e1 e0       	ldi	r30, 0x01	; 1
     ef4:	fe 06       	cpc	r15, r30
     ef6:	21 f4       	brne	.+8      	; 0xf00 <usart_init_spi+0x4e>
		sysclk_enable_module(SYSCLK_PORT_GEN, SYSCLK_DMA);
     ef8:	61 e0       	ldi	r22, 0x01	; 1
     efa:	80 e0       	ldi	r24, 0x00	; 0
     efc:	95 d5       	rcall	.+2858   	; 0x1a28 <sysclk_enable_module>
     efe:	9a c1       	rjmp	.+820    	; 0x1234 <__EEPROM_REGION_LENGTH__+0x234>
	else if (module == &EDMA) {
		sysclk_enable_module(SYSCLK_PORT_GEN, SYSCLK_EDMA);
	}
#endif
#ifdef ACA
	else if (module == &ACA) {
     f00:	f0 e8       	ldi	r31, 0x80	; 128
     f02:	ef 16       	cp	r14, r31
     f04:	f3 e0       	ldi	r31, 0x03	; 3
     f06:	ff 06       	cpc	r15, r31
		sysclk_enable_module(SYSCLK_PORT_A, SYSCLK_AC);
     f08:	21 f4       	brne	.+8      	; 0xf12 <usart_init_spi+0x60>
     f0a:	61 e0       	ldi	r22, 0x01	; 1
     f0c:	81 e0       	ldi	r24, 0x01	; 1
     f0e:	8c d5       	rcall	.+2840   	; 0x1a28 <sysclk_enable_module>
     f10:	91 c1       	rjmp	.+802    	; 0x1234 <__EEPROM_REGION_LENGTH__+0x234>
	}
#endif
#ifdef ACB
	else if (module == &ACB) {
     f12:	30 e9       	ldi	r19, 0x90	; 144
     f14:	e3 16       	cp	r14, r19
     f16:	33 e0       	ldi	r19, 0x03	; 3
     f18:	f3 06       	cpc	r15, r19
		sysclk_enable_module(SYSCLK_PORT_B, SYSCLK_AC);
     f1a:	21 f4       	brne	.+8      	; 0xf24 <usart_init_spi+0x72>
     f1c:	61 e0       	ldi	r22, 0x01	; 1
     f1e:	82 e0       	ldi	r24, 0x02	; 2
     f20:	83 d5       	rcall	.+2822   	; 0x1a28 <sysclk_enable_module>
     f22:	88 c1       	rjmp	.+784    	; 0x1234 <__EEPROM_REGION_LENGTH__+0x234>
	}
#endif
#ifdef ADCA
	else if (module == &ADCA) {
     f24:	e1 14       	cp	r14, r1
     f26:	82 e0       	ldi	r24, 0x02	; 2
     f28:	f8 06       	cpc	r15, r24
		sysclk_enable_module(SYSCLK_PORT_A, SYSCLK_ADC);
     f2a:	21 f4       	brne	.+8      	; 0xf34 <usart_init_spi+0x82>
     f2c:	62 e0       	ldi	r22, 0x02	; 2
     f2e:	81 e0       	ldi	r24, 0x01	; 1
     f30:	7b d5       	rcall	.+2806   	; 0x1a28 <sysclk_enable_module>
     f32:	80 c1       	rjmp	.+768    	; 0x1234 <__EEPROM_REGION_LENGTH__+0x234>
	}
#endif
#ifdef ADCB
	else if (module == &ADCB) {
     f34:	e0 e4       	ldi	r30, 0x40	; 64
     f36:	ee 16       	cp	r14, r30
     f38:	e2 e0       	ldi	r30, 0x02	; 2
     f3a:	fe 06       	cpc	r15, r30
		sysclk_enable_module(SYSCLK_PORT_B, SYSCLK_ADC);
     f3c:	21 f4       	brne	.+8      	; 0xf46 <usart_init_spi+0x94>
     f3e:	62 e0       	ldi	r22, 0x02	; 2
     f40:	82 e0       	ldi	r24, 0x02	; 2
     f42:	72 d5       	rcall	.+2788   	; 0x1a28 <sysclk_enable_module>
     f44:	77 c1       	rjmp	.+750    	; 0x1234 <__EEPROM_REGION_LENGTH__+0x234>
	}
#endif
// Workaround for bad XMEGA D header file
#if !XMEGA_D
#ifdef DACB
	else if (module == &DACB) {
     f46:	f0 e2       	ldi	r31, 0x20	; 32
     f48:	ef 16       	cp	r14, r31
     f4a:	f3 e0       	ldi	r31, 0x03	; 3
     f4c:	ff 06       	cpc	r15, r31
		sysclk_enable_module(SYSCLK_PORT_B, SYSCLK_DAC);
     f4e:	21 f4       	brne	.+8      	; 0xf58 <usart_init_spi+0xa6>
     f50:	64 e0       	ldi	r22, 0x04	; 4
     f52:	82 e0       	ldi	r24, 0x02	; 2
     f54:	69 d5       	rcall	.+2770   	; 0x1a28 <sysclk_enable_module>
	}
#endif
#endif // Workaround end
#ifdef TCC0
	else if (module == &TCC0) {
     f56:	6e c1       	rjmp	.+732    	; 0x1234 <__EEPROM_REGION_LENGTH__+0x234>
     f58:	e1 14       	cp	r14, r1
     f5a:	38 e0       	ldi	r19, 0x08	; 8
     f5c:	f3 06       	cpc	r15, r19
		sysclk_enable_module(SYSCLK_PORT_C, SYSCLK_TC0);
     f5e:	21 f4       	brne	.+8      	; 0xf68 <usart_init_spi+0xb6>
     f60:	61 e0       	ldi	r22, 0x01	; 1
     f62:	83 e0       	ldi	r24, 0x03	; 3
     f64:	61 d5       	rcall	.+2754   	; 0x1a28 <sysclk_enable_module>
	}
#endif
#ifdef TCD0
	else if (module == &TCD0) {
     f66:	66 c1       	rjmp	.+716    	; 0x1234 <__EEPROM_REGION_LENGTH__+0x234>
     f68:	e1 14       	cp	r14, r1
     f6a:	89 e0       	ldi	r24, 0x09	; 9
     f6c:	f8 06       	cpc	r15, r24
		sysclk_enable_module(SYSCLK_PORT_D, SYSCLK_TC0);
     f6e:	21 f4       	brne	.+8      	; 0xf78 <usart_init_spi+0xc6>
     f70:	61 e0       	ldi	r22, 0x01	; 1
     f72:	84 e0       	ldi	r24, 0x04	; 4
     f74:	59 d5       	rcall	.+2738   	; 0x1a28 <sysclk_enable_module>
	}
#endif
#ifdef TCE0
	else if (module == &TCE0) {
     f76:	5e c1       	rjmp	.+700    	; 0x1234 <__EEPROM_REGION_LENGTH__+0x234>
     f78:	e1 14       	cp	r14, r1
     f7a:	ea e0       	ldi	r30, 0x0A	; 10
     f7c:	fe 06       	cpc	r15, r30
		sysclk_enable_module(SYSCLK_PORT_E, SYSCLK_TC0);
     f7e:	21 f4       	brne	.+8      	; 0xf88 <usart_init_spi+0xd6>
     f80:	61 e0       	ldi	r22, 0x01	; 1
     f82:	85 e0       	ldi	r24, 0x05	; 5
     f84:	51 d5       	rcall	.+2722   	; 0x1a28 <sysclk_enable_module>
	}
#endif
#ifdef TCF0
	else if (module == &TCF0) {
     f86:	56 c1       	rjmp	.+684    	; 0x1234 <__EEPROM_REGION_LENGTH__+0x234>
     f88:	e1 14       	cp	r14, r1
     f8a:	fb e0       	ldi	r31, 0x0B	; 11
     f8c:	ff 06       	cpc	r15, r31
		sysclk_enable_module(SYSCLK_PORT_F, SYSCLK_TC0);
     f8e:	21 f4       	brne	.+8      	; 0xf98 <usart_init_spi+0xe6>
     f90:	61 e0       	ldi	r22, 0x01	; 1
     f92:	86 e0       	ldi	r24, 0x06	; 6
     f94:	49 d5       	rcall	.+2706   	; 0x1a28 <sysclk_enable_module>
	}
#endif
#ifdef TCC1
	else if (module == &TCC1) {
     f96:	4e c1       	rjmp	.+668    	; 0x1234 <__EEPROM_REGION_LENGTH__+0x234>
     f98:	30 e4       	ldi	r19, 0x40	; 64
     f9a:	e3 16       	cp	r14, r19
     f9c:	38 e0       	ldi	r19, 0x08	; 8
		sysclk_enable_module(SYSCLK_PORT_C, SYSCLK_TC1);
     f9e:	f3 06       	cpc	r15, r19
     fa0:	21 f4       	brne	.+8      	; 0xfaa <usart_init_spi+0xf8>
     fa2:	62 e0       	ldi	r22, 0x02	; 2
     fa4:	83 e0       	ldi	r24, 0x03	; 3
     fa6:	40 d5       	rcall	.+2688   	; 0x1a28 <sysclk_enable_module>
	}
#endif
#ifdef TCD1
	else if (module == &TCD1) {
     fa8:	45 c1       	rjmp	.+650    	; 0x1234 <__EEPROM_REGION_LENGTH__+0x234>
     faa:	80 e4       	ldi	r24, 0x40	; 64
     fac:	e8 16       	cp	r14, r24
     fae:	89 e0       	ldi	r24, 0x09	; 9
		sysclk_enable_module(SYSCLK_PORT_D, SYSCLK_TC1);
     fb0:	f8 06       	cpc	r15, r24
     fb2:	21 f4       	brne	.+8      	; 0xfbc <usart_init_spi+0x10a>
     fb4:	62 e0       	ldi	r22, 0x02	; 2
     fb6:	84 e0       	ldi	r24, 0x04	; 4
     fb8:	37 d5       	rcall	.+2670   	; 0x1a28 <sysclk_enable_module>
	}
#endif
#ifdef TCE1
	else if (module == &TCE1) {
     fba:	3c c1       	rjmp	.+632    	; 0x1234 <__EEPROM_REGION_LENGTH__+0x234>
     fbc:	e0 e4       	ldi	r30, 0x40	; 64
     fbe:	ee 16       	cp	r14, r30
     fc0:	ea e0       	ldi	r30, 0x0A	; 10
		sysclk_enable_module(SYSCLK_PORT_E, SYSCLK_TC1);
     fc2:	fe 06       	cpc	r15, r30
     fc4:	21 f4       	brne	.+8      	; 0xfce <usart_init_spi+0x11c>
     fc6:	62 e0       	ldi	r22, 0x02	; 2
     fc8:	85 e0       	ldi	r24, 0x05	; 5
     fca:	2e d5       	rcall	.+2652   	; 0x1a28 <sysclk_enable_module>
	else if (module == &TCD5) {
		sysclk_enable_module(SYSCLK_PORT_D, SYSCLK_TC5);
	}
#endif
#ifdef HIRESC
	else if (module == &HIRESC) {
     fcc:	33 c1       	rjmp	.+614    	; 0x1234 <__EEPROM_REGION_LENGTH__+0x234>
     fce:	f0 e9       	ldi	r31, 0x90	; 144
     fd0:	ef 16       	cp	r14, r31
     fd2:	f8 e0       	ldi	r31, 0x08	; 8
			sysclk_enable_module(SYSCLK_PORT_C, SYSCLK_HIRES);
     fd4:	ff 06       	cpc	r15, r31
     fd6:	21 f4       	brne	.+8      	; 0xfe0 <usart_init_spi+0x12e>
     fd8:	64 e0       	ldi	r22, 0x04	; 4
     fda:	83 e0       	ldi	r24, 0x03	; 3
     fdc:	25 d5       	rcall	.+2634   	; 0x1a28 <sysclk_enable_module>
	}
#endif
#ifdef HIRESD
	else if (module == &HIRESD) {
     fde:	2a c1       	rjmp	.+596    	; 0x1234 <__EEPROM_REGION_LENGTH__+0x234>
     fe0:	30 e9       	ldi	r19, 0x90	; 144
     fe2:	e3 16       	cp	r14, r19
     fe4:	39 e0       	ldi	r19, 0x09	; 9
		sysclk_enable_module(SYSCLK_PORT_D, SYSCLK_HIRES);
     fe6:	f3 06       	cpc	r15, r19
     fe8:	21 f4       	brne	.+8      	; 0xff2 <usart_init_spi+0x140>
     fea:	64 e0       	ldi	r22, 0x04	; 4
     fec:	84 e0       	ldi	r24, 0x04	; 4
	}
#endif
#ifdef HIRESE
	else if (module == &HIRESE) {
     fee:	1c d5       	rcall	.+2616   	; 0x1a28 <sysclk_enable_module>
     ff0:	21 c1       	rjmp	.+578    	; 0x1234 <__EEPROM_REGION_LENGTH__+0x234>
     ff2:	80 e9       	ldi	r24, 0x90	; 144
     ff4:	e8 16       	cp	r14, r24
     ff6:	8a e0       	ldi	r24, 0x0A	; 10
		sysclk_enable_module(SYSCLK_PORT_E, SYSCLK_HIRES);
     ff8:	f8 06       	cpc	r15, r24
     ffa:	21 f4       	brne	.+8      	; 0x1004 <__EEPROM_REGION_LENGTH__+0x4>
     ffc:	64 e0       	ldi	r22, 0x04	; 4
     ffe:	85 e0       	ldi	r24, 0x05	; 5
	}
#endif
#ifdef HIRESF
	else if (module == &HIRESF) {
    1000:	13 d5       	rcall	.+2598   	; 0x1a28 <sysclk_enable_module>
    1002:	18 c1       	rjmp	.+560    	; 0x1234 <__EEPROM_REGION_LENGTH__+0x234>
    1004:	e0 e9       	ldi	r30, 0x90	; 144
    1006:	ee 16       	cp	r14, r30
    1008:	eb e0       	ldi	r30, 0x0B	; 11
		sysclk_enable_module(SYSCLK_PORT_F, SYSCLK_HIRES);
    100a:	fe 06       	cpc	r15, r30
    100c:	21 f4       	brne	.+8      	; 0x1016 <__EEPROM_REGION_LENGTH__+0x16>
    100e:	64 e0       	ldi	r22, 0x04	; 4
    1010:	86 e0       	ldi	r24, 0x06	; 6
	}
#endif
#ifdef SPIC
	else if (module == &SPIC) {
    1012:	0a d5       	rcall	.+2580   	; 0x1a28 <sysclk_enable_module>
    1014:	0f c1       	rjmp	.+542    	; 0x1234 <__EEPROM_REGION_LENGTH__+0x234>
    1016:	f0 ec       	ldi	r31, 0xC0	; 192
    1018:	ef 16       	cp	r14, r31
    101a:	f8 e0       	ldi	r31, 0x08	; 8
		sysclk_enable_module(SYSCLK_PORT_C, SYSCLK_SPI);
    101c:	ff 06       	cpc	r15, r31
    101e:	21 f4       	brne	.+8      	; 0x1028 <__EEPROM_REGION_LENGTH__+0x28>
    1020:	68 e0       	ldi	r22, 0x08	; 8
    1022:	83 e0       	ldi	r24, 0x03	; 3
	}
#endif
#ifdef SPID
	else if (module == &SPID) {
    1024:	01 d5       	rcall	.+2562   	; 0x1a28 <sysclk_enable_module>
    1026:	06 c1       	rjmp	.+524    	; 0x1234 <__EEPROM_REGION_LENGTH__+0x234>
    1028:	30 ec       	ldi	r19, 0xC0	; 192
    102a:	e3 16       	cp	r14, r19
    102c:	39 e0       	ldi	r19, 0x09	; 9
		sysclk_enable_module(SYSCLK_PORT_D, SYSCLK_SPI);
    102e:	f3 06       	cpc	r15, r19
    1030:	21 f4       	brne	.+8      	; 0x103a <__EEPROM_REGION_LENGTH__+0x3a>
    1032:	68 e0       	ldi	r22, 0x08	; 8
    1034:	84 e0       	ldi	r24, 0x04	; 4
    1036:	f8 d4       	rcall	.+2544   	; 0x1a28 <sysclk_enable_module>
	else if (module == &SPIF) {
		sysclk_enable_module(SYSCLK_PORT_F, SYSCLK_SPI);
	}
#endif
#ifdef USARTC0
	else if (module == &USARTC0) {
    1038:	fd c0       	rjmp	.+506    	; 0x1234 <__EEPROM_REGION_LENGTH__+0x234>
    103a:	80 ea       	ldi	r24, 0xA0	; 160
    103c:	e8 16       	cp	r14, r24
    103e:	88 e0       	ldi	r24, 0x08	; 8
		sysclk_enable_module(SYSCLK_PORT_C, SYSCLK_USART0);
    1040:	f8 06       	cpc	r15, r24
    1042:	61 f4       	brne	.+24     	; 0x105c <__EEPROM_REGION_LENGTH__+0x5c>
    1044:	60 e1       	ldi	r22, 0x10	; 16
    1046:	83 e0       	ldi	r24, 0x03	; 3
 *
 * \param usart Pointer to the USART module.
 */
static inline void usart_rx_disable(USART_t *usart)
{
	(usart)->CTRLB &= ~USART_RXEN_bm;
    1048:	ef d4       	rcall	.+2526   	; 0x1a28 <sysclk_enable_module>
    104a:	e0 ea       	ldi	r30, 0xA0	; 160
    104c:	f8 e0       	ldi	r31, 0x08	; 8
    104e:	84 81       	ldd	r24, Z+4	; 0x04
	sysclk_enable_peripheral_clock(usart);

	usart_rx_disable(usart);

	/* configure Clock polarity using INVEN bit of the correct SCK I/O port **/
	invert_sck = (opt->spimode == 2) || (opt->spimode == 3);
    1050:	8f 7e       	andi	r24, 0xEF	; 239
    1052:	84 83       	std	Z+4, r24	; 0x04
    1054:	f8 01       	movw	r30, r16
    1056:	24 81       	ldd	r18, Z+4	; 0x04
	}
#endif
#ifdef USARTD0
	else if (module == &USARTD0) {
    1058:	22 50       	subi	r18, 0x02	; 2
    105a:	4c c0       	rjmp	.+152    	; 0x10f4 <__EEPROM_REGION_LENGTH__+0xf4>
    105c:	f0 ea       	ldi	r31, 0xA0	; 160
    105e:	ef 16       	cp	r14, r31
		sysclk_enable_module(SYSCLK_PORT_D, SYSCLK_USART0);
    1060:	f9 e0       	ldi	r31, 0x09	; 9
    1062:	ff 06       	cpc	r15, r31
    1064:	21 f4       	brne	.+8      	; 0x106e <__EEPROM_REGION_LENGTH__+0x6e>
    1066:	60 e1       	ldi	r22, 0x10	; 16
    1068:	84 e0       	ldi	r24, 0x04	; 4
	}
#endif
#ifdef USARTE0
	else if (module == &USARTE0) {
    106a:	de d4       	rcall	.+2492   	; 0x1a28 <sysclk_enable_module>
    106c:	e3 c0       	rjmp	.+454    	; 0x1234 <__EEPROM_REGION_LENGTH__+0x234>
    106e:	30 ea       	ldi	r19, 0xA0	; 160
    1070:	e3 16       	cp	r14, r19
		sysclk_enable_module(SYSCLK_PORT_E, SYSCLK_USART0);
    1072:	3a e0       	ldi	r19, 0x0A	; 10
    1074:	f3 06       	cpc	r15, r19
    1076:	21 f4       	brne	.+8      	; 0x1080 <__EEPROM_REGION_LENGTH__+0x80>
    1078:	60 e1       	ldi	r22, 0x10	; 16
    107a:	85 e0       	ldi	r24, 0x05	; 5
	}
#endif
#ifdef USARTF0
	else if (module == &USARTF0) {
    107c:	d5 d4       	rcall	.+2474   	; 0x1a28 <sysclk_enable_module>
    107e:	da c0       	rjmp	.+436    	; 0x1234 <__EEPROM_REGION_LENGTH__+0x234>
    1080:	80 ea       	ldi	r24, 0xA0	; 160
    1082:	e8 16       	cp	r14, r24
		sysclk_enable_module(SYSCLK_PORT_F, SYSCLK_USART0);
    1084:	8b e0       	ldi	r24, 0x0B	; 11
    1086:	f8 06       	cpc	r15, r24
    1088:	21 f4       	brne	.+8      	; 0x1092 <__EEPROM_REGION_LENGTH__+0x92>
    108a:	60 e1       	ldi	r22, 0x10	; 16
    108c:	86 e0       	ldi	r24, 0x06	; 6
	}
#endif
#ifdef USARTC1
	else if (module == &USARTC1) {
    108e:	cc d4       	rcall	.+2456   	; 0x1a28 <sysclk_enable_module>
    1090:	d1 c0       	rjmp	.+418    	; 0x1234 <__EEPROM_REGION_LENGTH__+0x234>
    1092:	e0 eb       	ldi	r30, 0xB0	; 176
    1094:	ee 16       	cp	r14, r30
		sysclk_enable_module(SYSCLK_PORT_C, SYSCLK_USART1);
    1096:	e8 e0       	ldi	r30, 0x08	; 8
    1098:	fe 06       	cpc	r15, r30
    109a:	21 f4       	brne	.+8      	; 0x10a4 <__EEPROM_REGION_LENGTH__+0xa4>
    109c:	60 e2       	ldi	r22, 0x20	; 32
	}
#endif
#ifdef USARTD1
	else if (module == &USARTD1) {
    109e:	83 e0       	ldi	r24, 0x03	; 3
    10a0:	c3 d4       	rcall	.+2438   	; 0x1a28 <sysclk_enable_module>
    10a2:	c8 c0       	rjmp	.+400    	; 0x1234 <__EEPROM_REGION_LENGTH__+0x234>
    10a4:	f0 eb       	ldi	r31, 0xB0	; 176
    10a6:	ef 16       	cp	r14, r31
		sysclk_enable_module(SYSCLK_PORT_D, SYSCLK_USART1);
    10a8:	f9 e0       	ldi	r31, 0x09	; 9
    10aa:	ff 06       	cpc	r15, r31
    10ac:	21 f4       	brne	.+8      	; 0x10b6 <__EEPROM_REGION_LENGTH__+0xb6>
    10ae:	60 e2       	ldi	r22, 0x20	; 32
    10b0:	84 e0       	ldi	r24, 0x04	; 4
	else if (module == &USARTF1) {
		sysclk_enable_module(SYSCLK_PORT_F, SYSCLK_USART1);
	}
#endif
#ifdef TWIC
	else if (module == &TWIC) {
    10b2:	ba d4       	rcall	.+2420   	; 0x1a28 <sysclk_enable_module>
    10b4:	bf c0       	rjmp	.+382    	; 0x1234 <__EEPROM_REGION_LENGTH__+0x234>
    10b6:	30 e8       	ldi	r19, 0x80	; 128
    10b8:	e3 16       	cp	r14, r19
    10ba:	34 e0       	ldi	r19, 0x04	; 4
		sysclk_enable_module(SYSCLK_PORT_C, SYSCLK_TWI);
    10bc:	f3 06       	cpc	r15, r19
    10be:	21 f4       	brne	.+8      	; 0x10c8 <__EEPROM_REGION_LENGTH__+0xc8>
    10c0:	60 e4       	ldi	r22, 0x40	; 64
    10c2:	83 e0       	ldi	r24, 0x03	; 3
    10c4:	b1 d4       	rcall	.+2402   	; 0x1a28 <sysclk_enable_module>
	else if (module == &TWID) {
		sysclk_enable_module(SYSCLK_PORT_D, SYSCLK_TWI);
	}
#endif
#ifdef TWIE
	else if (module == &TWIE) {
    10c6:	b6 c0       	rjmp	.+364    	; 0x1234 <__EEPROM_REGION_LENGTH__+0x234>
    10c8:	80 ea       	ldi	r24, 0xA0	; 160
    10ca:	e8 16       	cp	r14, r24
    10cc:	84 e0       	ldi	r24, 0x04	; 4
    10ce:	f8 06       	cpc	r15, r24
		sysclk_enable_module(SYSCLK_PORT_E, SYSCLK_TWI);
    10d0:	21 f4       	brne	.+8      	; 0x10da <__EEPROM_REGION_LENGTH__+0xda>
    10d2:	60 e4       	ldi	r22, 0x40	; 64
    10d4:	85 e0       	ldi	r24, 0x05	; 5
    10d6:	a8 d4       	rcall	.+2384   	; 0x1a28 <sysclk_enable_module>
    10d8:	ad c0       	rjmp	.+346    	; 0x1234 <__EEPROM_REGION_LENGTH__+0x234>
    10da:	f7 01       	movw	r30, r14
    10dc:	84 81       	ldd	r24, Z+4	; 0x04
    10de:	8f 7e       	andi	r24, 0xEF	; 239
    10e0:	84 83       	std	Z+4, r24	; 0x04
    10e2:	fb 01       	movw	r30, r22
    10e4:	24 81       	ldd	r18, Z+4	; 0x04
    10e6:	22 50       	subi	r18, 0x02	; 2
	UNUSED(invert_sck);

#ifdef USARTC0
	if ((uint16_t)usart == (uint16_t)&USARTC0) {
    10e8:	c7 01       	movw	r24, r14
    10ea:	f0 ea       	ldi	r31, 0xA0	; 160
    10ec:	ef 16       	cp	r14, r31
    10ee:	f8 e0       	ldi	r31, 0x08	; 8
    10f0:	ff 06       	cpc	r15, r31
    10f2:	49 f4       	brne	.+18     	; 0x1106 <__EEPROM_REGION_LENGTH__+0x106>
#  ifdef PORT_USART0_bm
		if (PORTC.REMAP & PORT_USART0_bm) {
    10f4:	80 91 4e 06 	lds	r24, 0x064E	; 0x80064e <__TEXT_REGION_LENGTH__+0x7be64e>
    10f8:	84 fd       	sbrc	r24, 4
    10fa:	a5 c0       	rjmp	.+330    	; 0x1246 <__EEPROM_REGION_LENGTH__+0x246>
			sck_pin = IOPORT_CREATE_PIN(PORTC, 5);
		} else {
			sck_pin = IOPORT_CREATE_PIN(PORTC, 1);
    10fc:	0f 2e       	mov	r0, r31
    10fe:	f1 e1       	ldi	r31, 0x11	; 17
    1100:	df 2e       	mov	r13, r31
    1102:	f0 2d       	mov	r31, r0
    1104:	a4 c0       	rjmp	.+328    	; 0x124e <__EEPROM_REGION_LENGTH__+0x24e>
		sck_pin = IOPORT_CREATE_PIN(PORTC, 1);
#  endif
	}
#endif
#ifdef USARTC1
	if ((uint16_t)usart == (uint16_t)&USARTC1) {
    1106:	80 3b       	cpi	r24, 0xB0	; 176
    1108:	38 e0       	ldi	r19, 0x08	; 8
    110a:	93 07       	cpc	r25, r19
    110c:	91 f0       	breq	.+36     	; 0x1132 <__EEPROM_REGION_LENGTH__+0x132>
		sck_pin = IOPORT_CREATE_PIN(PORTC, 5);
	}
#endif
#ifdef USARTD0
	if ((uint16_t)usart == (uint16_t)&USARTD0) {
    110e:	80 3a       	cpi	r24, 0xA0	; 160
    1110:	e9 e0       	ldi	r30, 0x09	; 9
    1112:	9e 07       	cpc	r25, r30
    1114:	49 f4       	brne	.+18     	; 0x1128 <__EEPROM_REGION_LENGTH__+0x128>
#  ifdef PORT_USART0_bm
		if (PORTD.REMAP & PORT_USART0_bm) {
    1116:	30 91 6e 06 	lds	r19, 0x066E	; 0x80066e <__TEXT_REGION_LENGTH__+0x7be66e>
    111a:	34 fd       	sbrc	r19, 4
    111c:	9b c0       	rjmp	.+310    	; 0x1254 <__EEPROM_REGION_LENGTH__+0x254>
			sck_pin = IOPORT_CREATE_PIN(PORTD, 5);
		} else {
			sck_pin = IOPORT_CREATE_PIN(PORTD, 1);
    111e:	0f 2e       	mov	r0, r31
    1120:	f9 e1       	ldi	r31, 0x19	; 25
    1122:	df 2e       	mov	r13, r31
    1124:	f0 2d       	mov	r31, r0
    1126:	16 c0       	rjmp	.+44     	; 0x1154 <__EEPROM_REGION_LENGTH__+0x154>
		sck_pin = IOPORT_CREATE_PIN(PORTD, 1);
#  endif
	}
#endif
#ifdef USARTD1
	if ((uint16_t)usart == (uint16_t)&USARTD1) {
    1128:	80 3b       	cpi	r24, 0xB0	; 176
    112a:	f9 e0       	ldi	r31, 0x09	; 9
    112c:	9f 07       	cpc	r25, r31
    112e:	f1 f0       	breq	.+60     	; 0x116c <__EEPROM_REGION_LENGTH__+0x16c>
    1130:	04 c0       	rjmp	.+8      	; 0x113a <__EEPROM_REGION_LENGTH__+0x13a>
#  endif
	}
#endif
#ifdef USARTC1
	if ((uint16_t)usart == (uint16_t)&USARTC1) {
		sck_pin = IOPORT_CREATE_PIN(PORTC, 5);
    1132:	0f 2e       	mov	r0, r31
    1134:	f5 e1       	ldi	r31, 0x15	; 21
    1136:	df 2e       	mov	r13, r31
    1138:	f0 2d       	mov	r31, r0
	if ((uint16_t)usart == (uint16_t)&USARTD1) {
		sck_pin = IOPORT_CREATE_PIN(PORTD, 5);
	}
#endif
#ifdef USARTE0
	if ((uint16_t)usart == (uint16_t)&USARTE0) {
    113a:	80 3a       	cpi	r24, 0xA0	; 160
    113c:	3a e0       	ldi	r19, 0x0A	; 10
    113e:	93 07       	cpc	r25, r19
    1140:	49 f4       	brne	.+18     	; 0x1154 <__EEPROM_REGION_LENGTH__+0x154>
#  ifdef PORT_USART0_bm
		if(PORTE.REMAP & PORT_USART0_bm) {
    1142:	80 91 8e 06 	lds	r24, 0x068E	; 0x80068e <__TEXT_REGION_LENGTH__+0x7be68e>
    1146:	84 fd       	sbrc	r24, 4
    1148:	8a c0       	rjmp	.+276    	; 0x125e <__EEPROM_REGION_LENGTH__+0x25e>
			sck_pin = IOPORT_CREATE_PIN(PORTE, 5);
		} else {
			sck_pin = IOPORT_CREATE_PIN(PORTE, 1);
    114a:	0f 2e       	mov	r0, r31
    114c:	f1 e2       	ldi	r31, 0x21	; 33
    114e:	df 2e       	mov	r13, r31
    1150:	f0 2d       	mov	r31, r0
    1152:	15 c0       	rjmp	.+42     	; 0x117e <__EEPROM_REGION_LENGTH__+0x17e>
	if ((uint16_t)usart == (uint16_t)&USARTE1) {
		sck_pin = IOPORT_CREATE_PIN(PORTE, 5);
	}
#endif
#ifdef USARTF0
	if ((uint16_t)usart == (uint16_t)&USARTF0) {
    1154:	80 3a       	cpi	r24, 0xA0	; 160
    1156:	9b 40       	sbci	r25, 0x0B	; 11
    1158:	91 f4       	brne	.+36     	; 0x117e <__EEPROM_REGION_LENGTH__+0x17e>
#  ifdef PORT_USART0_bm
		if(PORTF.REMAP & PORT_USART0_bm) {
    115a:	80 91 ae 06 	lds	r24, 0x06AE	; 0x8006ae <__TEXT_REGION_LENGTH__+0x7be6ae>
    115e:	84 fd       	sbrc	r24, 4
    1160:	0a c0       	rjmp	.+20     	; 0x1176 <__EEPROM_REGION_LENGTH__+0x176>
			sck_pin = IOPORT_CREATE_PIN(PORTF, 5);
		} else {
			sck_pin = IOPORT_CREATE_PIN(PORTF, 1);
    1162:	0f 2e       	mov	r0, r31
    1164:	f9 e2       	ldi	r31, 0x29	; 41
    1166:	df 2e       	mov	r13, r31
    1168:	f0 2d       	mov	r31, r0
    116a:	09 c0       	rjmp	.+18     	; 0x117e <__EEPROM_REGION_LENGTH__+0x17e>
#  endif
	}
#endif
#ifdef USARTD1
	if ((uint16_t)usart == (uint16_t)&USARTD1) {
		sck_pin = IOPORT_CREATE_PIN(PORTD, 5);
    116c:	0f 2e       	mov	r0, r31
    116e:	fd e1       	ldi	r31, 0x1D	; 29
    1170:	df 2e       	mov	r13, r31
    1172:	f0 2d       	mov	r31, r0
    1174:	04 c0       	rjmp	.+8      	; 0x117e <__EEPROM_REGION_LENGTH__+0x17e>
#endif
#ifdef USARTF0
	if ((uint16_t)usart == (uint16_t)&USARTF0) {
#  ifdef PORT_USART0_bm
		if(PORTF.REMAP & PORT_USART0_bm) {
			sck_pin = IOPORT_CREATE_PIN(PORTF, 5);
    1176:	0f 2e       	mov	r0, r31
    1178:	fd e2       	ldi	r31, 0x2D	; 45
    117a:	df 2e       	mov	r13, r31
    117c:	f0 2d       	mov	r31, r0
	return pin >> 3;
}

__always_inline static PORT_t *arch_ioport_port_to_base(ioport_port_t port)
{
	return (PORT_t *)((uintptr_t)IOPORT_BASE_ADDRESS +
    117e:	ed 2d       	mov	r30, r13
    1180:	e6 95       	lsr	r30
    1182:	e6 95       	lsr	r30
    1184:	e6 95       	lsr	r30
    1186:	30 e2       	ldi	r19, 0x20	; 32
    1188:	e3 9f       	mul	r30, r19
    118a:	f0 01       	movw	r30, r0
    118c:	11 24       	eor	r1, r1
    118e:	fa 5f       	subi	r31, 0xFA	; 250
    1190:	3d 2d       	mov	r19, r13
    1192:	37 70       	andi	r19, 0x07	; 7
}

__always_inline static ioport_port_mask_t arch_ioport_pin_to_mask(
		ioport_pin_t pin)
{
	return 1U << (pin & 0x07);
    1194:	81 e0       	ldi	r24, 0x01	; 1
    1196:	90 e0       	ldi	r25, 0x00	; 0
    1198:	03 2e       	mov	r0, r19
    119a:	02 c0       	rjmp	.+4      	; 0x11a0 <__EEPROM_REGION_LENGTH__+0x1a0>
    119c:	88 0f       	add	r24, r24
    119e:	99 1f       	adc	r25, r25
    11a0:	0a 94       	dec	r0
    11a2:	e2 f7       	brpl	.-8      	; 0x119c <__EEPROM_REGION_LENGTH__+0x19c>
		enum ioport_direction dir)
{
	PORT_t *base = arch_ioport_pin_to_base(pin);

	if (dir == IOPORT_DIR_OUTPUT) {
		base->DIRSET = arch_ioport_pin_to_mask(pin);
    11a4:	81 83       	std	Z+1, r24	; 0x01
	}
#endif

	/* Configure the USART output pin */
	ioport_set_pin_dir(sck_pin, IOPORT_DIR_OUTPUT);
	ioport_set_pin_mode(sck_pin,
    11a6:	22 30       	cpi	r18, 0x02	; 2
    11a8:	10 f0       	brcs	.+4      	; 0x11ae <__EEPROM_REGION_LENGTH__+0x1ae>
    11aa:	40 e0       	ldi	r20, 0x00	; 0
    11ac:	01 c0       	rjmp	.+2      	; 0x11b0 <__EEPROM_REGION_LENGTH__+0x1b0>
    11ae:	40 e4       	ldi	r20, 0x40	; 64
__always_inline static void arch_ioport_set_pin_mode(ioport_pin_t pin,
		ioport_mode_t mode)
{
	PORT_t *base = arch_ioport_pin_to_base(pin);
	volatile uint8_t *pin_ctrl
		= (&base->PIN0CTRL + arch_ioport_pin_to_index(pin));
    11b0:	df 01       	movw	r26, r30
    11b2:	50 96       	adiw	r26, 0x10	; 16

__always_inline static void arch_ioport_set_pin_mode(ioport_pin_t pin,
		ioport_mode_t mode)
{
	PORT_t *base = arch_ioport_pin_to_base(pin);
	volatile uint8_t *pin_ctrl
    11b4:	a3 0f       	add	r26, r19
    11b6:	b1 1d       	adc	r27, r1

typedef uint8_t irqflags_t;

static inline irqflags_t cpu_irq_save(void)
{
	volatile irqflags_t flags = SREG;
    11b8:	9f b7       	in	r25, 0x3f	; 63
    11ba:	99 83       	std	Y+1, r25	; 0x01
	cpu_irq_disable();
    11bc:	f8 94       	cli
	return flags;
    11be:	39 81       	ldd	r19, Y+1	; 0x01
		= (&base->PIN0CTRL + arch_ioport_pin_to_index(pin));

	uint8_t flags = cpu_irq_save();

	*pin_ctrl &= PORT_ISC_gm;
    11c0:	2c 91       	ld	r18, X
    11c2:	27 70       	andi	r18, 0x07	; 7
    11c4:	2c 93       	st	X, r18
	*pin_ctrl |= mode;
    11c6:	9c 91       	ld	r25, X
    11c8:	94 2b       	or	r25, r20
    11ca:	9c 93       	st	X, r25
}

static inline void cpu_irq_restore(irqflags_t flags)
{
	barrier();
	SREG = flags;
    11cc:	3f bf       	out	0x3f, r19	; 63
		bool level)
{
	PORT_t *base = arch_ioport_pin_to_base(pin);

	if (level) {
		base->OUTSET = arch_ioport_pin_to_mask(pin);
    11ce:	85 83       	std	Z+5, r24	; 0x05
 * - 0x2        : IrDA mode.
 * - 0x3        : Master SPI mode.
 */
static inline void usart_set_mode(USART_t *usart, USART_CMODE_t usartmode)
{
	(usart)->CTRLC = ((usart)->CTRLC & (~USART_CMODE_gm)) | usartmode;
    11d0:	f7 01       	movw	r30, r14
    11d2:	85 81       	ldd	r24, Z+5	; 0x05
    11d4:	80 6c       	ori	r24, 0xC0	; 192
    11d6:	85 83       	std	Z+5, r24	; 0x05
			IOPORT_MODE_TOTEM | (invert_sck? IOPORT_MODE_INVERT_PIN : 0));
	ioport_set_pin_level(sck_pin, IOPORT_PIN_LEVEL_HIGH);

	usart_set_mode(usart, USART_CMODE_MSPI_gc);

	if (opt->spimode == 1 || opt->spimode == 3) {
    11d8:	f8 01       	movw	r30, r16
    11da:	84 81       	ldd	r24, Z+4	; 0x04
    11dc:	8d 7f       	andi	r24, 0xFD	; 253
    11de:	81 30       	cpi	r24, 0x01	; 1
    11e0:	29 f4       	brne	.+10     	; 0x11ec <__EEPROM_REGION_LENGTH__+0x1ec>
		usart->CTRLC |= USART_UCPHA_bm;
    11e2:	f7 01       	movw	r30, r14
    11e4:	85 81       	ldd	r24, Z+5	; 0x05
    11e6:	82 60       	ori	r24, 0x02	; 2
    11e8:	85 83       	std	Z+5, r24	; 0x05
	} else {
		usart->CTRLC &= ~USART_UCPHA_bm;
    11ea:	04 c0       	rjmp	.+8      	; 0x11f4 <__EEPROM_REGION_LENGTH__+0x1f4>
    11ec:	f7 01       	movw	r30, r14
    11ee:	85 81       	ldd	r24, Z+5	; 0x05
    11f0:	8d 7f       	andi	r24, 0xFD	; 253
	}
	if (opt->data_order) {
    11f2:	85 83       	std	Z+5, r24	; 0x05
    11f4:	f8 01       	movw	r30, r16
    11f6:	85 81       	ldd	r24, Z+5	; 0x05
    11f8:	88 23       	and	r24, r24
		(usart)->CTRLC |= USART_DORD_bm;
    11fa:	29 f0       	breq	.+10     	; 0x1206 <__EEPROM_REGION_LENGTH__+0x206>
    11fc:	f7 01       	movw	r30, r14
    11fe:	85 81       	ldd	r24, Z+5	; 0x05
    1200:	84 60       	ori	r24, 0x04	; 4
    1202:	85 83       	std	Z+5, r24	; 0x05
	} else {
		(usart)->CTRLC &= ~USART_DORD_bm;
    1204:	04 c0       	rjmp	.+8      	; 0x120e <__EEPROM_REGION_LENGTH__+0x20e>
    1206:	f7 01       	movw	r30, r14
    1208:	85 81       	ldd	r24, Z+5	; 0x05
    120a:	8b 7f       	andi	r24, 0xFB	; 251
	}

	usart_spi_set_baudrate(usart, opt->baudrate, sysclk_get_per_hz());
    120c:	85 83       	std	Z+5, r24	; 0x05
    120e:	f8 01       	movw	r30, r16
    1210:	40 81       	ld	r20, Z
    1212:	51 81       	ldd	r21, Z+1	; 0x01
    1214:	62 81       	ldd	r22, Z+2	; 0x02
    1216:	73 81       	ldd	r23, Z+3	; 0x03
    1218:	00 e8       	ldi	r16, 0x80	; 128
    121a:	14 e8       	ldi	r17, 0x84	; 132
    121c:	2e e1       	ldi	r18, 0x1E	; 30
    121e:	30 e0       	ldi	r19, 0x00	; 0
    1220:	c7 01       	movw	r24, r14
    1222:	15 de       	rcall	.-982    	; 0xe4e <usart_spi_set_baudrate>
 *
 * \param usart Pointer to the USART module.
 */
static inline void usart_tx_enable(USART_t *usart)
{
	(usart)->CTRLB |= USART_TXEN_bm;
    1224:	f7 01       	movw	r30, r14
    1226:	84 81       	ldd	r24, Z+4	; 0x04
    1228:	88 60       	ori	r24, 0x08	; 8
    122a:	84 83       	std	Z+4, r24	; 0x04
 *
 * \param usart Pointer to the USART module
 */
static inline void usart_rx_enable(USART_t *usart)
{
	(usart)->CTRLB |= USART_RXEN_bm;
    122c:	84 81       	ldd	r24, Z+4	; 0x04
    122e:	80 61       	ori	r24, 0x10	; 16
    1230:	84 83       	std	Z+4, r24	; 0x04
	usart_tx_enable(usart);
	usart_rx_enable(usart);
}
    1232:	1a c0       	rjmp	.+52     	; 0x1268 <__EEPROM_REGION_LENGTH__+0x268>
 *
 * \param usart Pointer to the USART module.
 */
static inline void usart_rx_disable(USART_t *usart)
{
	(usart)->CTRLB &= ~USART_RXEN_bm;
    1234:	f7 01       	movw	r30, r14
    1236:	84 81       	ldd	r24, Z+4	; 0x04
    1238:	8f 7e       	andi	r24, 0xEF	; 239
    123a:	84 83       	std	Z+4, r24	; 0x04
	sysclk_enable_peripheral_clock(usart);

	usart_rx_disable(usart);

	/* configure Clock polarity using INVEN bit of the correct SCK I/O port **/
	invert_sck = (opt->spimode == 2) || (opt->spimode == 3);
    123c:	f8 01       	movw	r30, r16
    123e:	24 81       	ldd	r18, Z+4	; 0x04
    1240:	22 50       	subi	r18, 0x02	; 2
	UNUSED(invert_sck);

#ifdef USARTC0
	if ((uint16_t)usart == (uint16_t)&USARTC0) {
    1242:	c7 01       	movw	r24, r14
    1244:	60 cf       	rjmp	.-320    	; 0x1106 <__EEPROM_REGION_LENGTH__+0x106>
#  ifdef PORT_USART0_bm
		if (PORTC.REMAP & PORT_USART0_bm) {
			sck_pin = IOPORT_CREATE_PIN(PORTC, 5);
    1246:	0f 2e       	mov	r0, r31
    1248:	f5 e1       	ldi	r31, 0x15	; 21
    124a:	df 2e       	mov	r13, r31
    124c:	f0 2d       	mov	r31, r0
 *
 * \param usart The USART module.
 * \param opt The RS232 configuration option.
 */
void usart_init_spi(USART_t *usart, const usart_spi_options_t *opt)
{
    124e:	80 ea       	ldi	r24, 0xA0	; 160
    1250:	98 e0       	ldi	r25, 0x08	; 8
    1252:	6a cf       	rjmp	.-300    	; 0x1128 <__EEPROM_REGION_LENGTH__+0x128>
#endif
#ifdef USARTD0
	if ((uint16_t)usart == (uint16_t)&USARTD0) {
#  ifdef PORT_USART0_bm
		if (PORTD.REMAP & PORT_USART0_bm) {
			sck_pin = IOPORT_CREATE_PIN(PORTD, 5);
    1254:	0f 2e       	mov	r0, r31
    1256:	fd e1       	ldi	r31, 0x1D	; 29
    1258:	df 2e       	mov	r13, r31
    125a:	f0 2d       	mov	r31, r0
    125c:	7b cf       	rjmp	.-266    	; 0x1154 <__EEPROM_REGION_LENGTH__+0x154>
#endif
#ifdef USARTE0
	if ((uint16_t)usart == (uint16_t)&USARTE0) {
#  ifdef PORT_USART0_bm
		if(PORTE.REMAP & PORT_USART0_bm) {
			sck_pin = IOPORT_CREATE_PIN(PORTE, 5);
    125e:	0f 2e       	mov	r0, r31
    1260:	f5 e2       	ldi	r31, 0x25	; 37
    1262:	df 2e       	mov	r13, r31
    1264:	f0 2d       	mov	r31, r0
    1266:	8b cf       	rjmp	.-234    	; 0x117e <__EEPROM_REGION_LENGTH__+0x17e>
	}

	usart_spi_set_baudrate(usart, opt->baudrate, sysclk_get_per_hz());
	usart_tx_enable(usart);
	usart_rx_enable(usart);
}
    1268:	0f 90       	pop	r0
    126a:	df 91       	pop	r29
    126c:	cf 91       	pop	r28
    126e:	1f 91       	pop	r17
    1270:	0f 91       	pop	r16
    1272:	ff 90       	pop	r15
    1274:	ef 90       	pop	r14
    1276:	df 90       	pop	r13
    1278:	08 95       	ret

0000127a <__vector_71>:
 *
 * Calls the callback function that has been set for the ADC when the channel's
 * interrupt flag is set, if its interrupt has been enabled.
 */
ISR(ADCA_CH0_vect)
{
    127a:	1f 92       	push	r1
    127c:	0f 92       	push	r0
    127e:	0f b6       	in	r0, 0x3f	; 63
    1280:	0f 92       	push	r0
    1282:	11 24       	eor	r1, r1
    1284:	0b b6       	in	r0, 0x3b	; 59
    1286:	0f 92       	push	r0
    1288:	2f 93       	push	r18
    128a:	3f 93       	push	r19
    128c:	4f 93       	push	r20
    128e:	5f 93       	push	r21
    1290:	6f 93       	push	r22
    1292:	7f 93       	push	r23
    1294:	8f 93       	push	r24
    1296:	9f 93       	push	r25
    1298:	af 93       	push	r26
    129a:	bf 93       	push	r27
    129c:	ef 93       	push	r30
    129e:	ff 93       	push	r31
	adca_callback(&ADCA, ADC_CH0, adc_get_result(&ADCA, ADC_CH0));
    12a0:	40 91 24 02 	lds	r20, 0x0224	; 0x800224 <__TEXT_REGION_LENGTH__+0x7be224>
    12a4:	50 91 25 02 	lds	r21, 0x0225	; 0x800225 <__TEXT_REGION_LENGTH__+0x7be225>
    12a8:	e0 91 f4 22 	lds	r30, 0x22F4	; 0x8022f4 <adca_callback>
    12ac:	f0 91 f5 22 	lds	r31, 0x22F5	; 0x8022f5 <adca_callback+0x1>
    12b0:	61 e0       	ldi	r22, 0x01	; 1
    12b2:	80 e0       	ldi	r24, 0x00	; 0
    12b4:	92 e0       	ldi	r25, 0x02	; 2
    12b6:	19 95       	eicall
}
    12b8:	ff 91       	pop	r31
    12ba:	ef 91       	pop	r30
    12bc:	bf 91       	pop	r27
    12be:	af 91       	pop	r26
    12c0:	9f 91       	pop	r25
    12c2:	8f 91       	pop	r24
    12c4:	7f 91       	pop	r23
    12c6:	6f 91       	pop	r22
    12c8:	5f 91       	pop	r21
    12ca:	4f 91       	pop	r20
    12cc:	3f 91       	pop	r19
    12ce:	2f 91       	pop	r18
    12d0:	0f 90       	pop	r0
    12d2:	0b be       	out	0x3b, r0	; 59
    12d4:	0f 90       	pop	r0
    12d6:	0f be       	out	0x3f, r0	; 63
    12d8:	0f 90       	pop	r0
    12da:	1f 90       	pop	r1
    12dc:	18 95       	reti

000012de <__vector_72>:
 *
 * Calls the callback function that has been set for the ADC when the channel's
 * interrupt flag is set, if its interrupt has been enabled.
 */
ISR(ADCA_CH1_vect)
{
    12de:	1f 92       	push	r1
    12e0:	0f 92       	push	r0
    12e2:	0f b6       	in	r0, 0x3f	; 63
    12e4:	0f 92       	push	r0
    12e6:	11 24       	eor	r1, r1
    12e8:	0b b6       	in	r0, 0x3b	; 59
    12ea:	0f 92       	push	r0
    12ec:	2f 93       	push	r18
    12ee:	3f 93       	push	r19
    12f0:	4f 93       	push	r20
    12f2:	5f 93       	push	r21
    12f4:	6f 93       	push	r22
    12f6:	7f 93       	push	r23
    12f8:	8f 93       	push	r24
    12fa:	9f 93       	push	r25
    12fc:	af 93       	push	r26
    12fe:	bf 93       	push	r27
    1300:	ef 93       	push	r30
    1302:	ff 93       	push	r31
	adca_callback(&ADCA, ADC_CH1, adc_get_result(&ADCA, ADC_CH1));
    1304:	40 91 2c 02 	lds	r20, 0x022C	; 0x80022c <__TEXT_REGION_LENGTH__+0x7be22c>
    1308:	50 91 2d 02 	lds	r21, 0x022D	; 0x80022d <__TEXT_REGION_LENGTH__+0x7be22d>
    130c:	e0 91 f4 22 	lds	r30, 0x22F4	; 0x8022f4 <adca_callback>
    1310:	f0 91 f5 22 	lds	r31, 0x22F5	; 0x8022f5 <adca_callback+0x1>
    1314:	62 e0       	ldi	r22, 0x02	; 2
    1316:	80 e0       	ldi	r24, 0x00	; 0
    1318:	92 e0       	ldi	r25, 0x02	; 2
    131a:	19 95       	eicall
}
    131c:	ff 91       	pop	r31
    131e:	ef 91       	pop	r30
    1320:	bf 91       	pop	r27
    1322:	af 91       	pop	r26
    1324:	9f 91       	pop	r25
    1326:	8f 91       	pop	r24
    1328:	7f 91       	pop	r23
    132a:	6f 91       	pop	r22
    132c:	5f 91       	pop	r21
    132e:	4f 91       	pop	r20
    1330:	3f 91       	pop	r19
    1332:	2f 91       	pop	r18
    1334:	0f 90       	pop	r0
    1336:	0b be       	out	0x3b, r0	; 59
    1338:	0f 90       	pop	r0
    133a:	0f be       	out	0x3f, r0	; 63
    133c:	0f 90       	pop	r0
    133e:	1f 90       	pop	r1
    1340:	18 95       	reti

00001342 <__vector_73>:
 *
 * Calls the callback function that has been set for the ADC when the channel's
 * interrupt flag is set, if its interrupt has been enabled.
 */
ISR(ADCA_CH2_vect)
{
    1342:	1f 92       	push	r1
    1344:	0f 92       	push	r0
    1346:	0f b6       	in	r0, 0x3f	; 63
    1348:	0f 92       	push	r0
    134a:	11 24       	eor	r1, r1
    134c:	0b b6       	in	r0, 0x3b	; 59
    134e:	0f 92       	push	r0
    1350:	2f 93       	push	r18
    1352:	3f 93       	push	r19
    1354:	4f 93       	push	r20
    1356:	5f 93       	push	r21
    1358:	6f 93       	push	r22
    135a:	7f 93       	push	r23
    135c:	8f 93       	push	r24
    135e:	9f 93       	push	r25
    1360:	af 93       	push	r26
    1362:	bf 93       	push	r27
    1364:	ef 93       	push	r30
    1366:	ff 93       	push	r31
	adca_callback(&ADCA, ADC_CH2, adc_get_result(&ADCA, ADC_CH2));
    1368:	40 91 34 02 	lds	r20, 0x0234	; 0x800234 <__TEXT_REGION_LENGTH__+0x7be234>
    136c:	50 91 35 02 	lds	r21, 0x0235	; 0x800235 <__TEXT_REGION_LENGTH__+0x7be235>
    1370:	e0 91 f4 22 	lds	r30, 0x22F4	; 0x8022f4 <adca_callback>
    1374:	f0 91 f5 22 	lds	r31, 0x22F5	; 0x8022f5 <adca_callback+0x1>
    1378:	64 e0       	ldi	r22, 0x04	; 4
    137a:	80 e0       	ldi	r24, 0x00	; 0
    137c:	92 e0       	ldi	r25, 0x02	; 2
    137e:	19 95       	eicall
}
    1380:	ff 91       	pop	r31
    1382:	ef 91       	pop	r30
    1384:	bf 91       	pop	r27
    1386:	af 91       	pop	r26
    1388:	9f 91       	pop	r25
    138a:	8f 91       	pop	r24
    138c:	7f 91       	pop	r23
    138e:	6f 91       	pop	r22
    1390:	5f 91       	pop	r21
    1392:	4f 91       	pop	r20
    1394:	3f 91       	pop	r19
    1396:	2f 91       	pop	r18
    1398:	0f 90       	pop	r0
    139a:	0b be       	out	0x3b, r0	; 59
    139c:	0f 90       	pop	r0
    139e:	0f be       	out	0x3f, r0	; 63
    13a0:	0f 90       	pop	r0
    13a2:	1f 90       	pop	r1
    13a4:	18 95       	reti

000013a6 <__vector_74>:
 *
 * Calls the callback function that has been set for the ADC when the channel's
 * interrupt flag is set, if its interrupt has been enabled.
 */
ISR(ADCA_CH3_vect)
{
    13a6:	1f 92       	push	r1
    13a8:	0f 92       	push	r0
    13aa:	0f b6       	in	r0, 0x3f	; 63
    13ac:	0f 92       	push	r0
    13ae:	11 24       	eor	r1, r1
    13b0:	0b b6       	in	r0, 0x3b	; 59
    13b2:	0f 92       	push	r0
    13b4:	2f 93       	push	r18
    13b6:	3f 93       	push	r19
    13b8:	4f 93       	push	r20
    13ba:	5f 93       	push	r21
    13bc:	6f 93       	push	r22
    13be:	7f 93       	push	r23
    13c0:	8f 93       	push	r24
    13c2:	9f 93       	push	r25
    13c4:	af 93       	push	r26
    13c6:	bf 93       	push	r27
    13c8:	ef 93       	push	r30
    13ca:	ff 93       	push	r31
	adca_callback(&ADCA, ADC_CH3, adc_get_result(&ADCA, ADC_CH3));
    13cc:	40 91 3c 02 	lds	r20, 0x023C	; 0x80023c <__TEXT_REGION_LENGTH__+0x7be23c>
    13d0:	50 91 3d 02 	lds	r21, 0x023D	; 0x80023d <__TEXT_REGION_LENGTH__+0x7be23d>
    13d4:	e0 91 f4 22 	lds	r30, 0x22F4	; 0x8022f4 <adca_callback>
    13d8:	f0 91 f5 22 	lds	r31, 0x22F5	; 0x8022f5 <adca_callback+0x1>
    13dc:	68 e0       	ldi	r22, 0x08	; 8
    13de:	80 e0       	ldi	r24, 0x00	; 0
    13e0:	92 e0       	ldi	r25, 0x02	; 2
    13e2:	19 95       	eicall
}
    13e4:	ff 91       	pop	r31
    13e6:	ef 91       	pop	r30
    13e8:	bf 91       	pop	r27
    13ea:	af 91       	pop	r26
    13ec:	9f 91       	pop	r25
    13ee:	8f 91       	pop	r24
    13f0:	7f 91       	pop	r23
    13f2:	6f 91       	pop	r22
    13f4:	5f 91       	pop	r21
    13f6:	4f 91       	pop	r20
    13f8:	3f 91       	pop	r19
    13fa:	2f 91       	pop	r18
    13fc:	0f 90       	pop	r0
    13fe:	0b be       	out	0x3b, r0	; 59
    1400:	0f 90       	pop	r0
    1402:	0f be       	out	0x3f, r0	; 63
    1404:	0f 90       	pop	r0
    1406:	1f 90       	pop	r1
    1408:	18 95       	reti

0000140a <__vector_39>:
 *
 * Calls the callback function that has been set for the ADC when the channel's
 * interrupt flag is set, if its interrupt has been enabled.
 */
ISR(ADCB_CH0_vect)
{
    140a:	1f 92       	push	r1
    140c:	0f 92       	push	r0
    140e:	0f b6       	in	r0, 0x3f	; 63
    1410:	0f 92       	push	r0
    1412:	11 24       	eor	r1, r1
    1414:	0b b6       	in	r0, 0x3b	; 59
    1416:	0f 92       	push	r0
    1418:	2f 93       	push	r18
    141a:	3f 93       	push	r19
    141c:	4f 93       	push	r20
    141e:	5f 93       	push	r21
    1420:	6f 93       	push	r22
    1422:	7f 93       	push	r23
    1424:	8f 93       	push	r24
    1426:	9f 93       	push	r25
    1428:	af 93       	push	r26
    142a:	bf 93       	push	r27
    142c:	ef 93       	push	r30
    142e:	ff 93       	push	r31
	adcb_callback(&ADCB, ADC_CH0, adc_get_result(&ADCB, ADC_CH0));
    1430:	40 91 64 02 	lds	r20, 0x0264	; 0x800264 <__TEXT_REGION_LENGTH__+0x7be264>
    1434:	50 91 65 02 	lds	r21, 0x0265	; 0x800265 <__TEXT_REGION_LENGTH__+0x7be265>
    1438:	e0 91 f2 22 	lds	r30, 0x22F2	; 0x8022f2 <adcb_callback>
    143c:	f0 91 f3 22 	lds	r31, 0x22F3	; 0x8022f3 <adcb_callback+0x1>
    1440:	61 e0       	ldi	r22, 0x01	; 1
    1442:	80 e4       	ldi	r24, 0x40	; 64
    1444:	92 e0       	ldi	r25, 0x02	; 2
    1446:	19 95       	eicall
}
    1448:	ff 91       	pop	r31
    144a:	ef 91       	pop	r30
    144c:	bf 91       	pop	r27
    144e:	af 91       	pop	r26
    1450:	9f 91       	pop	r25
    1452:	8f 91       	pop	r24
    1454:	7f 91       	pop	r23
    1456:	6f 91       	pop	r22
    1458:	5f 91       	pop	r21
    145a:	4f 91       	pop	r20
    145c:	3f 91       	pop	r19
    145e:	2f 91       	pop	r18
    1460:	0f 90       	pop	r0
    1462:	0b be       	out	0x3b, r0	; 59
    1464:	0f 90       	pop	r0
    1466:	0f be       	out	0x3f, r0	; 63
    1468:	0f 90       	pop	r0
    146a:	1f 90       	pop	r1
    146c:	18 95       	reti

0000146e <__vector_40>:
 *
 * Calls the callback function that has been set for the ADC when the channel's
 * interrupt flag is set, if its interrupt has been enabled.
 */
ISR(ADCB_CH1_vect)
{
    146e:	1f 92       	push	r1
    1470:	0f 92       	push	r0
    1472:	0f b6       	in	r0, 0x3f	; 63
    1474:	0f 92       	push	r0
    1476:	11 24       	eor	r1, r1
    1478:	0b b6       	in	r0, 0x3b	; 59
    147a:	0f 92       	push	r0
    147c:	2f 93       	push	r18
    147e:	3f 93       	push	r19
    1480:	4f 93       	push	r20
    1482:	5f 93       	push	r21
    1484:	6f 93       	push	r22
    1486:	7f 93       	push	r23
    1488:	8f 93       	push	r24
    148a:	9f 93       	push	r25
    148c:	af 93       	push	r26
    148e:	bf 93       	push	r27
    1490:	ef 93       	push	r30
    1492:	ff 93       	push	r31
	adcb_callback(&ADCB, ADC_CH1, adc_get_result(&ADCB, ADC_CH1));
    1494:	40 91 6c 02 	lds	r20, 0x026C	; 0x80026c <__TEXT_REGION_LENGTH__+0x7be26c>
    1498:	50 91 6d 02 	lds	r21, 0x026D	; 0x80026d <__TEXT_REGION_LENGTH__+0x7be26d>
    149c:	e0 91 f2 22 	lds	r30, 0x22F2	; 0x8022f2 <adcb_callback>
    14a0:	f0 91 f3 22 	lds	r31, 0x22F3	; 0x8022f3 <adcb_callback+0x1>
    14a4:	62 e0       	ldi	r22, 0x02	; 2
    14a6:	80 e4       	ldi	r24, 0x40	; 64
    14a8:	92 e0       	ldi	r25, 0x02	; 2
    14aa:	19 95       	eicall
}
    14ac:	ff 91       	pop	r31
    14ae:	ef 91       	pop	r30
    14b0:	bf 91       	pop	r27
    14b2:	af 91       	pop	r26
    14b4:	9f 91       	pop	r25
    14b6:	8f 91       	pop	r24
    14b8:	7f 91       	pop	r23
    14ba:	6f 91       	pop	r22
    14bc:	5f 91       	pop	r21
    14be:	4f 91       	pop	r20
    14c0:	3f 91       	pop	r19
    14c2:	2f 91       	pop	r18
    14c4:	0f 90       	pop	r0
    14c6:	0b be       	out	0x3b, r0	; 59
    14c8:	0f 90       	pop	r0
    14ca:	0f be       	out	0x3f, r0	; 63
    14cc:	0f 90       	pop	r0
    14ce:	1f 90       	pop	r1
    14d0:	18 95       	reti

000014d2 <__vector_41>:
 *
 * Calls the callback function that has been set for the ADC when the channel's
 * interrupt flag is set, if its interrupt has been enabled.
 */
ISR(ADCB_CH2_vect)
{
    14d2:	1f 92       	push	r1
    14d4:	0f 92       	push	r0
    14d6:	0f b6       	in	r0, 0x3f	; 63
    14d8:	0f 92       	push	r0
    14da:	11 24       	eor	r1, r1
    14dc:	0b b6       	in	r0, 0x3b	; 59
    14de:	0f 92       	push	r0
    14e0:	2f 93       	push	r18
    14e2:	3f 93       	push	r19
    14e4:	4f 93       	push	r20
    14e6:	5f 93       	push	r21
    14e8:	6f 93       	push	r22
    14ea:	7f 93       	push	r23
    14ec:	8f 93       	push	r24
    14ee:	9f 93       	push	r25
    14f0:	af 93       	push	r26
    14f2:	bf 93       	push	r27
    14f4:	ef 93       	push	r30
    14f6:	ff 93       	push	r31
	adcb_callback(&ADCB, ADC_CH2, adc_get_result(&ADCB, ADC_CH2));
    14f8:	40 91 74 02 	lds	r20, 0x0274	; 0x800274 <__TEXT_REGION_LENGTH__+0x7be274>
    14fc:	50 91 75 02 	lds	r21, 0x0275	; 0x800275 <__TEXT_REGION_LENGTH__+0x7be275>
    1500:	e0 91 f2 22 	lds	r30, 0x22F2	; 0x8022f2 <adcb_callback>
    1504:	f0 91 f3 22 	lds	r31, 0x22F3	; 0x8022f3 <adcb_callback+0x1>
    1508:	64 e0       	ldi	r22, 0x04	; 4
    150a:	80 e4       	ldi	r24, 0x40	; 64
    150c:	92 e0       	ldi	r25, 0x02	; 2
    150e:	19 95       	eicall
}
    1510:	ff 91       	pop	r31
    1512:	ef 91       	pop	r30
    1514:	bf 91       	pop	r27
    1516:	af 91       	pop	r26
    1518:	9f 91       	pop	r25
    151a:	8f 91       	pop	r24
    151c:	7f 91       	pop	r23
    151e:	6f 91       	pop	r22
    1520:	5f 91       	pop	r21
    1522:	4f 91       	pop	r20
    1524:	3f 91       	pop	r19
    1526:	2f 91       	pop	r18
    1528:	0f 90       	pop	r0
    152a:	0b be       	out	0x3b, r0	; 59
    152c:	0f 90       	pop	r0
    152e:	0f be       	out	0x3f, r0	; 63
    1530:	0f 90       	pop	r0
    1532:	1f 90       	pop	r1
    1534:	18 95       	reti

00001536 <__vector_42>:
 *
 * Calls the callback function that has been set for the ADC when the channel's
 * interrupt flag is set, if its interrupt has been enabled.
 */
ISR(ADCB_CH3_vect)
{
    1536:	1f 92       	push	r1
    1538:	0f 92       	push	r0
    153a:	0f b6       	in	r0, 0x3f	; 63
    153c:	0f 92       	push	r0
    153e:	11 24       	eor	r1, r1
    1540:	0b b6       	in	r0, 0x3b	; 59
    1542:	0f 92       	push	r0
    1544:	2f 93       	push	r18
    1546:	3f 93       	push	r19
    1548:	4f 93       	push	r20
    154a:	5f 93       	push	r21
    154c:	6f 93       	push	r22
    154e:	7f 93       	push	r23
    1550:	8f 93       	push	r24
    1552:	9f 93       	push	r25
    1554:	af 93       	push	r26
    1556:	bf 93       	push	r27
    1558:	ef 93       	push	r30
    155a:	ff 93       	push	r31
	adcb_callback(&ADCB, ADC_CH3, adc_get_result(&ADCB, ADC_CH3));
    155c:	40 91 7c 02 	lds	r20, 0x027C	; 0x80027c <__TEXT_REGION_LENGTH__+0x7be27c>
    1560:	50 91 7d 02 	lds	r21, 0x027D	; 0x80027d <__TEXT_REGION_LENGTH__+0x7be27d>
    1564:	e0 91 f2 22 	lds	r30, 0x22F2	; 0x8022f2 <adcb_callback>
    1568:	f0 91 f3 22 	lds	r31, 0x22F3	; 0x8022f3 <adcb_callback+0x1>
    156c:	68 e0       	ldi	r22, 0x08	; 8
    156e:	80 e4       	ldi	r24, 0x40	; 64
    1570:	92 e0       	ldi	r25, 0x02	; 2
    1572:	19 95       	eicall
}
    1574:	ff 91       	pop	r31
    1576:	ef 91       	pop	r30
    1578:	bf 91       	pop	r27
    157a:	af 91       	pop	r26
    157c:	9f 91       	pop	r25
    157e:	8f 91       	pop	r24
    1580:	7f 91       	pop	r23
    1582:	6f 91       	pop	r22
    1584:	5f 91       	pop	r21
    1586:	4f 91       	pop	r20
    1588:	3f 91       	pop	r19
    158a:	2f 91       	pop	r18
    158c:	0f 90       	pop	r0
    158e:	0b be       	out	0x3b, r0	; 59
    1590:	0f 90       	pop	r0
    1592:	0f be       	out	0x3f, r0	; 63
    1594:	0f 90       	pop	r0
    1596:	1f 90       	pop	r1
    1598:	18 95       	reti

0000159a <adc_write_configuration>:
 *
 * \param adc Pointer to ADC module.
 * \param conf Pointer to ADC module configuration.
 */
void adc_write_configuration(ADC_t *adc, const struct adc_config *conf)
{
    159a:	bf 92       	push	r11
    159c:	cf 92       	push	r12
    159e:	df 92       	push	r13
    15a0:	ef 92       	push	r14
    15a2:	ff 92       	push	r15
    15a4:	0f 93       	push	r16
    15a6:	1f 93       	push	r17
    15a8:	cf 93       	push	r28
    15aa:	df 93       	push	r29
    15ac:	1f 92       	push	r1
    15ae:	cd b7       	in	r28, 0x3d	; 61
    15b0:	de b7       	in	r29, 0x3e	; 62
    15b2:	8c 01       	movw	r16, r24
    15b4:	7b 01       	movw	r14, r22
	uint16_t cal;
	uint8_t enable;
	irqflags_t flags;

#ifdef ADCA
	if ((uintptr_t)adc == (uintptr_t)&ADCA) {
    15b6:	81 15       	cp	r24, r1
    15b8:	22 e0       	ldi	r18, 0x02	; 2
    15ba:	92 07       	cpc	r25, r18
    15bc:	71 f4       	brne	.+28     	; 0x15da <adc_write_configuration+0x40>
 *
 * \param address Byte offset into the signature row
 */
static inline uint8_t nvm_read_production_signature_row(uint8_t address)
{
	return nvm_read_byte(NVM_CMD_READ_CALIB_ROW_gc, address);
    15be:	61 e2       	ldi	r22, 0x21	; 33
    15c0:	70 e0       	ldi	r23, 0x00	; 0
    15c2:	82 e0       	ldi	r24, 0x02	; 2
    15c4:	5c d2       	rcall	.+1208   	; 0x1a7e <nvm_read_byte>
	uint16_t data;

	switch (cal) {
#ifdef ADCA
	case ADC_CAL_ADCA:
		data = nvm_read_production_signature_row(ADCACAL1);
    15c6:	c8 2e       	mov	r12, r24
    15c8:	d1 2c       	mov	r13, r1
    15ca:	60 e2       	ldi	r22, 0x20	; 32
    15cc:	70 e0       	ldi	r23, 0x00	; 0
    15ce:	82 e0       	ldi	r24, 0x02	; 2
    15d0:	56 d2       	rcall	.+1196   	; 0x1a7e <nvm_read_byte>
		data <<= 8;
		data |= nvm_read_production_signature_row(ADCACAL0);
    15d2:	dc 2c       	mov	r13, r12
    15d4:	cc 24       	eor	r12, r12
    15d6:	c8 2a       	or	r12, r24
    15d8:	10 c0       	rjmp	.+32     	; 0x15fa <adc_write_configuration+0x60>
		cal = adc_get_calibration_data(ADC_CAL_ADCA);
	} else
#endif

#ifdef ADCB
	if ((uintptr_t)adc == (uintptr_t)&ADCB) {
    15da:	80 34       	cpi	r24, 0x40	; 64
    15dc:	92 40       	sbci	r25, 0x02	; 2
    15de:	c1 f5       	brne	.+112    	; 0x1650 <adc_write_configuration+0xb6>
    15e0:	65 e2       	ldi	r22, 0x25	; 37
    15e2:	70 e0       	ldi	r23, 0x00	; 0
    15e4:	82 e0       	ldi	r24, 0x02	; 2
    15e6:	4b d2       	rcall	.+1174   	; 0x1a7e <nvm_read_byte>
		break;
#endif

#ifdef ADCB
	case ADC_CAL_ADCB:
		data = nvm_read_production_signature_row(ADCBCAL1);
    15e8:	c8 2e       	mov	r12, r24
    15ea:	d1 2c       	mov	r13, r1
    15ec:	64 e2       	ldi	r22, 0x24	; 36
    15ee:	70 e0       	ldi	r23, 0x00	; 0
    15f0:	82 e0       	ldi	r24, 0x02	; 2
    15f2:	45 d2       	rcall	.+1162   	; 0x1a7e <nvm_read_byte>
		data <<= 8;
		data |= nvm_read_production_signature_row(ADCBCAL0);
    15f4:	dc 2c       	mov	r13, r12
    15f6:	cc 24       	eor	r12, r12
    15f8:	c8 2a       	or	r12, r24

typedef uint8_t irqflags_t;

static inline irqflags_t cpu_irq_save(void)
{
	volatile irqflags_t flags = SREG;
    15fa:	8f b7       	in	r24, 0x3f	; 63
	cpu_irq_disable();
    15fc:	89 83       	std	Y+1, r24	; 0x01
	return flags;
    15fe:	f8 94       	cli
		Assert(0);
		return;
	}

	flags = cpu_irq_save();
	adc_enable_clock(adc);
    1600:	b9 80       	ldd	r11, Y+1	; 0x01
    1602:	c8 01       	movw	r24, r16
    1604:	bc db       	rcall	.-2184   	; 0xd7e <adc_enable_clock>
	enable = adc->CTRLA & ADC_ENABLE_bm;
    1606:	f8 01       	movw	r30, r16
    1608:	80 81       	ld	r24, Z

	adc->CTRLA = ADC_FLUSH_bm;
    160a:	92 e0       	ldi	r25, 0x02	; 2
    160c:	90 83       	st	Z, r25
	adc->CAL = cal;
    160e:	c4 86       	std	Z+12, r12	; 0x0c
    1610:	d5 86       	std	Z+13, r13	; 0x0d
	adc->CMP = conf->cmp;
    1612:	f7 01       	movw	r30, r14
    1614:	25 81       	ldd	r18, Z+5	; 0x05
    1616:	36 81       	ldd	r19, Z+6	; 0x06
    1618:	f8 01       	movw	r30, r16
    161a:	20 8f       	std	Z+24, r18	; 0x18
    161c:	31 8f       	std	Z+25, r19	; 0x19
	adc->REFCTRL = conf->refctrl;
    161e:	f7 01       	movw	r30, r14
    1620:	92 81       	ldd	r25, Z+2	; 0x02
    1622:	f8 01       	movw	r30, r16
    1624:	92 83       	std	Z+2, r25	; 0x02
	adc->PRESCALER = conf->prescaler;
    1626:	f7 01       	movw	r30, r14
    1628:	94 81       	ldd	r25, Z+4	; 0x04
    162a:	f8 01       	movw	r30, r16
    162c:	94 83       	std	Z+4, r25	; 0x04
	adc->EVCTRL = conf->evctrl;
    162e:	f7 01       	movw	r30, r14
    1630:	93 81       	ldd	r25, Z+3	; 0x03
    1632:	f8 01       	movw	r30, r16
    1634:	93 83       	std	Z+3, r25	; 0x03
	adc->CTRLB = conf->ctrlb;
    1636:	f7 01       	movw	r30, r14
    1638:	91 81       	ldd	r25, Z+1	; 0x01
    163a:	f8 01       	movw	r30, r16
    163c:	91 83       	std	Z+1, r25	; 0x01

	adc->CTRLA = enable | conf->ctrla;
    163e:	81 70       	andi	r24, 0x01	; 1
    1640:	f7 01       	movw	r30, r14
    1642:	90 81       	ld	r25, Z
    1644:	89 2b       	or	r24, r25
    1646:	f8 01       	movw	r30, r16

	adc_disable_clock(adc);
    1648:	80 83       	st	Z, r24
    164a:	c8 01       	movw	r24, r16
    164c:	b7 db       	rcall	.-2194   	; 0xdbc <adc_disable_clock>
}

static inline void cpu_irq_restore(irqflags_t flags)
{
	barrier();
	SREG = flags;
    164e:	bf be       	out	0x3f, r11	; 63

	cpu_irq_restore(flags);
}
    1650:	0f 90       	pop	r0
    1652:	df 91       	pop	r29
    1654:	cf 91       	pop	r28
    1656:	1f 91       	pop	r17
    1658:	0f 91       	pop	r16
    165a:	ff 90       	pop	r15
    165c:	ef 90       	pop	r14
    165e:	df 90       	pop	r13
    1660:	cf 90       	pop	r12
    1662:	bf 90       	pop	r11
    1664:	08 95       	ret

00001666 <adc_read_configuration>:
 *
 * \param adc Pointer to ADC module.
 * \param conf Pointer to ADC module configuration.
 */
void adc_read_configuration(ADC_t *adc, struct adc_config *conf)
{
    1666:	df 92       	push	r13
    1668:	ef 92       	push	r14
    166a:	ff 92       	push	r15
    166c:	0f 93       	push	r16
    166e:	1f 93       	push	r17
    1670:	cf 93       	push	r28
    1672:	df 93       	push	r29
    1674:	1f 92       	push	r1
    1676:	cd b7       	in	r28, 0x3d	; 61
    1678:	de b7       	in	r29, 0x3e	; 62
    167a:	8c 01       	movw	r16, r24
    167c:	7b 01       	movw	r14, r22

typedef uint8_t irqflags_t;

static inline irqflags_t cpu_irq_save(void)
{
	volatile irqflags_t flags = SREG;
    167e:	8f b7       	in	r24, 0x3f	; 63
    1680:	89 83       	std	Y+1, r24	; 0x01
	cpu_irq_disable();
    1682:	f8 94       	cli
	return flags;
    1684:	d9 80       	ldd	r13, Y+1	; 0x01
	irqflags_t flags = cpu_irq_save();

	adc_enable_clock(adc);
    1686:	c8 01       	movw	r24, r16
    1688:	7a db       	rcall	.-2316   	; 0xd7e <adc_enable_clock>

	conf->ctrla = adc->CTRLA & ADC_DMASEL_gm;
    168a:	f8 01       	movw	r30, r16
    168c:	80 81       	ld	r24, Z
    168e:	80 7c       	andi	r24, 0xC0	; 192
    1690:	f7 01       	movw	r30, r14
    1692:	80 83       	st	Z, r24

	conf->cmp = adc->CMP;
    1694:	f8 01       	movw	r30, r16
    1696:	80 8d       	ldd	r24, Z+24	; 0x18
    1698:	91 8d       	ldd	r25, Z+25	; 0x19
    169a:	f7 01       	movw	r30, r14
    169c:	85 83       	std	Z+5, r24	; 0x05
    169e:	96 83       	std	Z+6, r25	; 0x06
	conf->refctrl = adc->REFCTRL;
    16a0:	f8 01       	movw	r30, r16
    16a2:	82 81       	ldd	r24, Z+2	; 0x02
    16a4:	f7 01       	movw	r30, r14
    16a6:	82 83       	std	Z+2, r24	; 0x02
	conf->prescaler = adc->PRESCALER;
    16a8:	f8 01       	movw	r30, r16
    16aa:	84 81       	ldd	r24, Z+4	; 0x04
    16ac:	f7 01       	movw	r30, r14
    16ae:	84 83       	std	Z+4, r24	; 0x04
	conf->evctrl = adc->EVCTRL;
    16b0:	f8 01       	movw	r30, r16
    16b2:	83 81       	ldd	r24, Z+3	; 0x03
    16b4:	f7 01       	movw	r30, r14
    16b6:	83 83       	std	Z+3, r24	; 0x03
	conf->ctrlb = adc->CTRLB;
    16b8:	f8 01       	movw	r30, r16
    16ba:	81 81       	ldd	r24, Z+1	; 0x01
    16bc:	f7 01       	movw	r30, r14
    16be:	81 83       	std	Z+1, r24	; 0x01

	adc_disable_clock(adc);
    16c0:	c8 01       	movw	r24, r16
    16c2:	7c db       	rcall	.-2312   	; 0xdbc <adc_disable_clock>
}

static inline void cpu_irq_restore(irqflags_t flags)
{
	barrier();
	SREG = flags;
    16c4:	df be       	out	0x3f, r13	; 63

	cpu_irq_restore(flags);
}
    16c6:	0f 90       	pop	r0
    16c8:	df 91       	pop	r29
    16ca:	cf 91       	pop	r28
    16cc:	1f 91       	pop	r17
    16ce:	0f 91       	pop	r16
    16d0:	ff 90       	pop	r15
    16d2:	ef 90       	pop	r14
    16d4:	df 90       	pop	r13
    16d6:	08 95       	ret

000016d8 <adcch_write_configuration>:
 * is called if callbacks are enabled and interrupts are enabled in the
 * channel configuration.
 */
void adcch_write_configuration(ADC_t *adc, uint8_t ch_mask,
		const struct adc_channel_config *ch_conf)
{
    16d8:	af 92       	push	r10
    16da:	bf 92       	push	r11
    16dc:	cf 92       	push	r12
    16de:	df 92       	push	r13
    16e0:	ef 92       	push	r14
    16e2:	ff 92       	push	r15
    16e4:	0f 93       	push	r16
    16e6:	1f 93       	push	r17
    16e8:	cf 93       	push	r28
    16ea:	df 93       	push	r29
    16ec:	1f 92       	push	r1
    16ee:	cd b7       	in	r28, 0x3d	; 61
    16f0:	de b7       	in	r29, 0x3e	; 62
    16f2:	6c 01       	movw	r12, r24
    16f4:	b6 2e       	mov	r11, r22
    16f6:	7a 01       	movw	r14, r20
		index += 4;
		ch_mask >>= 4;
	}
#endif
#if ADC_NR_OF_CHANNELS > 2
	if (!(ch_mask & 0x03)) {
    16f8:	86 2f       	mov	r24, r22
    16fa:	83 70       	andi	r24, 0x03	; 3
    16fc:	29 f4       	brne	.+10     	; 0x1708 <adcch_write_configuration+0x30>
		index += 2;
		ch_mask >>= 2;
    16fe:	96 2f       	mov	r25, r22
    1700:	96 95       	lsr	r25
    1702:	96 95       	lsr	r25
		ch_mask >>= 4;
	}
#endif
#if ADC_NR_OF_CHANNELS > 2
	if (!(ch_mask & 0x03)) {
		index += 2;
    1704:	82 e0       	ldi	r24, 0x02	; 2
    1706:	02 c0       	rjmp	.+4      	; 0x170c <adcch_write_configuration+0x34>
		index += 4;
		ch_mask >>= 4;
	}
#endif
#if ADC_NR_OF_CHANNELS > 2
	if (!(ch_mask & 0x03)) {
    1708:	96 2f       	mov	r25, r22
 * \return Pointer to ADC channel
 */
__always_inline static  ADC_CH_t *adc_get_channel(
		ADC_t *adc, uint8_t ch_mask)
{
	uint8_t index = 0;
    170a:	80 e0       	ldi	r24, 0x00	; 0
		index += 2;
		ch_mask >>= 2;
	}
#endif
#if ADC_NR_OF_CHANNELS > 1
	if (!(ch_mask & 0x01)) {
    170c:	90 ff       	sbrs	r25, 0
		index++;
    170e:	8f 5f       	subi	r24, 0xFF	; 255
	}
#endif

	return (ADC_CH_t *)(&adc->CH0 + index);
    1710:	86 01       	movw	r16, r12
    1712:	00 5e       	subi	r16, 0xE0	; 224
    1714:	1f 4f       	sbci	r17, 0xFF	; 255
    1716:	98 e0       	ldi	r25, 0x08	; 8
    1718:	89 9f       	mul	r24, r25
    171a:	00 0d       	add	r16, r0
    171c:	11 1d       	adc	r17, r1
    171e:	11 24       	eor	r1, r1

typedef uint8_t irqflags_t;

static inline irqflags_t cpu_irq_save(void)
{
	volatile irqflags_t flags = SREG;
    1720:	8f b7       	in	r24, 0x3f	; 63
    1722:	89 83       	std	Y+1, r24	; 0x01
	cpu_irq_disable();
    1724:	f8 94       	cli
	return flags;
    1726:	a9 80       	ldd	r10, Y+1	; 0x01
			return;
		}
	}
#endif

	adc_enable_clock(adc);
    1728:	c6 01       	movw	r24, r12
    172a:	29 db       	rcall	.-2478   	; 0xd7e <adc_enable_clock>
	adc_ch->CTRL = ch_conf->ctrl;
    172c:	f7 01       	movw	r30, r14
    172e:	80 81       	ld	r24, Z
    1730:	f8 01       	movw	r30, r16
    1732:	80 83       	st	Z, r24
	adc_ch->INTCTRL = ch_conf->intctrl;
    1734:	f7 01       	movw	r30, r14
    1736:	82 81       	ldd	r24, Z+2	; 0x02
    1738:	f8 01       	movw	r30, r16
    173a:	82 83       	std	Z+2, r24	; 0x02
	adc_ch->MUXCTRL = ch_conf->muxctrl;
    173c:	f7 01       	movw	r30, r14
    173e:	81 81       	ldd	r24, Z+1	; 0x01
    1740:	f8 01       	movw	r30, r16
    1742:	81 83       	std	Z+1, r24	; 0x01
	if (ch_mask & ADC_CH0) {
    1744:	b0 fe       	sbrs	r11, 0
    1746:	04 c0       	rjmp	.+8      	; 0x1750 <adcch_write_configuration+0x78>
		/* USB devices has channel scan available on ADC channel 0 */
		adc_ch->SCAN = ch_conf->scan;
    1748:	f7 01       	movw	r30, r14
    174a:	83 81       	ldd	r24, Z+3	; 0x03
    174c:	f8 01       	movw	r30, r16
    174e:	86 83       	std	Z+6, r24	; 0x06
	}
	adc_disable_clock(adc);
    1750:	c6 01       	movw	r24, r12
    1752:	34 db       	rcall	.-2456   	; 0xdbc <adc_disable_clock>
}

static inline void cpu_irq_restore(irqflags_t flags)
{
	barrier();
	SREG = flags;
    1754:	af be       	out	0x3f, r10	; 63

	cpu_irq_restore(flags);
}
    1756:	0f 90       	pop	r0
    1758:	df 91       	pop	r29
    175a:	cf 91       	pop	r28
    175c:	1f 91       	pop	r17
    175e:	0f 91       	pop	r16
    1760:	ff 90       	pop	r15
    1762:	ef 90       	pop	r14
    1764:	df 90       	pop	r13
    1766:	cf 90       	pop	r12
    1768:	bf 90       	pop	r11
    176a:	af 90       	pop	r10
    176c:	08 95       	ret

0000176e <adcch_read_configuration>:
 * can be given in mask)
 * \param ch_conf Pointer to ADC channel configuration.
 */
void adcch_read_configuration(ADC_t *adc, uint8_t ch_mask,
		struct adc_channel_config *ch_conf)
{
    176e:	af 92       	push	r10
    1770:	bf 92       	push	r11
    1772:	cf 92       	push	r12
    1774:	df 92       	push	r13
    1776:	ef 92       	push	r14
    1778:	ff 92       	push	r15
    177a:	0f 93       	push	r16
    177c:	1f 93       	push	r17
    177e:	cf 93       	push	r28
    1780:	df 93       	push	r29
    1782:	1f 92       	push	r1
    1784:	cd b7       	in	r28, 0x3d	; 61
    1786:	de b7       	in	r29, 0x3e	; 62
    1788:	6c 01       	movw	r12, r24
    178a:	b6 2e       	mov	r11, r22
    178c:	7a 01       	movw	r14, r20
		index += 4;
		ch_mask >>= 4;
	}
#endif
#if ADC_NR_OF_CHANNELS > 2
	if (!(ch_mask & 0x03)) {
    178e:	86 2f       	mov	r24, r22
    1790:	83 70       	andi	r24, 0x03	; 3
    1792:	29 f4       	brne	.+10     	; 0x179e <adcch_read_configuration+0x30>
		index += 2;
		ch_mask >>= 2;
    1794:	96 2f       	mov	r25, r22
    1796:	96 95       	lsr	r25
    1798:	96 95       	lsr	r25
		ch_mask >>= 4;
	}
#endif
#if ADC_NR_OF_CHANNELS > 2
	if (!(ch_mask & 0x03)) {
		index += 2;
    179a:	82 e0       	ldi	r24, 0x02	; 2
    179c:	02 c0       	rjmp	.+4      	; 0x17a2 <adcch_read_configuration+0x34>
		index += 4;
		ch_mask >>= 4;
	}
#endif
#if ADC_NR_OF_CHANNELS > 2
	if (!(ch_mask & 0x03)) {
    179e:	96 2f       	mov	r25, r22
 * \return Pointer to ADC channel
 */
__always_inline static  ADC_CH_t *adc_get_channel(
		ADC_t *adc, uint8_t ch_mask)
{
	uint8_t index = 0;
    17a0:	80 e0       	ldi	r24, 0x00	; 0
		index += 2;
		ch_mask >>= 2;
	}
#endif
#if ADC_NR_OF_CHANNELS > 1
	if (!(ch_mask & 0x01)) {
    17a2:	90 ff       	sbrs	r25, 0
		index++;
    17a4:	8f 5f       	subi	r24, 0xFF	; 255
	}
#endif

	return (ADC_CH_t *)(&adc->CH0 + index);
    17a6:	86 01       	movw	r16, r12
    17a8:	00 5e       	subi	r16, 0xE0	; 224
    17aa:	1f 4f       	sbci	r17, 0xFF	; 255
    17ac:	98 e0       	ldi	r25, 0x08	; 8
    17ae:	89 9f       	mul	r24, r25
    17b0:	00 0d       	add	r16, r0
    17b2:	11 1d       	adc	r17, r1
    17b4:	11 24       	eor	r1, r1

typedef uint8_t irqflags_t;

static inline irqflags_t cpu_irq_save(void)
{
	volatile irqflags_t flags = SREG;
    17b6:	8f b7       	in	r24, 0x3f	; 63
    17b8:	89 83       	std	Y+1, r24	; 0x01
	cpu_irq_disable();
    17ba:	f8 94       	cli
	return flags;
    17bc:	a9 80       	ldd	r10, Y+1	; 0x01

	adc_ch = adc_get_channel(adc, ch_mask);

	flags = cpu_irq_save();

	adc_enable_clock(adc);
    17be:	c6 01       	movw	r24, r12
    17c0:	de da       	rcall	.-2628   	; 0xd7e <adc_enable_clock>
	ch_conf->ctrl = adc_ch->CTRL;
    17c2:	f8 01       	movw	r30, r16
    17c4:	80 81       	ld	r24, Z
    17c6:	f7 01       	movw	r30, r14
    17c8:	80 83       	st	Z, r24
	ch_conf->intctrl = adc_ch->INTCTRL;
    17ca:	f8 01       	movw	r30, r16
    17cc:	82 81       	ldd	r24, Z+2	; 0x02
    17ce:	f7 01       	movw	r30, r14
    17d0:	82 83       	std	Z+2, r24	; 0x02
	ch_conf->muxctrl = adc_ch->MUXCTRL;
    17d2:	f8 01       	movw	r30, r16
    17d4:	81 81       	ldd	r24, Z+1	; 0x01
    17d6:	f7 01       	movw	r30, r14
    17d8:	81 83       	std	Z+1, r24	; 0x01
	if (ch_mask & ADC_CH0) {
    17da:	b0 fe       	sbrs	r11, 0
    17dc:	04 c0       	rjmp	.+8      	; 0x17e6 <adcch_read_configuration+0x78>
		/* USB devices has channel scan available on ADC channel 0 */
		ch_conf->scan = adc_ch->SCAN;
    17de:	f8 01       	movw	r30, r16
    17e0:	86 81       	ldd	r24, Z+6	; 0x06
    17e2:	f7 01       	movw	r30, r14
    17e4:	83 83       	std	Z+3, r24	; 0x03
	}
	adc_disable_clock(adc);
    17e6:	c6 01       	movw	r24, r12
    17e8:	e9 da       	rcall	.-2606   	; 0xdbc <adc_disable_clock>
}

static inline void cpu_irq_restore(irqflags_t flags)
{
	barrier();
	SREG = flags;
    17ea:	af be       	out	0x3f, r10	; 63

	cpu_irq_restore(flags);
}
    17ec:	0f 90       	pop	r0
    17ee:	df 91       	pop	r29
    17f0:	cf 91       	pop	r28
    17f2:	1f 91       	pop	r17
    17f4:	0f 91       	pop	r16
    17f6:	ff 90       	pop	r15
    17f8:	ef 90       	pop	r14
    17fa:	df 90       	pop	r13
    17fc:	cf 90       	pop	r12
    17fe:	bf 90       	pop	r11
    1800:	af 90       	pop	r10
    1802:	08 95       	ret

00001804 <usart_spi_init>:
		*data = usart_spi_transmit(usart, CONFIG_USART_SPI_DUMMY);
		len--;
		data++;
 	}
	return STATUS_OK;
}
    1804:	80 3a       	cpi	r24, 0xA0	; 160
    1806:	28 e0       	ldi	r18, 0x08	; 8
    1808:	92 07       	cpc	r25, r18
    180a:	21 f4       	brne	.+8      	; 0x1814 <usart_spi_init+0x10>
    180c:	60 e1       	ldi	r22, 0x10	; 16
    180e:	83 e0       	ldi	r24, 0x03	; 3
    1810:	0b c1       	rjmp	.+534    	; 0x1a28 <sysclk_enable_module>
    1812:	08 95       	ret
    1814:	80 3b       	cpi	r24, 0xB0	; 176
    1816:	28 e0       	ldi	r18, 0x08	; 8
    1818:	92 07       	cpc	r25, r18
    181a:	21 f4       	brne	.+8      	; 0x1824 <usart_spi_init+0x20>
    181c:	60 e2       	ldi	r22, 0x20	; 32
    181e:	83 e0       	ldi	r24, 0x03	; 3
    1820:	03 c1       	rjmp	.+518    	; 0x1a28 <sysclk_enable_module>
    1822:	08 95       	ret
    1824:	80 3a       	cpi	r24, 0xA0	; 160
    1826:	29 e0       	ldi	r18, 0x09	; 9
    1828:	92 07       	cpc	r25, r18
    182a:	21 f4       	brne	.+8      	; 0x1834 <usart_spi_init+0x30>
    182c:	60 e1       	ldi	r22, 0x10	; 16
    182e:	84 e0       	ldi	r24, 0x04	; 4
    1830:	fb c0       	rjmp	.+502    	; 0x1a28 <sysclk_enable_module>
    1832:	08 95       	ret
    1834:	80 3b       	cpi	r24, 0xB0	; 176
    1836:	29 e0       	ldi	r18, 0x09	; 9
    1838:	92 07       	cpc	r25, r18
    183a:	21 f4       	brne	.+8      	; 0x1844 <usart_spi_init+0x40>
    183c:	60 e2       	ldi	r22, 0x20	; 32
    183e:	84 e0       	ldi	r24, 0x04	; 4
    1840:	f3 c0       	rjmp	.+486    	; 0x1a28 <sysclk_enable_module>
    1842:	08 95       	ret
    1844:	80 3a       	cpi	r24, 0xA0	; 160
    1846:	2a e0       	ldi	r18, 0x0A	; 10
    1848:	92 07       	cpc	r25, r18
    184a:	21 f4       	brne	.+8      	; 0x1854 <usart_spi_init+0x50>
    184c:	60 e1       	ldi	r22, 0x10	; 16
    184e:	85 e0       	ldi	r24, 0x05	; 5
    1850:	eb c0       	rjmp	.+470    	; 0x1a28 <sysclk_enable_module>
    1852:	08 95       	ret
    1854:	80 3a       	cpi	r24, 0xA0	; 160
    1856:	9b 40       	sbci	r25, 0x0B	; 11
    1858:	19 f4       	brne	.+6      	; 0x1860 <usart_spi_init+0x5c>
    185a:	60 e1       	ldi	r22, 0x10	; 16
    185c:	86 e0       	ldi	r24, 0x06	; 6
    185e:	e4 c0       	rjmp	.+456    	; 0x1a28 <sysclk_enable_module>
    1860:	08 95       	ret

00001862 <usart_spi_setup_device>:
    1862:	0f 93       	push	r16
    1864:	1f 93       	push	r17
    1866:	cf 93       	push	r28
    1868:	df 93       	push	r29
    186a:	00 d0       	rcall	.+0      	; 0x186c <usart_spi_setup_device+0xa>
    186c:	00 d0       	rcall	.+0      	; 0x186e <usart_spi_setup_device+0xc>
    186e:	cd b7       	in	r28, 0x3d	; 61
    1870:	de b7       	in	r29, 0x3e	; 62
    1872:	09 83       	std	Y+1, r16	; 0x01
    1874:	1a 83       	std	Y+2, r17	; 0x02
    1876:	2b 83       	std	Y+3, r18	; 0x03
    1878:	3c 83       	std	Y+4, r19	; 0x04
    187a:	4d 83       	std	Y+5, r20	; 0x05
    187c:	1e 82       	std	Y+6, r1	; 0x06
    187e:	be 01       	movw	r22, r28
    1880:	6f 5f       	subi	r22, 0xFF	; 255
    1882:	7f 4f       	sbci	r23, 0xFF	; 255
    1884:	16 db       	rcall	.-2516   	; 0xeb2 <usart_init_spi>
    1886:	26 96       	adiw	r28, 0x06	; 6
    1888:	cd bf       	out	0x3d, r28	; 61
    188a:	de bf       	out	0x3e, r29	; 62
    188c:	df 91       	pop	r29
    188e:	cf 91       	pop	r28
    1890:	1f 91       	pop	r17
    1892:	0f 91       	pop	r16
    1894:	08 95       	ret

00001896 <usart_spi_select_device>:

void usart_spi_select_device(USART_t *usart, struct usart_spi_device *device)
{
	ioport_set_pin_low(device->id);
    1896:	fb 01       	movw	r30, r22
    1898:	80 81       	ld	r24, Z
	return pin >> 3;
}

__always_inline static PORT_t *arch_ioport_port_to_base(ioport_port_t port)
{
	return (PORT_t *)((uintptr_t)IOPORT_BASE_ADDRESS +
    189a:	e8 2f       	mov	r30, r24
    189c:	e6 95       	lsr	r30
    189e:	e6 95       	lsr	r30
    18a0:	e6 95       	lsr	r30
    18a2:	40 e2       	ldi	r20, 0x20	; 32
    18a4:	e4 9f       	mul	r30, r20
    18a6:	f0 01       	movw	r30, r0
    18a8:	11 24       	eor	r1, r1
    18aa:	fa 5f       	subi	r31, 0xFA	; 250
}

__always_inline static ioport_port_mask_t arch_ioport_pin_to_mask(
		ioport_pin_t pin)
{
	return 1U << (pin & 0x07);
    18ac:	87 70       	andi	r24, 0x07	; 7
    18ae:	21 e0       	ldi	r18, 0x01	; 1
    18b0:	30 e0       	ldi	r19, 0x00	; 0
    18b2:	a9 01       	movw	r20, r18
    18b4:	02 c0       	rjmp	.+4      	; 0x18ba <usart_spi_select_device+0x24>
    18b6:	44 0f       	add	r20, r20
    18b8:	55 1f       	adc	r21, r21
    18ba:	8a 95       	dec	r24
    18bc:	e2 f7       	brpl	.-8      	; 0x18b6 <usart_spi_select_device+0x20>
	PORT_t *base = arch_ioport_pin_to_base(pin);

	if (level) {
		base->OUTSET = arch_ioport_pin_to_mask(pin);
	} else {
		base->OUTCLR = arch_ioport_pin_to_mask(pin);
    18be:	46 83       	std	Z+6, r20	; 0x06
    18c0:	08 95       	ret

000018c2 <usart_spi_deselect_device>:
}

void usart_spi_deselect_device(USART_t *usart, struct usart_spi_device *device)
{
	ioport_set_pin_high(device->id);
    18c2:	fb 01       	movw	r30, r22
    18c4:	80 81       	ld	r24, Z
	return pin >> 3;
}

__always_inline static PORT_t *arch_ioport_port_to_base(ioport_port_t port)
{
	return (PORT_t *)((uintptr_t)IOPORT_BASE_ADDRESS +
    18c6:	e8 2f       	mov	r30, r24
    18c8:	e6 95       	lsr	r30
    18ca:	e6 95       	lsr	r30
    18cc:	e6 95       	lsr	r30
    18ce:	40 e2       	ldi	r20, 0x20	; 32
    18d0:	e4 9f       	mul	r30, r20
    18d2:	f0 01       	movw	r30, r0
    18d4:	11 24       	eor	r1, r1
    18d6:	fa 5f       	subi	r31, 0xFA	; 250
}

__always_inline static ioport_port_mask_t arch_ioport_pin_to_mask(
		ioport_pin_t pin)
{
	return 1U << (pin & 0x07);
    18d8:	87 70       	andi	r24, 0x07	; 7
    18da:	21 e0       	ldi	r18, 0x01	; 1
    18dc:	30 e0       	ldi	r19, 0x00	; 0
    18de:	a9 01       	movw	r20, r18
    18e0:	02 c0       	rjmp	.+4      	; 0x18e6 <usart_spi_deselect_device+0x24>
    18e2:	44 0f       	add	r20, r20
    18e4:	55 1f       	adc	r21, r21
    18e6:	8a 95       	dec	r24
    18e8:	e2 f7       	brpl	.-8      	; 0x18e2 <usart_spi_deselect_device+0x20>
		bool level)
{
	PORT_t *base = arch_ioport_pin_to_base(pin);

	if (level) {
		base->OUTSET = arch_ioport_pin_to_mask(pin);
    18ea:	45 83       	std	Z+5, r20	; 0x05
    18ec:	08 95       	ret

000018ee <gfx_mono_set_framebuffer>:
	gfx_coord_t *framebuffer_pt = fbpointer +
			((page * GFX_MONO_LCD_WIDTH) + column);
	do {
		*data++ = *framebuffer_pt++;
	} while (--width > 0);
}
    18ee:	80 93 70 22 	sts	0x2270, r24	; 0x802270 <fbpointer>
    18f2:	90 93 71 22 	sts	0x2271, r25	; 0x802271 <fbpointer+0x1>
    18f6:	08 95       	ret

000018f8 <gfx_mono_framebuffer_put_byte>:
\endcode
 */
void gfx_mono_framebuffer_put_byte(gfx_coord_t page, gfx_coord_t column,
		uint8_t data)
{
	*(fbpointer + (page * GFX_MONO_LCD_WIDTH) + column) = data;
    18f8:	20 91 70 22 	lds	r18, 0x2270	; 0x802270 <fbpointer>
    18fc:	30 91 71 22 	lds	r19, 0x2271	; 0x802271 <fbpointer+0x1>
    1900:	90 e8       	ldi	r25, 0x80	; 128
    1902:	89 9f       	mul	r24, r25
    1904:	20 0d       	add	r18, r0
    1906:	31 1d       	adc	r19, r1
    1908:	11 24       	eor	r1, r1
    190a:	f9 01       	movw	r30, r18
    190c:	e6 0f       	add	r30, r22
    190e:	f1 1d       	adc	r31, r1
    1910:	40 83       	st	Z, r20
    1912:	08 95       	ret

00001914 <gfx_mono_framebuffer_get_byte>:
	data = gfx_mono_framebuffer_get_byte(0, 0);
\endcode
 */
uint8_t gfx_mono_framebuffer_get_byte(gfx_coord_t page, gfx_coord_t column)
{
	return *(fbpointer + (page * GFX_MONO_LCD_WIDTH) + column);
    1914:	20 91 70 22 	lds	r18, 0x2270	; 0x802270 <fbpointer>
    1918:	30 91 71 22 	lds	r19, 0x2271	; 0x802271 <fbpointer+0x1>
    191c:	90 e8       	ldi	r25, 0x80	; 128
    191e:	89 9f       	mul	r24, r25
    1920:	20 0d       	add	r18, r0
    1922:	31 1d       	adc	r19, r1
    1924:	11 24       	eor	r1, r1
    1926:	f9 01       	movw	r30, r18
    1928:	e6 0f       	add	r30, r22
    192a:	f1 1d       	adc	r31, r1
}
    192c:	80 81       	ld	r24, Z
    192e:	08 95       	ret

00001930 <gfx_mono_generic_draw_horizontal_line>:
	gfx_mono_draw_horizontal_line(x, y, width, color);
	gfx_mono_draw_horizontal_line(x, y + height - 1, width, color);

	gfx_mono_draw_vertical_line(x, y, height, color);
	gfx_mono_draw_vertical_line(x + width - 1, y, height, color);
}
    1930:	ff 92       	push	r15
    1932:	0f 93       	push	r16
    1934:	1f 93       	push	r17
    1936:	cf 93       	push	r28
    1938:	df 93       	push	r29
    193a:	e4 2f       	mov	r30, r20
    193c:	f0 e0       	ldi	r31, 0x00	; 0
    193e:	e8 0f       	add	r30, r24
    1940:	f1 1d       	adc	r31, r1
    1942:	e1 38       	cpi	r30, 0x81	; 129
    1944:	f1 05       	cpc	r31, r1
    1946:	1c f0       	brlt	.+6      	; 0x194e <gfx_mono_generic_draw_horizontal_line+0x1e>
    1948:	c0 e8       	ldi	r28, 0x80	; 128
    194a:	4c 2f       	mov	r20, r28
    194c:	48 1b       	sub	r20, r24
    194e:	44 23       	and	r20, r20
    1950:	09 f4       	brne	.+2      	; 0x1954 <gfx_mono_generic_draw_horizontal_line+0x24>
    1952:	4a c0       	rjmp	.+148    	; 0x19e8 <gfx_mono_generic_draw_horizontal_line+0xb8>
    1954:	d6 2f       	mov	r29, r22
    1956:	d6 95       	lsr	r29
    1958:	d6 95       	lsr	r29
    195a:	d6 95       	lsr	r29
    195c:	70 e0       	ldi	r23, 0x00	; 0
    195e:	98 e0       	ldi	r25, 0x08	; 8
    1960:	d9 9f       	mul	r29, r25
    1962:	60 19       	sub	r22, r0
    1964:	71 09       	sbc	r23, r1
    1966:	11 24       	eor	r1, r1
    1968:	e1 e0       	ldi	r30, 0x01	; 1
    196a:	f0 e0       	ldi	r31, 0x00	; 0
    196c:	df 01       	movw	r26, r30
    196e:	02 c0       	rjmp	.+4      	; 0x1974 <gfx_mono_generic_draw_horizontal_line+0x44>
    1970:	aa 0f       	add	r26, r26
    1972:	bb 1f       	adc	r27, r27
    1974:	6a 95       	dec	r22
    1976:	e2 f7       	brpl	.-8      	; 0x1970 <gfx_mono_generic_draw_horizontal_line+0x40>
    1978:	fa 2e       	mov	r15, r26
    197a:	21 30       	cpi	r18, 0x01	; 1
    197c:	21 f0       	breq	.+8      	; 0x1986 <gfx_mono_generic_draw_horizontal_line+0x56>
    197e:	98 f0       	brcs	.+38     	; 0x19a6 <gfx_mono_generic_draw_horizontal_line+0x76>
    1980:	22 30       	cpi	r18, 0x02	; 2
    1982:	19 f1       	breq	.+70     	; 0x19ca <gfx_mono_generic_draw_horizontal_line+0x9a>
    1984:	31 c0       	rjmp	.+98     	; 0x19e8 <gfx_mono_generic_draw_horizontal_line+0xb8>
    1986:	c4 2f       	mov	r28, r20
    1988:	1f ef       	ldi	r17, 0xFF	; 255
    198a:	18 0f       	add	r17, r24
    198c:	01 2f       	mov	r16, r17
    198e:	0c 0f       	add	r16, r28
    1990:	60 2f       	mov	r22, r16
    1992:	8d 2f       	mov	r24, r29
    1994:	d2 d9       	rcall	.-3164   	; 0xd3a <gfx_mono_st7565r_get_byte>
    1996:	4f 2d       	mov	r20, r15
    1998:	48 2b       	or	r20, r24
    199a:	60 2f       	mov	r22, r16
    199c:	8d 2f       	mov	r24, r29
    199e:	ae d8       	rcall	.-3748   	; 0xafc <gfx_mono_st7565r_put_byte>
    19a0:	c1 50       	subi	r28, 0x01	; 1
    19a2:	a1 f7       	brne	.-24     	; 0x198c <gfx_mono_generic_draw_horizontal_line+0x5c>
    19a4:	21 c0       	rjmp	.+66     	; 0x19e8 <gfx_mono_generic_draw_horizontal_line+0xb8>
    19a6:	c4 2f       	mov	r28, r20
    19a8:	1f ef       	ldi	r17, 0xFF	; 255
    19aa:	18 0f       	add	r17, r24
    19ac:	fa 2e       	mov	r15, r26
    19ae:	f0 94       	com	r15
    19b0:	01 2f       	mov	r16, r17
    19b2:	0c 0f       	add	r16, r28
    19b4:	60 2f       	mov	r22, r16
    19b6:	8d 2f       	mov	r24, r29
    19b8:	c0 d9       	rcall	.-3200   	; 0xd3a <gfx_mono_st7565r_get_byte>
    19ba:	4f 2d       	mov	r20, r15
    19bc:	48 23       	and	r20, r24
    19be:	60 2f       	mov	r22, r16
    19c0:	8d 2f       	mov	r24, r29
    19c2:	9c d8       	rcall	.-3784   	; 0xafc <gfx_mono_st7565r_put_byte>
    19c4:	c1 50       	subi	r28, 0x01	; 1
    19c6:	a1 f7       	brne	.-24     	; 0x19b0 <gfx_mono_generic_draw_horizontal_line+0x80>
    19c8:	0f c0       	rjmp	.+30     	; 0x19e8 <gfx_mono_generic_draw_horizontal_line+0xb8>
    19ca:	c4 2f       	mov	r28, r20
    19cc:	1f ef       	ldi	r17, 0xFF	; 255
    19ce:	18 0f       	add	r17, r24
    19d0:	01 2f       	mov	r16, r17
    19d2:	0c 0f       	add	r16, r28
    19d4:	60 2f       	mov	r22, r16
    19d6:	8d 2f       	mov	r24, r29
    19d8:	b0 d9       	rcall	.-3232   	; 0xd3a <gfx_mono_st7565r_get_byte>
    19da:	4f 2d       	mov	r20, r15
    19dc:	48 27       	eor	r20, r24
    19de:	60 2f       	mov	r22, r16
    19e0:	8d 2f       	mov	r24, r29
    19e2:	8c d8       	rcall	.-3816   	; 0xafc <gfx_mono_st7565r_put_byte>
    19e4:	c1 50       	subi	r28, 0x01	; 1
    19e6:	a1 f7       	brne	.-24     	; 0x19d0 <gfx_mono_generic_draw_horizontal_line+0xa0>
    19e8:	df 91       	pop	r29
    19ea:	cf 91       	pop	r28
    19ec:	1f 91       	pop	r17
    19ee:	0f 91       	pop	r16
    19f0:	ff 90       	pop	r15
    19f2:	08 95       	ret

000019f4 <gfx_mono_generic_draw_filled_rect>:
 * \param  color       Pixel operation of the line
 */
void gfx_mono_generic_draw_filled_rect(gfx_coord_t x, gfx_coord_t y,
		gfx_coord_t width, gfx_coord_t height,
		enum gfx_mono_color color)
{
    19f4:	ff 92       	push	r15
    19f6:	0f 93       	push	r16
    19f8:	1f 93       	push	r17
    19fa:	cf 93       	push	r28
    19fc:	df 93       	push	r29
	if (height == 0) {
    19fe:	22 23       	and	r18, r18
    1a00:	69 f0       	breq	.+26     	; 0x1a1c <gfx_mono_generic_draw_filled_rect+0x28>
    1a02:	f4 2e       	mov	r15, r20
    1a04:	18 2f       	mov	r17, r24
    1a06:	c2 2f       	mov	r28, r18
		/* Nothing to do. Move along. */
		return;
	}

	while (height-- > 0) {
		gfx_mono_draw_horizontal_line(x, y + height, width, color);
    1a08:	df ef       	ldi	r29, 0xFF	; 255
    1a0a:	d6 0f       	add	r29, r22
    1a0c:	6d 2f       	mov	r22, r29
    1a0e:	6c 0f       	add	r22, r28
    1a10:	20 2f       	mov	r18, r16
    1a12:	4f 2d       	mov	r20, r15
    1a14:	81 2f       	mov	r24, r17
    1a16:	8c df       	rcall	.-232    	; 0x1930 <gfx_mono_generic_draw_horizontal_line>
    1a18:	c1 50       	subi	r28, 0x01	; 1
	if (height == 0) {
		/* Nothing to do. Move along. */
		return;
	}

	while (height-- > 0) {
    1a1a:	c1 f7       	brne	.-16     	; 0x1a0c <gfx_mono_generic_draw_filled_rect+0x18>
		gfx_mono_draw_horizontal_line(x, y + height, width, color);
	}
}
    1a1c:	df 91       	pop	r29
    1a1e:	cf 91       	pop	r28
    1a20:	1f 91       	pop	r17
    1a22:	0f 91       	pop	r16
    1a24:	ff 90       	pop	r15
    1a26:	08 95       	ret

00001a28 <sysclk_enable_module>:
	sysclk_rtcsrc_enable(CONFIG_RTC_SOURCE);
#endif
}

void sysclk_enable_module(enum sysclk_port_id port, uint8_t id)
{
    1a28:	cf 93       	push	r28
    1a2a:	df 93       	push	r29
    1a2c:	1f 92       	push	r1
    1a2e:	cd b7       	in	r28, 0x3d	; 61
    1a30:	de b7       	in	r29, 0x3e	; 62

typedef uint8_t irqflags_t;

static inline irqflags_t cpu_irq_save(void)
{
	volatile irqflags_t flags = SREG;
    1a32:	9f b7       	in	r25, 0x3f	; 63
    1a34:	99 83       	std	Y+1, r25	; 0x01
	cpu_irq_disable();
    1a36:	f8 94       	cli
	return flags;
    1a38:	99 81       	ldd	r25, Y+1	; 0x01
	irqflags_t flags = cpu_irq_save();

	*((uint8_t *)&PR.PRGEN + port) &= ~id;
    1a3a:	e8 2f       	mov	r30, r24
    1a3c:	f0 e0       	ldi	r31, 0x00	; 0
    1a3e:	e0 59       	subi	r30, 0x90	; 144
    1a40:	ff 4f       	sbci	r31, 0xFF	; 255
    1a42:	60 95       	com	r22
    1a44:	80 81       	ld	r24, Z
    1a46:	68 23       	and	r22, r24
    1a48:	60 83       	st	Z, r22
}

static inline void cpu_irq_restore(irqflags_t flags)
{
	barrier();
	SREG = flags;
    1a4a:	9f bf       	out	0x3f, r25	; 63

	cpu_irq_restore(flags);
}
    1a4c:	0f 90       	pop	r0
    1a4e:	df 91       	pop	r29
    1a50:	cf 91       	pop	r28
    1a52:	08 95       	ret

00001a54 <sysclk_disable_module>:

void sysclk_disable_module(enum sysclk_port_id port, uint8_t id)
{
    1a54:	cf 93       	push	r28
    1a56:	df 93       	push	r29
    1a58:	1f 92       	push	r1
    1a5a:	cd b7       	in	r28, 0x3d	; 61
    1a5c:	de b7       	in	r29, 0x3e	; 62

typedef uint8_t irqflags_t;

static inline irqflags_t cpu_irq_save(void)
{
	volatile irqflags_t flags = SREG;
    1a5e:	9f b7       	in	r25, 0x3f	; 63
    1a60:	99 83       	std	Y+1, r25	; 0x01
	cpu_irq_disable();
    1a62:	f8 94       	cli
	return flags;
    1a64:	99 81       	ldd	r25, Y+1	; 0x01
	irqflags_t flags = cpu_irq_save();

	*((uint8_t *)&PR.PRGEN + port) |= id;
    1a66:	e8 2f       	mov	r30, r24
    1a68:	f0 e0       	ldi	r31, 0x00	; 0
    1a6a:	e0 59       	subi	r30, 0x90	; 144
    1a6c:	ff 4f       	sbci	r31, 0xFF	; 255
    1a6e:	80 81       	ld	r24, Z
    1a70:	68 2b       	or	r22, r24
    1a72:	60 83       	st	Z, r22
}

static inline void cpu_irq_restore(irqflags_t flags)
{
	barrier();
	SREG = flags;
    1a74:	9f bf       	out	0x3f, r25	; 63

	cpu_irq_restore(flags);
}
    1a76:	0f 90       	pop	r0
    1a78:	df 91       	pop	r29
    1a7a:	cf 91       	pop	r28
    1a7c:	08 95       	ret

00001a7e <nvm_read_byte>:
#endif

#ifndef __DOXYGEN__
	PUBLIC_FUNCTION(nvm_read_byte)
#if defined(__GNUC__)
	lds r20, NVM_CMD          ; Store NVM command register
    1a7e:	40 91 ca 01 	lds	r20, 0x01CA	; 0x8001ca <__TEXT_REGION_LENGTH__+0x7be1ca>
	mov ZL, r22               ; Load byte index into low byte of Z.
    1a82:	e6 2f       	mov	r30, r22
	mov ZH, r23               ; Load high byte into Z.
    1a84:	f7 2f       	mov	r31, r23
	sts NVM_CMD, r24          ; Load prepared command into NVM Command register.
    1a86:	80 93 ca 01 	sts	0x01CA, r24	; 0x8001ca <__TEXT_REGION_LENGTH__+0x7be1ca>
	lpm r24, Z                ; Perform an LPM to read out byte
    1a8a:	84 91       	lpm	r24, Z
	sts NVM_CMD, r20          ; Restore NVM command register
    1a8c:	40 93 ca 01 	sts	0x01CA, r20	; 0x8001ca <__TEXT_REGION_LENGTH__+0x7be1ca>
	sts NVM_CMD, r16          ; Load prepared command into NVM Command register.
	lpm r16, Z                ; Perform an LPM to read out byte
	sts NVM_CMD, r20          ; Restore NVM command register
#endif

	ret
    1a90:	08 95       	ret

00001a92 <gfx_mono_draw_char>:
 * \param y        Y coordinate on screen.
 * \param font     Font to draw character in
 */
void gfx_mono_draw_char(const char c, const gfx_coord_t x, const gfx_coord_t y,
		const struct font *font)
{
    1a92:	af 92       	push	r10
    1a94:	bf 92       	push	r11
    1a96:	cf 92       	push	r12
    1a98:	df 92       	push	r13
    1a9a:	ef 92       	push	r14
    1a9c:	ff 92       	push	r15
    1a9e:	0f 93       	push	r16
    1aa0:	1f 93       	push	r17
    1aa2:	cf 93       	push	r28
    1aa4:	df 93       	push	r29
    1aa6:	c8 2f       	mov	r28, r24
    1aa8:	e6 2e       	mov	r14, r22
    1aaa:	b4 2e       	mov	r11, r20
    1aac:	69 01       	movw	r12, r18
	gfx_mono_draw_filled_rect(x, y, font->width, font->height,
    1aae:	00 e0       	ldi	r16, 0x00	; 0
    1ab0:	f9 01       	movw	r30, r18
    1ab2:	24 81       	ldd	r18, Z+4	; 0x04
    1ab4:	43 81       	ldd	r20, Z+3	; 0x03
    1ab6:	6b 2d       	mov	r22, r11
    1ab8:	8e 2d       	mov	r24, r14
    1aba:	9c df       	rcall	.-200    	; 0x19f4 <gfx_mono_generic_draw_filled_rect>
			GFX_PIXEL_CLR);

	switch (font->type) {
    1abc:	f6 01       	movw	r30, r12
    1abe:	80 81       	ld	r24, Z
    1ac0:	81 11       	cpse	r24, r1
    1ac2:	39 c0       	rjmp	.+114    	; 0x1b36 <gfx_mono_draw_char+0xa4>
	Assert(font != NULL);

	gfx_coord_t inc_x = x;
	gfx_coord_t inc_y = y;

	char_row_size = font->width / CONFIG_FONT_PIXELS_PER_BYTE;
    1ac4:	83 81       	ldd	r24, Z+3	; 0x03
    1ac6:	28 2f       	mov	r18, r24
    1ac8:	26 95       	lsr	r18
    1aca:	26 95       	lsr	r18
    1acc:	26 95       	lsr	r18
	if (font->width % CONFIG_FONT_PIXELS_PER_BYTE) {
    1ace:	87 70       	andi	r24, 0x07	; 7
    1ad0:	09 f0       	breq	.+2      	; 0x1ad4 <gfx_mono_draw_char+0x42>
		char_row_size++;
    1ad2:	2f 5f       	subi	r18, 0xFF	; 255
	}

	glyph_data_offset = char_row_size * font->height *
    1ad4:	f6 01       	movw	r30, r12
    1ad6:	a4 80       	ldd	r10, Z+4	; 0x04
			((uint8_t)ch - font->first_char);
	glyph_data = font->data.progmem + glyph_data_offset;
    1ad8:	8c 2f       	mov	r24, r28
    1ada:	90 e0       	ldi	r25, 0x00	; 0
    1adc:	35 81       	ldd	r19, Z+5	; 0x05
